:020000040000FA
:080000000002040000000000F2
:020000040000FA
:10040000EF8721000E7F22000E018800000000000F
:100410000C00070040D32E0001002000110007004F
:10042000000020000000E000020032000000020096
:1004300000000000F0E40200000000000040DA00CC
:100440000000FE004440A90040B621000000E0008A
:100450000300320000002000A00188004440A800F2
:100460000000060091018800800078000000EB0089
:1004700015003700E280400032A0B4009101BA00BC
:10048000E280400032A0B4009102BA00E280400055
:1004900032A0B4000002EB00472BDE00F507B200EB
:1004A000602CE10004003A000059EB008301E900F0
:1004B000FDFF3E00040037006128E100010032002A
:1004C0000082EB00040007001101BA000200E00006
:1004D000E8FF3A00000006003159BA008301E90044
:1004E0000C0032002159BA008301E90008003200F3
:1004F0000400E00003003A00E280400032A0B400B3
:10050000F5FF370011D9BA008301E900FAFF3A007C
:100510008100E800E180400032A0B4000000060045
:100520004C1B040001000000C61B04000100000079
:10053000241C040001000000FA0D0400010000006A
:10054000620E040001000000BE0E04000100000065
:10055000ACA7040000000000B6A7040000000000E3
:10056000D2A70400000000000AA50400000000005B
:1005700024A50400000000008CA604000000000078
:100580001AA5040000000000AAA504000000000055
:1005900094A6040000000000921C0400010000006A
:1005A000261D0400010000008C1D04000100000055
:1005B00020F30400000000003EF3040000000000EF
:1005C00056F30400000000006EF304000000000079
:1005D0007AF304000000000092F304000000000021
:1005E000EEF304000000000006F404000000000028
:1005F00032F404000000000052F404000000000087
:1006000098F4040000000000B8F4040000000000AA
:10061000DAF4040000000000FAF404000000000016
:1006200050F50400000000005CF50400000000002C
:1006300068F504000000000074F5040000000000EC
:1006400086F3040000000000DAC00400000000008F
:10065000F2C004000000000036C1040000000000E9
:1006600044C10400000000005CC104000000000060
:1006700078C1040000000000BEC1040000000000BA
:1006800002C204000000000048C204000000000094
:1006900080C2040000000000F0C20400000000005E
:1006A00010C30400000000002AC304000000000082
:1006B00050C30400000000007AC3040000000000E2
:1006C0009CC3040000000000CCC304000000000034
:1006D000F2C304000000000018C404000000000081
:1006E0003EC404000000000060C4040000000000DC
:1006F0007CC4040000000000B4C30400000000003B
:1007000088C4040000000000B6C40400000000001B
:10071000E4C404000000000012C504000000000052
:1007200032C50400000000001EF7040000000000B5
:100730003CF704000000000048F70400000000003F
:100740006AF704000000000076F7040000000000D3
:1007500082F704000000000006F80400000000001A
:100760001CF80400000000003CF804000000000039
:100770007EF80400000000008AF804000000000079
:1007800004F904000000000092F8040000000000DA
:100790009EF8040000000000BEF804000000000005
:1007A000C0F70400000000000040DA000000FE0076
:1007B0001004B100030035009001B10001003C00BD
:1007C0001000050000000500800078001104B10051
:1007D000030035009101B10001003C000050A00071
:1007E000000006001004B100070035009001B100C0
:1007F000040034007000B100030035009001B10026
:1008000001003C0010000500000005006900E10047
:10081000040035006D00E100030034000002B10067
:100820000100320000000500100005002002E20077
:1008300004003D002342AB00020032002302AB0063
:10084000FEFF32000040DA00FEFF37000A00FA0027
:1008500080017800E20F500028003E00D0BF8000E9
:10086000E10F500008003200802320000000E0006B
:100870000500320004232000252320004623200009
:100880008001780004003700042220002522200087
:100890004622200083222000144090000004E00043
:1008A000040035008009EB00144090000074A000A3
:1008B00010429800154090000028A30003003A0061
:1008C000154090000024A000904298008001EB00A9
:1008D00007003700154090000008A300FDFF32001C
:1008E00063C078000000FB00000B78008301E80083
:1008F000828F5100F7FF3A000800370030002000D7
:10090000B0BF9F00C3BF9F00D1BF9F00E2BF9F0049
:100910006A80570000C0DA006FB9970002007800C3
:100920000080FA00000006000A00FA001100200012
:10093000B1BF9F00C0BF9F006A80570000C0DA00AF
:100940004FB897000080FA00000006000A00FA0085
:1009500051002000B1BF9F00C0BF9F006A805700B8
:1009600000C0DA005FB897000080FA0000000600BF
:100970000A00FA00881F7800800178000000E0007B
:1009800029003A00D0BF8000E10F5000080032007B
:10099000802320000000E000050032000423200036
:1009A0002523200067232000800178000400370001
:1009B000042220002522200067222000832220001C
:1009C000144090000004E000040035008009EB00B2
:1009D000144090000074A000104298000002EB0048
:1009E0000C003700130A20001544780061406400B1
:1009F00002003A008301E900FBFF3A000402E8002C
:100A00009541780061C06100050032001700780050
:100A10008058780004035100820F5200F1FF3A0021
:100A2000060051000800370020002000A0BF9F00F2
:100A3000B3BF9F00C1BF9F00D2BF9F006C80570013
:100A400000C0DA005FB897004F0478000080FA0019
:100A500000000600889FBE0080047800E0BF800090
:100A60000000E00003003A00100007000000E00072
:100A70000A003500E0BF80000900E00002003A00F3
:100A800000047800060037000004780009004000E8
:100A9000060007000000E00001003D000084EB00BC
:100AA000080078004F04BE000000060080007800B7
:100AB0000000E00004003A00E07F2100E0BF880071
:100AC00001017800060037000081EB00E08721007B
:100AD000808F500002003E00E1BF88000001EB0063
:100AE0000200780000000600020AB900001BB900ED
:100AF0000200B800810042008100430000000600AF
:100B000003F0A200889FBE008A9FBE008C1F780061
:100B1000940207009B0233006450E1004F00320052
:100B20006420E1005200320003826C0007003B00A9
:100B30000905D0000306D000820F54000C065D00AA
:100B400002003900020032008901780003067800B3
:100B50008582550004003D000003FD008103FD0077
:100B60008502EA008B854200840F720002003B0080
:100B700060001000E08018006011B8000005EB0074
:100B80007A28E1000A00390006007800C75DDD0020
:100B9000F707B200878075002D0037008281710051
:100BA0000A017800610560008180D1000080D300D7
:100BB0008502E900F9FF3B000604400087844800F5
:100BC00002003B0060041400E0841C000988A300BC
:100BD000070032008A817100828171006101640026
:100BE0008904D1000884D3008B05E8001700370082
:100BF0000978A30013003A000B00E0001300340052
:100C00008B05E9000804440089844C000A44740000
:100C10000978A3000D003A000B00E0000700340043
:100C20008B05E9000804440089844C0001003A0067
:100C30000B0020000978A300F7FF32000001EB0051
:100C400002003700828171000A0178005D0207000E
:100C50000CF0A70001F0A000530237006420E1006F
:100C600002003A00838F6C00530233000801BE007B
:100C70000200BE004C023700889FBE008A9FBE0063
:100C80008C1F7800370207003E02330003866C0099
:100C90006450E1002E0032006420E1003300320095
:100CA0006150E1002F0032006120E100310032008C
:100CB00085855500EB07B0000900200008042000DE
:100CC000050037000804440089844C000A00310004
:100CD0000603430087834B000001530081815B00C2
:100CE000F8FF33000203BE000800A000080444001F
:100CF00089844C00F6FF3900C639DD00830173009A
:100D000001003200130020008904D1000884D300C0
:100D10000998A300050032000800A7000300A00006
:100D20008904D1000884D3008B05E8008904D10030
:100D30000884D3000001EB000281D20021020700E9
:100D400001F0A1000CF0A70001F0A000160237008E
:100D50006420E100180232000801BE000200BE005B
:100D6000F7FF37006120E100130232006000B80095
:100D7000F3FF37000000200001F82700F0FF3700E4
:100D8000889FBE008A9FBE00010578000100E00038
:100D90000400350008003C000000E00020003200A4
:100DA0000500370060001000E080180002003B00E2
:100DB00001F02C001A0037000004BE006011B800DA
:100DC0006B0920000982CF00020039000882CF00A1
:100DD0000441B000694252000E00320008003B009E
:100DE00082817100610164008904D1000884D3000C
:100DF0008B05E8000442E800F9FF3A0005003700DF
:100E00000804440089844C008B05E9000442E90091
:100E1000FBFF3A00EB0107000AF0A70001F0A00079
:100E20004F05BE004F04BE00000006000400200075
:100E30000A023700889FBE008A9FBE008C1F780080
:100E4000C8010700CF01330003866C006450E10045
:100E5000240032006420E100270032006150E100EC
:100E6000220032006120E100210032008B85420027
:100E7000EB07B1000134B800003AB80008044200A2
:100E800089844A00013AB8000030B80088804000E8
:100E900009014A000400330000004000818048003E
:100EA000020149008B05E900C909DD0083017000DA
:100EB0000100320013002000C814DE004814DD00D9
:100EC0004709DE001200B200C808DE000884700086
:100ED000BC01070001F0A1000CF0A70001F0A00088
:100EE000B10137006120E100B30132000801BE000A
:100EF0000200BE00F7FF37006150E100FCFF3A003E
:100F0000AD0137000001BE00EF0107000470A7002B
:100F100003F0A10003F8A30013003A006509B10033
:100F200010003200090035006928E1000200350098
:100F300001002800000005000000400081804800FA
:100F40008502E900FCFF3A0000000600F88F42002D
:100F5000050035008100D1000080D3008502E80043
:100F6000FCFF3A00000006008000EB0000000500D6
:100F70000001BE00D40107000470A70003F0A10027
:100F80006509B100160032000D0035006828E10047
:100F900006003500F0FF2F00F1FF27000300E000FE
:100FA00013003B0001002800000005000000400085
:100FB000818048008502E900FCFF3A000800370004
:100FC000F88F420002003C008000EB0000000500AA
:100FD0008100D1000080D3008502E800FCFF3A00C8
:100FE0000300E00002003B0060001000E0801800F9
:100FF000000006006022B800060220000000D000B9
:101000008180D2000482D2008582D2000000A0003C
:101010000202520083825A000300310002024200A1
:1010200083824A000000A1000603E900F3FF3A00B2
:1010300000000600EFFF07000400BE0000000600ED
:101040000001EB00B501070004003200020020009F
:1010500003F8230001F0A600AAFE07000000060026
:101060000001EB00AD010700040032000200200087
:1010700003F8230001F0A700A1FE0700000006000E
:10108000889FBE008A9FBE008C1F78000205BE00AC
:101090000004BE000006EB00E00F5000E08F580097
:1010A000E00F5900E08F590007003D006000B800D4
:1010B0006011B80008045000898458000A055900DE
:1010C0008B8559001C002000E00F5200E08F5A0071
:1010D000E00F5B00E08F5B0002003D000F000700A7
:1010E0000C00A2000800BE000A01BE00B201070009
:1010F0000203BE000002BE000C00E000010032004E
:10110000060007000400BE000601BE004F0678007E
:101110004F05BE004F04BE00000006006000B8008E
:101120006011B8000402500085825800060359007F
:101130008783590000000600881F780000047800AB
:101140005001BE004000BE00040040008580480001
:101150000601490087814900009CBE000294BE0040
:101160000400E1000588E1000690E1000798E10035
:1011700002003100680044001008E8004F047800C5
:1011800000000600F4874700889FBE008A9FBE00CB
:101190008C9FBE008E1F78000205BE000004BE00BA
:1011A000D4B79F00E5B79F00F6B79F0087BF9F00A9
:1011B0000000EB00C0B79F00B0B79F00A0B79F0032
:1011C00090B79F0080B79F000D042000BFB097002C
:1011D0004FB09700000140000000E0000F003D000C
:1011E0004F08DE0000007100C0B79F009E0007009E
:1011F00001003D0012002000A100070001003D0099
:1012000012002000A6000700B1000700B60007008A
:101210000F004000C8FF0700220037004F08DE0023
:1012200000067100CCB79F008F00070001003D0051
:10123000120020009200070001003D001200200073
:1012400097000700A20007000FB297009FB2970017
:101250002FB39700BFB39700A9000700000052000A
:1012600081805A0002015B0083815B0080B79F0090
:1012700091B79F00A2B79F00B3B79F000007EB0094
:101280009F0007000020E10001A8E10002B0E1009A
:1012900003B8E100010031001E0020000E005600DE
:1012A000C0B79F004FB297000400E0000700350070
:1012B00010002000010020006011B8000804700038
:1012C000898470000A0571008B8571008D06E90024
:1012D000BEFF3A000400E00003003D00820007006A
:1012E0000F00400094FF07004FA897000000E000A7
:1012F00004003A000FB497009FB497002FB59700F1
:10130000BFB59700940007004F0778004F06BE0056
:101310004F05BE004F04BE004F01B10000000600A3
:10132000881F780018002000881F780095FF0700AC
:101330008F87E9004F04780000000600801FEB0053
:1013400090FF07008F87E90000000600889FBE001D
:101350008A9FBE008C1F78006E00070007003D00CA
:1013600073000700E00F5B00E08F5B0007003D00AB
:10137000320007000006EB000400370034000700CD
:1013800002003D002A0007001C0020007200070038
:10139000E3FF07000203BE000002BE000C00E000F5
:1013A00001003200220007000400BE000601BE005A
:1013B0004F0678004F05BE004F04BE000000060037
:1013C000889FBE008A9FBE008C1F780051000700D6
:1013D00005003D0056000700E00F5B00E08F5B005A
:1013E00006003D00040037001900070003003D001F
:1013F0006000B8006011B800100007005600070038
:10140000CEFF07000203BE000002BE000C00E00099
:1014100001003200060007000400BE000601BE0005
:101420004F0678004F05BE004F04BE0000000600C6
:101430006000B8006011B8000000370004025000DE
:101440008582580006035900878359000000060072
:101450000006EB00E00F5200E08F5A00E00F5B0047
:10146000E08F5B00000006000180400090B79F0005
:101470000001EB008FB097000100E00000000600C3
:101480000200700090B79F000180400080B79F006D
:101490000001EB00FFA897000100E000000006003B
:1014A0000200700080B79F00018040006FAA970083
:1014B000CF20DE0001007000F0AF9F000402420068
:1014C000250007004F18DE00000272000000060031
:1014D000E4AF9F000804440089844C000A054D00D5
:1014E0008B854D00000006003FB29700CFB29700F9
:1014F0005FB39700EFB3970000FE2F0000000600D7
:101500003FB09700CFB097005FB19700EFB1970061
:10151000000006000205BE000004BE00E00F5000FF
:10152000E08F5800E00F5900E08F590000000600DE
:101530006000B8006011B8000804500089845800A9
:101540000A0559008B8559001C002000E00F52004D
:10155000E08F5A00000006000800BE000A01BE002D
:10156000000006000004BE00570007000003BE0094
:101570000405BE000200BE0053000700844F750042
:10158000000006000200BE006450E10005003600C5
:101590006420E100020036000968A30001003A005F
:1015A0000800BE000160A0004F0678004F05BE0095
:1015B0004F04BE0000000600F0FF2F00F1FF2700DF
:1015C000F9FF370081002000618055000B003D00CD
:1015D0000B00200061FE2F000100E1001D0034001F
:1015E00082817100610164008904D1000884D30004
:1015F0000000E800FAFF3A0071002000610064007A
:101600000300700002006000090032006104440021
:10161000E0844C000988A500050032008B05E80035
:101620006808E10002003A008904D1000884D30070
:10163000F20F20000258E10005003D00C75DDD000B
:10164000F907B200898075000800780000000600E4
:101650000BF827008B00780000000500889FBE0073
:101660008A9FBE00841F7800BEFF07004F007800ED
:1016700011003300F0FF2F00838F6C0006003B0049
:10168000040565000A00A7000800370009F0A6005D
:101690001000200008003700820F5400838F5C0088
:1016A000030039001000200001003E00000020006F
:1016B00009F0A7000000EA004F05BE004F04BE007D
:1016C0000000E00000000600C70ADE00F107B200DB
:1016D000F50FB20008003200E1CF420002003200F4
:1016E0000170A00024000500810F7000010032008D
:1016F0000408050044000500810F700002003A0054
:10170000140005008502E9000000400081C0480087
:10171000FCFF3B000170A00024000500889FBE0074
:101720008A9FBE000003BE00E7FF07008505780022
:1017300082815200020020006220E10004003A0091
:10174000F307B100040035007718E100040035000C
:101750000600BE00140037006000B8000F0037001C
:10176000F50F2000FAFF2F008502D1000A85D30073
:101770008301E900FCFF3B008184620000046500F6
:10178000890F7400F2FF32008582EA000A85EA00C0
:1017900081846200000465008AFF070007F0A7004B
:1017A00001F0A0000081EB000200E0004F05BE0048
:1017B0004F04BE0000000600889FBE008A9FBE0046
:1017C0008C9FBE000404B8000506B80089044600DA
:1017D00060854E000606B8000A054600E0854E000A
:1017E0000706B8008B054600040EB80089044600C1
:1017F0000A854E00E0854D00050EB8000A0546003A
:101800008B854E00060EB8008B0546000416B80006
:101810000A0546008B854E000516B8008B0546006C
:10182000041EB8008B0546000800BE000A01BE0079
:101830004F06BE004F05BE004F04BE00000006006C
:101840000400FA00E0BF9F00E4815700812978007E
:101850000002EB000F0037006FB89700904078004F
:101860007FB89700104078000402E80080CF500055
:10187000040032008180FB000080FB0000805000EB
:10188000070037006FB897000000E800E0BF9F0036
:101890009309E800820F5200EFFF3A000000EB00CE
:1018A0000080FA000000060010417800B1415100AC
:1018B00003003A000000E8000204E000FAFF3A00EA
:1018C0000300FB00000006008001EB00020037006F
:1018D000817178008301E800828F5100FCFF3A009B
:1018E000000006000000FA00CFB89700688157009A
:1018F000D40007000080FA00000006008101780093
:101900000000E9000081EB00E50F500004003E00FC
:1019100080004000E07D21006081780003B0780005
:101920000200780000000600000178000000E900D5
:10193000E50F50000F003E0080004000E07D2100D8
:10194000E08078000100E00002003A001000200072
:1019500071030700E18F4000060032000000EB0039
:10196000E18F500004003200020078000100010005
:10197000000005000080EB000000060010002000C1
:10198000E9FF0700100020006303070080027800D1
:1019900080017800010037008301E8001304E000B3
:1019A000FDFF3A000002EB00820F520006003200F9
:1019B00064C07800805978000402E8000004E00068
:1019C00002003200F8FF37008049EB000500780084
:1019D000000006000C00FA00889FBE00000478009A
:1019E000CFB09700F0FF2700D0BF9F008004EB002E
:1019F00099BF9F0088BF9F00A8BF9F00200C2000B8
:101A0000B0BF9F0078815700708057008D0007009D
:101A10000FB89700094878000FB8970008045000E5
:101A2000080078004F04BE000080FA0000000600A5
:101A3000800178000001780031407800005978007A
:101A40000004E000FCFF3A000300780000000600FC
:101A50008001EB000200370061F079008301E800AB
:101A6000828F5100FCFF3A000000060081017800DF
:101A70000002EB000B003700E44078000104E000B6
:101A8000030032000402E80093CF5000040032004B
:101A90008180FB001380FB000080500000000600E6
:101AA0008301E800820F5200F3FF3A0000000500B6
:101AB0000C00FA00A0BF9F00C0BF9F000A000700F3
:101AC000B0BF9F00F0BF9F00100C2000D0BF9F0050
:101AD00074815700EFB097006C8057003E030700F9
:101AE0000080FA0000000600800078003004E0006A
:101AF000FEFF3A00010050000000E900000006006F
:101B000010417800814F5100040032000000E800CD
:101B10000204E000FAFF3A000000EB0000000600BB
:101B2000889FBE008A9FBE008000780000C2B3007C
:101B3000010037008900780081047800394478007A
:101B4000804F5400FBFF3200E94F5400F9FF320090
:101B5000D0C2B300804F540004003A00194478000A
:101B60008184E8001AC0B300060037000045EB008E
:101B7000B0C2B300804F540002003A00194478000C
:101B80008184E8006022B8000A003700A20020002B
:101B9000030020000400BE00D3FB07000B414400FB
:101BA0000281FB0003002000000241008182490005
:101BB000394478000880FB000BFD2F000B0040002B
:101BC000E90F5000F1FF36000A04E0000200320085
:101BD00060021200E0821A000400BE004F05BE0041
:101BE0004F04BE0000000600000378008002780069
:101BF000020278008001EB00080037000402E900CF
:101C000063C07800805A78008301E8000004E00097
:101C100002003A008000EB0006003700828F51007E
:101C2000F6FF3A00FBFF37000040EB0080F07A003F
:101C30008100E800848F5000FBFF3A000600780026
:101C400000000600FE874700889FBE008A9FBE00F6
:101C50008C9FBE008E1F7800F0B79F0001077800B0
:101C600082BF9F000000EB00A0B79F009F023700DB
:101C70008006EB0050C2B30080CF50000900320054
:101C80000100FB00FFB09700F4030700E10F4000E4
:101C900096023200AFB097008100E800A1B79F0024
:101CA000920237009E407800D0C2B30080CF50002F
:101CB0000C00320007003C006D40500080CF500007
:101CC0000A0032006B40400080CF50000E003A0006
:101CD0000800370000C3B30080CF50000A003A006C
:101CE000060037000D30A000050037000D00A000F1
:101CF000030037000D10A000010037000D20A000E8
:101D00000E07E800E7FF37000D18A30001003200BE
:101D10000D00A1000D38A300010032000D20A1002C
:101D20000100FB0002FD2F0002004000E90F5000FF
:101D30000E003E000002EB00C4B79F008201780055
:101D4000CFB297006A28B9001E01FB0000014100D4
:101D500003014100C2B79F005E00FB00030040008A
:101D6000E90F50000B003E00F5FF37000006EB00C6
:101D7000CCB79F00A0C2B30080CF500005003A004E
:101D80000FB89700C000780080BF9F00C1B79F00C8
:101D90000E07E8000001EB00B2B79F00E0C2B300FD
:101DA0009E4F100018003A000DE0A0008E00E800E1
:101DB00064405000914F100002003200010778008B
:101DC0000C0037000FBA9700C402780084BF9F0050
:101DD000B5B79F000E87E8000B0037003FB69700AD
:101DE0006A60B9000000410003004000B0B79F00E6
:101DF0000E07E8001E01FB0003FD2F000300410059
:101E0000E90F5000F5FF3600BE407800E1D79F0093
:101E1000C0C6B30080CF5000220032000F003C004B
:101E20006940500080CF50007700320004003C0031
:101E30000104E000310232006B4050000F00370017
:101E400040C6B30080CF5000930032006540400090
:101E500080CF50008B003A008F00370030C7B300AE
:101E600080CF50001A00320007003C006440500050
:101E700080CF5000110032000040E80080CF5000B9
:101E800080003A000F00370050C7B30080CF5000E9
:101E9000800032006340400080CF500079003A005B
:101EA00009003700000028000D48A30001003A0097
:101EB0000001200080867600D3FF37000D60A0006F
:101EC000750037000D50A0000D70A00072003700A3
:101ED0008FB897004100780081BF9F000004780010
:101EE0000000E00001003A00E87821008004EB00E7
:101EF000010037008104E800890078000880440070
:101F00001004E000FBFF3A003FB197000200E00040
:101F100003003200890F5100010031008204780073
:101F20000002EB00E4AF9F00CFB29700898F520010
:101F30000200360009805200E0AF9F004368DE00D7
:101F4000E10660001B003A000D067800090037002A
:101F5000FFB097000002200040030700E10F40009F
:101F6000030032002FB097000000E800A0B79F00E8
:101F70000C06E800EFA89700810F5600F4FF3A0026
:101F80000081EB00E2AF9F000A0037008800780074
:101F90003100FB0001047800FFB097002F03070019
:101FA000E10F4000030032002FB297000402E80066
:101FB000A4B79F000900E90080047800E10F400009
:101FC000F2FF3A000006EB000D00E0000A003A00C4
:101FD000C6013700FFB09700000220001F03070072
:101FE000E10F400003003200AFB297008502E80025
:101FF000A5B79F000C06E8006FA89700800F560059
:10200000F4FF3A00B90137008FB89700410078001B
:1020100081BF9F00CF80DE0001017800820178003F
:102020000205BE000004BE000203BE000002BE00A6
:102030004822DE00482EDD0004027600E4D79F002F
:102040000D48A3000A0032000404E000080032003A
:10205000E14F42000600320071FD2F000180470071
:10206000044878001840980029002000020037003A
:10207000F0D79F001900200072FD2F000284470056
:10208000A1FF370064FD2F000484470019002000E1
:102090009DFF37000D0CB3000D007800000CB2005E
:1020A00028003A000D00E00005003D008FBA9700BF
:1020B0004505BE004504BE0085BF9F0014003700E3
:1020C0000D48A3000B0032000FBE97004C00BE006D
:1020D0008CBF9F004F89DE00CF91DE000002BE0062
:1020E00002037800820378000605BE000404BE00E7
:1020F000070037008FB897004100780081BF9F002C
:1021000000047800CFC4DE00090578008A05780055
:10211000E00F5400E08F5C00E00F5D00E08F5D0099
:102120001F003D003D00B3006000B8006011B80022
:1021300008045000898458000A0559008B8559000D
:10214000170037000D00E00005003D000FB99700B3
:102150004205BE004204BE0082BF9F00100037004F
:102160000D48A300070032000FBA97004400BE00DC
:1021700084BF9F006011B8000205BE000004BE00CD
:10218000070037008FBA97004500780085BF9F0091
:1021900000047800090020000A0020000B00200045
:1021A0003FB697000C00E00007003A00E00F540033
:1021B000E08F5C00E00F5D00E08F5D0002003A0000
:1021C00010002000B0B79F008D007800010CB20015
:1021D000E1B79F0000042000808F500030003200E3
:1021E00003003C000100E00008003200400037001E
:1021F000000820006FB19700800F510014003200DA
:10220000000C2000800F510039003A0014C0B300C8
:10221000E56E21000B0037000400FB004300DD00E9
:10222000050040005001BE004000BE000040E1003B
:1022300001C8E10002D0E10003D8E1002B00390021
:102240000442E800F44F5200F3FF3A002700370041
:1022500000012000010020006011B80014C0B3008C
:102260000040E10001C8E10002D0E10003D8E10034
:102270001E003900450020000000D0008180D200FF
:102280000281D2008381D2008502E900FAFF3A0080
:102290000442E800F04F5200F1FF3A00130037000B
:1022A00080002000010020006011B80014C0B300BD
:1022B0000040E10001C8E10002D0E10003D8E100E4
:1022C0000A0039003C0020000000D0008180D200CC
:1022D0000281D2008381D2000C06E900FAFF3A00A5
:1022E0000442E800F54F5200F1FF3A00E4D79F00A6
:1022F000EFD097000100FB003FB19700820F500024
:1023000002003D00E2D79F00040037003FB2970073
:10231000800F520001003D00B0B79F00CFB2970080
:102320000500E00004003200638066000200320015
:102330008502E900C5B79F000DE8A3000B0032003D
:102340004FB697003FB09700800F560003003C0047
:102350008000EB00C1B79F00040037004FB1970029
:102360003FB2970004015100C2B79F00EFD297001F
:102370000500FB000006EB00DCAF9F00CFB097002C
:10238000808F50000200340000805000D0AF9F00CA
:102390000D28A30037003200E18066000D18A3006D
:1023A0000C003200D00220000100E00001003A00E1
:1023B0000080E900FFB0970028020700E10F40000D
:1023C0000E0032002FB197000201E800A2B79F0073
:1023D0000A0037000100E00008003200FFB097005B
:1023E000000220001D020700E10F40000300320040
:1023F0002FB297000402E800A4B79F00DFAA97005D
:102400000500E0000F0032000006EB00FFB097006F
:102410000003200011020700E10F4000030032001A
:102420002FB097000000E800A0B79F000C06E8005E
:10243000DFA89700810F5600F4FF3A000001EB007F
:10244000D2AF9F003FB29700C320DD00606E210035
:102450008080400091B79F004220DD006400500062
:1024600080B79F006320B900F0AF9F006306500063
:1024700084003700DFAA97000500E0001100320059
:10248000688066000F003A0000067800FFB09700F1
:1024900000022000F1010700E10F400003003200BC
:1024A0002FB097000000E800A0B79F000C06E800DE
:1024B000DFA89700810F5600F4FF3A000001EB00FF
:1024C000D2AF9F00E18066000D18A3000C0032001F
:1024D000D00220000100E00001003A000080E90085
:1024E000FFB09700DD010700E10F4000D5FF32008B
:1024F0002FB297000402E800A4B79F00D1FF370075
:102500000100E000CFFF3200FFB097000002200082
:10251000D2010700E10F4000CAFF3200AFB29700BE
:102520008502E800A5B79F00C6FF37000004200021
:10253000EFB09700808F50003100320003003C0064
:102540000100E000080032003E00370000082000D3
:102550006FB19700800F510011003200000C200075
:10256000800F510037003A001FB097003002BE00C4
:102570002003BE000800BE000A01BE0068FB070081
:10258000A4002000050020006033B8006BFB0700AA
:1025900004C3B30004424000E4D79F002900370081
:1025A00055792100D5B79F000D58A30002003A00CD
:1025B000607A2100D0B79F001400200005002000A1
:1025C0006033B8008FB097008100E9000500330048
:1025D0000402D0008582D2000683D2008783D20015
:1025E000F9FF37000800BE000A01BE004CFB0700DF
:1025F0006F0060005FB19700624078001000370004
:1026000014002000050020006033B8000C007800A2
:102610000000E900050033000402D0008582D200EA
:102620000683D2008783D200F9FF37000800BE007E
:102630000A01BE003AFB0700674060000043B0009B
:10264000E0D79F00EFD097000100FB00FFB097009C
:1026500082010700E10F4000030032002FB1970014
:102660000201E800A2B79F001FB297006802520063
:1026700094B79F008FB29700E482520085B79F0005
:1026800063065600D0FF2F003FB197000090B900BD
:102690007FAA97000000420063005000800F5600A0
:1026A000A2FF3A000D38A30010003200DFAA970005
:1026B0000500E0000D0034000006EB00FFB09700BD
:1026C0000002200065010700E10F40000300320016
:1026D0002FB097000000E800A0B79F000C06E800AC
:1026E000DFA89700810F5600F4FF3A00BE40780043
:1026F000E1D79F000104E0005DFD3A002FB0970094
:102700004F0778004F06BE004F05BE004F04BE00C5
:10271000EF01B100000006000004780096010700F8
:102720000800780041F80700889FBE000004780088
:102730008144780000FD2F0000004400E90F5000A4
:1027400002003E00000178000D003700080078000C
:1027500017F807000000E0000300320008007800CE
:1027600019F8070000047800080078001DF8070039
:102770000000E0000700320090FA2F000001440042
:102780000980FB00800F510002003D000280FB0029
:1027900001003700F00F20004F04BE0000000600CB
:1027A000881F780080BF8000810107000004780046
:1027B00016F807000000E000FAFF3A00E10F4400BD
:1027C0000300320081BF800008007800AC010700E0
:1027D0004F04780000000600EC874700889FBE0089
:1027E0008A9FBE008C9FBE008E1F780081BF9F0015
:1027F0000207780080BF88008046EB0004013700A4
:102800008884FB000900780000F807008000780049
:102810000000E00002003200E1FF0700FC0037008A
:1028200050C2B300804F5400F0003A000FBD970033
:1028300020C0B300C0EF9F00D1EF9F0081EF9F0049
:102840000300370040C0B300C0EF9F000FBD9700EA
:102850000FB99700B240780082BF9F008184FB00CF
:1028600090C6B30080CF50003500320017003E0004
:102870006640500080CF5000620032000C003E00E5
:102880007740500080CF50002800320006003E0004
:102890000104E0009B003200A0C2B30080CF5000D2
:1028A0006E003A001D00370080C5B30016003700E7
:1028B00040C6B30080CF5000210032006440400089
:1028C00080CF500065003A001200370030C7B300D7
:1028D00080CF50001E00320007003E0067405000CD
:1028E00080CF5000110032006340400080CF500084
:1028F0005A003A001400370050C7B30080CF500090
:102900000F0032006340400080CF500053003A0077
:102910006500370020C0B300CBFF3700DFE8970029
:102920008140E800D1EF9F00C8FF37004FE99700D2
:1029300080C0B300E24F5100C3FF3A00C1FF37002F
:10294000ACC0B300590037008CC0B300570037004B
:1029500093FF0700DFE897000104E00002003A005F
:102960004E017800D2B79F0080BF800010010700A1
:1029700000047800E10F4000A20032008FEC9700C5
:10298000120037000A85E8008ABF9F001600370052
:102990008FB897001100FB00800F5400F9FF320040
:1029A0005FE997000204E00003003A005FB097007F
:1029B00008587800D0B79F008944E9000A00320027
:1029C00080BF8000FA000700000478000800E800DB
:1029D000E10F500004003600080078008BF7070074
:1029E0000000E000EAFF3200DFE897000104E000A9
:1029F00087003A008D46E8005FB1970001497800F2
:102A0000830037005FE897000004E00003003A000D
:102A10008D46E800CE007800D1B79F0080BF8000CF
:102A2000E3000700E10F4000760032005FE9970005
:102A30000204E00003003A00DFB0970080587800FD
:102A4000D1B79F000FE997000241E90082EF9F0094
:102A50004240A9006E003400F0FF37000180FB0007
:102A600008FD2F0008004000E90F50005F003E0005
:102A70000A0078001F01070080EF9F00880078009F
:102A8000030037000FB897000000E80080BF9F00E8
:102A90000FB997001200FB0001004000E90F500041
:102AA000F8FF360069FF37000CC1B3003CFF070098
:102AB00080BF8000BE000700000578000040EB00EA
:102AC000E0EF9F00D0022000800F550005003A0083
:102AD00080BF8000B60007000005780011C0B30079
:102AE000E1EF9F008C4078000A0078000EFF07009D
:102AF000E14F40000A003A0081BF80000A007800E0
:102B0000DF0007000D04E0004B003A0080BF8000AA
:102B1000300090000048A300430032004800370016
:102B20008FED97006044B8000C81FB00030020008B
:102B30000800BE00ECF707000004BE008C407800DF
:102B40000A007800F8FE07000080FB00010020006A
:102B500008044000898448008B45E90007003200E2
:102B600080BF800092000700000578008C4078004C
:102B7000EDFE0700E14F4000EBFF3A008C4078008B
:102B80000A007800E8FE0700E14F400003003A0029
:102B900081BF80000A007800B90007006FE9970044
:102BA0000204E0000200320060041400E0841C0013
:102BB0005FE897000004E00015003A008D46E80049
:102BC000CFE89700E4CF500003003A004E007800B1
:102BD0000888BE000E0037000E81E9000207780069
:102BE00012007800080878000900370080BF8000D4
:102BF0006F000700808F540005003200E10F400095
:102C00000B003A000D04E0000D0032000A0037000E
:102C10008FB897003144780081BF9F000804E0001E
:102C2000F7FE3A00040037000000EB000500370013
:102C300081BF8000920007000D80FB00010037007B
:102C40000080EB004F0778004F06BE004F05BE0026
:102C50004F04BE00CF00B10000000600889FBE00F8
:102C60000001780001047800B10090000118A30071
:102C70003D0032000198A30003003A0018009000C4
:102C80000000E00038003A000190A00031049800F4
:102C900082047800F90FB200180090000000E000F4
:102CA00002003A0028009000000C7800EA8F5400DF
:102CB00006003A00380090000078A30003003A00B4
:102CC00088007800D0002000E4FF07009800900002
:102CD00058009000808F50000B0032000100E80087
:102CE000100498001800780009587800000C78004B
:102CF00011C0B300E07E210001487800EA8F540043
:102D0000060032001900370088007800094078007A
:102D10009C00070080047800140037003800900001
:102D20000088A3001100320018019000A800900054
:102D300048009000C5F6070098009000810F5000F1
:102D400004003200380090000003B3003004980003
:102D50008084EB000000EB00100498002800900035
:102D6000000C7800010037008084EB000900780037
:102D70004F04BE0000000600881F780090BF80004E
:102D80000000E0000100320000000100A87B2100EB
:102D900008007800BE0007006C044400E07D2100BC
:102DA000800F5400FAFF3A004F047800000006003C
:102DB000881F780000047800B00090000148A3004C
:102DC00007003A000108A300050032000198A300A3
:102DD00008003200100090000000E0000500320002
:102DE000380090000040A000300498008080EB0084
:102DF000200037000190A1003104980018009000D5
:102E00000000E000060034000000E9001004980013
:102E100018007800B080FB00000C78000600370036
:102E2000380090000068A300EDFF3A000800780029
:102E3000CF00070080007800380090000078A300E1
:102E40000C003A00FA8F500008003A002800900069
:102E50000000E000E2FF3200180090000000E800EF
:102E600010049800180CE900DDFF3700ED8F5000CA
:102E7000E2FF3200010078004F04780000000600F5
:102E800080017800E10F400017003200310090000F
:102E90000008A300140032000098A30012003A00BA
:102EA000210290000400E0000F00320011019000A8
:102EB00051009000800F51000B003200110078008B
:102EC000840F500002003A008008E800020037003A
:102ED0000200E800900098001100E90080087800E6
:102EE00003487800010037008081EB000300780080
:102EF000000006000001780000C2B30001003700A6
:102F00000201E8009240780080CF5000FCFF3200C0
:102F1000E9CF5000FAFF3200D0C2B30080CF50009A
:102F200003003A000201E80014C0B30005003700B6
:102F30000042EB00B0C2B30080CF500001003A0065
:102F40000201E8008000EB0005FD2F0004003700BF
:102F50006A08B90000804100850040000201E800D5
:102F60009201FB0005804100E90F5000F8FF360098
:102F70000404E000010032008100EA000100780052
:102F8000000006000200FA00889FBE00A0FF9F001C
:102F900001047800B1009000810478000904B200B7
:102FA000020032000000FB00360037000118A300C9
:102FB00005003A000103B300310498001904980099
:102FC0000080EB002F003700580090000000E00068
:102FD00006003A004800900012002000E6805700EA
:102FE0001AF6070019049800240037002800900002
:102FF0000000E00008003A00A07E210020049800B4
:10300000000C780020002000500498001004980064
:103010000130A0003104980018019000A800900031
:103020004800900009F6070028009000000C780086
:103030000080EB001004980018007800AFF89700AB
:1030400001587800000C78002FF89700EA4F5000E4
:103050000A003A00380090000088A3000700320000
:1030600018019000A800900048009000F7F50700B4
:1030700019049800A8009000010C7800AFF89700A0
:103080000100FB004F04BE000080FA0000000600B3
:10309000889FBE008A1F78000004780030009000EE
:1030A0006300600024003200080078007E00070002
:1030B0003805900080EF2F00000065003004980074
:1030C000280090000000E00004003200E8046500E1
:1030D00002003A00AD000700290498004800900063
:1030E00011F60700E10F400013003200B800900015
:1030F0000102B20010003A000AC8A3001800320012
:10310000B0BF80000000E000150032000001780030
:1031100081047800012A200012289000880F5000B6
:10312000070032004205B0004905B000818F54000D
:103130000B003200F8FF37000080EB000900370079
:103140000200780001F60700B0BF800009004000CF
:103150008000EB0011289800010078000100370082
:103160000000EB004F0578004F04BE000000060091
:103170000200FA00889FBE008A1F780000047800D1
:103180000000EB0010049800380090008080EB00F5
:103190000008A3003F003200E07E21001004E000A0
:1031A00010003200A97B21000A7C21001A0078005F
:1031B0006C0545002010B20021102000810F500046
:1031C00002003A000900780037000700EC84440050
:1031D000E07D2100808F5400F4FF3A00E07E210062
:1031E0000048EB0048009000580190000200E00009
:1031F0000D003A001204980012002000E8805700E9
:10320000DBF50700E10F500003003A000FF89700CC
:103210008080FB001F003700380090000040A000B5
:103220003004980012003700A8009000D0F5070085
:10323000100498000000E00003003200E10F40009D
:103240000D003A0003003700380090000040A00055
:1032500002003700380090000003B30030049800EB
:10326000A8009000010C78000000EB00100498000A
:103270008080EB0007003700A8009000010C780068
:103280000000E9001004980001007800B080FB0005
:10329000000C7800010078004F0578004F04BE0054
:1032A0000080FA0000000600881F78000004780003
:1032B000300090000008A300070032008000780072
:1032C0000120B20004003A0011049800A800900008
:1032D000010C7800170037000018A3001900320015
:1032E0000098A30017003200A80090000100E00041
:1032F00014003200180190000200E00011003200BA
:103300004800900051F5070098009000810F500090
:1033100003003200380090000003B300300498002E
:103320000000EB001004980028009000000C7800CA
:10333000380090000058A300020032000080EB002B
:10334000010037000000EB004F0478000000060089
:10335000A1BF80000100E0000300320011007800EE
:10336000A0BF88000300370020002000B9F5070047
:1033700080007800E18F400002003A00906E260045
:10338000C0BF88000100780000000600A1BF8000D7
:0C33900001087800A0BF880000000600C3
:020000040000FA
:0200000401F009
:04000C00FBFF0000F6
:020000040000FA
:0200000401F009
:04001000FDFF0000F0
:020000040000FA
:0200000401F009
:040014007FFF00006A
:020000040000FA
:10000800D403000064E400002CE4000048E400008D
:1000180080E400009CE40000D4030000D403000046
:10002800D4030000F2000100D4030000682101009D
:10003800D4030000D4030000D4030000D40300005C
:10004800D4E40000D4030000D40300005C1B0100CA
:10005800D4030000D4030000D4030000D40300003C
:10006800D4030000D4030000D4030000D40300002C
:10007800D4030000D4030000D4030000D40300001C
:10008800D4030000D4030000D4030000D0FD000016
:1000980060FE0000D4030000CC1C0100D403000063
:1000A800D4030000D4030000D4030000D4030000EC
:1000B800D4030000D4030000D4030000D4030000DC
:1000C800D4030000D4030000D4030000D4030000CC
:1000D800D4030000D4030000B8E40000D4030000F7
:1000E800D4030000D4030000D4030000D4030000AC
:1000F800D4030000D4030000D4030000D40300009C
:10010800D4030000D4030000D4030000D40300008B
:10011800D4030000D4030000D4030000D40300007B
:10012800D4030000D4030000D4030000D40300006B
:10013800D4030000D4030000D4030000D40300005B
:10014800D4030000D4030000D4030000D40300004B
:10015800D4030000D4030000D4030000D40300003B
:10016800D4030000D4030000D4030000D40300002B
:10017800D4030000D4030000D4030000D40300001B
:10018800D4030000D4030000D4030000D40300000B
:10019800D4030000D4030000D4030000D4030000FB
:1001A800D4030000D4030000D4030000D4030000EB
:1001B800D4030000D4030000D4030000D4030000DB
:1001C800D4030000D4030000D4030000D4030000CB
:1001D800D4030000D4030000D4030000D4030000BB
:1001E800D4030000D4030000D4030000D4030000AB
:0801F800D4030000D403000051
:020000040000FA
:10020800D403000064E400002CE4000048E400008B
:1002180080E400009CE40000D4030000D403000044
:10022800D4030000F2000100D4030000682101009B
:10023800D4030000D4030000D4030000D40300005A
:10024800D4E40000D4030000D40300005C1B0100C8
:10025800D4030000D4030000D4030000D40300003A
:10026800D4030000D4030000D4030000D40300002A
:10027800D4030000D4030000D4030000D40300001A
:10028800D4030000D4030000D4030000D0FD000014
:1002980060FE0000D4030000CC1C0100D403000061
:1002A800D4030000D4030000D4030000D4030000EA
:1002B800D4030000D4030000D4030000D4030000DA
:1002C800D4030000D4030000D4030000D4030000CA
:1002D800D4030000D4030000B8E40000D4030000F5
:1002E800D4030000D4030000D4030000D4030000AA
:1002F800D4030000D4030000D4030000D40300009A
:10030800D4030000D4030000D4030000D403000089
:10031800D4030000D4030000D4030000D403000079
:10032800D4030000D4030000D4030000D403000069
:10033800D4030000D4030000D4030000D403000059
:10034800D4030000D4030000D4030000D403000049
:10035800D4030000D4030000D4030000D403000039
:10036800D4030000D4030000D4030000D403000029
:10037800D4030000D4030000D4030000D403000019
:10038800D4030000D4030000D4030000D403000009
:10039800D4030000D4030000D4030000D4030000F9
:1003A800D4030000D4030000D4030000D4030000E9
:1003B800D4030000D4030000D4030000D4030000D9
:1003C800D4030000D4030000D4030000D4030000C9
:1003D800D4030000D4030000D4030000D4030000B9
:1003E800D4030000D4030000D4030000D4030000A9
:0803F800D4030000D40300004F
:020000040000FA
:10339C006865000061640000657200002E69000021
:1033AC006E630000006600006F6F00007465000023
:1033BC00722E0000696E00006300000021440000C2
:1033CC0045460000000D00000A0000007478000063
:1033DC0074000000687400006D0000006874000048
:1033EC006D6C00000063000067690000007800004D
:1033FC006D6C000000630000737300000067000038
:10340C0069660000007000006E670000006A000032
:10341C0070670000006300006C6100000077000022
:10342C0061760000000000000000000000000000B9
:10343C00EC990000F0990000F4990000F999000053
:10344C00FD990000019A0000059A0000099A0000FD
:10345C000D9A0000119A0000159A0000199A0000AC
:10346C0074650000787400002F7000006C6100001F
:10347C00696E00000074000065780000742F000075
:10348C00687400006D6C000000740000657800002A
:10349C00742F0000786D00006C0000007465000053
:1034AC00787400002F630000737300000069000043
:1034BC006D610000676500002F6700006966000001
:1034CC00006900006D610000676500002F7000004E
:1034DC006E670000006900006D6100006765000008
:1034EC002F6A00007065000067000000617000002A
:1034FC00706C00006963000061740000696F00006B
:10350C006E2F00006A610000766100002D760000CD
:10351C006D00000061750000646900006F2F0000F1
:10352C00782D000077610000766500000000000037
:10353C00369A0000419A0000419A0000419A00001E
:10354C004B9A0000549A00005D9A0000679A0000A4
:10355C00719A00007C9A0000909A00009D9A0000DD
:10356C0048540000545000002F3100002E31000050
:10357C002032000030300000204F00004B0D0000C6
:10358C000A4300006F6E00006E650000637400005B
:10359C00696F00006E3A0000206300006C6F000041
:1035AC00736500000D0A0000004800005454000030
:1035BC00502F0000312E000031200000343000006C
:1035CC0030200000426100006420000052650000C1
:1035DC007175000065730000740D00000A43000053
:1035EC006F6E00006E65000063740000696F000070
:1035FC006E3A0000206300006C6F000073650000E1
:10360C000D0A00000D0A00003430000030200000CC
:10361C0042610000642000005265000071750000DA
:10362C0065730000743A000020630000616E0000B6
:10363C002774000020680000616E0000646C0000BC
:10364C0065200000436F00006E740000656E000082
:10365C00742D00004C6500006E670000746800005B
:10366C000D0A00000048000054540000502F0000C8
:10367C00312E0000312000003430000031200000D9
:10368C00556E000061750000746800006F720000D8
:10369C00697A0000656400000D0A000057570000AD
:1036AC00572D00004175000074680000656E000025
:1036BC007469000063610000746500003A2000002A
:1036CC004261000073690000632000007265000015
:1036DC00616C00006D3D000022500000726F000014
:1036EC00746500006374000065640000220D000026
:1036FC000A4300006F6E00006E65000063740000EA
:10370C00696F00006E3A0000206300006C6F0000CF
:10371C00736500000D0A00000D0A00003430000033
:10372C0031200000556E00006175000074680000C7
:10373C006F720000697A0000656400003A20000096
:10374C005061000073730000776F0000726400001A
:10375C002072000065710000756900007265000040
:10376C00640D00000A000000485400005450000092
:10377C002F3100002E3100002034000030340000C6
:10378C00204E00006F740000206600006F75000072
:10379C006E6400000D0A0000436F00006E6E0000A6
:1037AC0065630000746900006F6E00003A20000031
:1037BC00636C00006F730000650D00000A4300008D
:1037CC006F6E0000746500006E7400002D540000D4
:1037DC0079700000653A00002074000065780000E4
:1037EC00742F0000687400006D6C00000D0A00005E
:1037FC000D0A000034300000343A0000204600006E
:10380C00696C0000652000006E6F000074200000E1
:10381C00666F0000756E0000643C00006272000070
:10382C003E55000073650000203C00006120000044
:10383C0068720000656600003D2200002F750000D4
:10384C00706C00006F610000642200003E4D0000AF
:10385C005046000053200000557000006C6F0000B3
:10386C00616400003C2F0000613E000020740000E9
:10387C006F200000707200006F6700007261000022
:10388C006D20000077650000622000007061000070
:10389C0067650000730D00000A000000485400002A
:1038AC00545000002F3100002E3100002034000055
:1038BC003134000020520000657100007565000075
:1038CC00737400002D550000524900002054000074
:1038DC006F6F0000204C00006F6E0000670D000041
:1038EC000A4300006F6E00006E65000063740000F8
:1038FC00696F00006E3A0000206300006C6F0000DE
:10390C00736500000D0A00000D0A00003431000040
:10391C0034200000526500007175000065730000D2
:10392C00742D00005552000049200000546F000017
:10393C006F2000004C6F00006E6700003A20000002
:10394C00427500006666000065720000206F000082
:10395C0076650000726600006C6F00007720000036
:10396C006465000074650000637400006564000009
:10397C000D0A00000048000054540000502F0000B5
:10398C00312E0000312000003530000030200000C6
:10399C00496E000074650000726E0000616C0000DE
:1039AC002053000065720000766500007220000054
:1039BC0045720000726F0000720D00000A43000097
:1039CC006F6E00006E65000063740000696F00008C
:1039DC006E3A0000206300006C6F000073650000FD
:1039EC000D0A00000D0A00003530000030200000E8
:1039FC00496E000074650000726E0000616C00007E
:103A0C0020530000657200007665000072200000F3
:103A1C0045720000726F0000723A000020450000F1
:103A2C00787000006563000074650000642000007D
:103A3C006461000074610000206E00006F7400006F
:103A4C002070000072650000736500006E74000049
:103A5C000D0A00000048000054540000502F0000D4
:103A6C00312E0000312000003530000031200000E4
:103A7C004E6F000074200000496D0000706C000057
:103A8C00656D0000656E000074650000640D00003B
:103A9C000A4300006F6E00006E6500006374000046
:103AAC00696F00006E3A0000206300006C6F00002C
:103ABC00736500000D0A00000D0A0000353000008F
:103ACC00312000004E6F000074200000496D000092
:103ADC00706C0000656D0000656E00007465000080
:103AEC00643A0000204F00006E6C0000792000004A
:103AFC004745000054200000616E00006420000067
:103B0C00504F0000535400002073000075700000EB
:103B1C00706F000072740000656400000D0A0000F4
:103B2C000048000054540000502F0000312E0000BB
:103B3C003120000032300000302000004F4B0000DC
:103B4C000D0A0000436F00006E6E000065630000FC
:103B5C00746900006F6E00003A200000636C000076
:103B6C006F730000650D00000A4300006F6E0000CB
:103B7C00746500006E7400002D5400007970000014
:103B8C00653A00002074000065780000742F000076
:103B9C00687400006D6C00000D0A00000D0A000036
:103BAC003C680000746D00006C3E00003C6200003C
:103BBC006F6400007920000073740000796C0000C1
:103BCC00653D0000226D0000617200006769000015
:103BDC006E3A000031300000307000007822000096
:103BEC003E3C0000666F0000726D0000206D00000E
:103BFC0065740000686F0000643D0000706F000089
:103C0C00737400002061000063740000696F000091
:103C1C006E3D0000222F0000757000006C6F0000DC
:103C2C006164000022200000656E000063740000D7
:103C3C0079700000653D0000226D0000756C00007D
:103C4C007469000070610000727400002F6600003F
:103C5C006F7200006D2D0000646100007461000043
:103C6C00223E00003C6200003E4D00005046000029
:103C7C0053200000496D00006167000065200000C2
:103C8C00557000006C6F0000616400003C2F000058
:103C9C00623E00003C7000003E3C0000696E00007B
:103CAC0070750000742000007479000070650000CD
:103CBC003D660000696C0000652000006E6100002C
:103CCC006D6500003D69000020730000697A0000FA
:103CDC00653D0000343000003E200000266E0000E0
:103CEC0062730000703B0000203C0000696E000015
:103CFC00707500007420000074790000706500007D
:103D0C003D730000756200006D69000074200000B6
:103D1C00766100006C750000653D000022550000C6
:103D2C00706C00006F610000642200003E3C0000DB
:103D3C002F6600006F7200006D3E00003C2F0000EB
:103D4C00626F0000647900003E3C00002F680000A8
:103D5C00746D00006C3E00000048000054540000DC
:103D6C00502F0000312E00003120000032300000B6
:103D7C00302000004F4B00000D0A0000436F000084
:103D8C006E6E000065630000746900006F6E0000C9
:103D9C003A200000636C00006F730000650D00009A
:103DAC000A4300006F6E0000746500006E74000022
:103DBC002D54000079700000653A0000207400005A
:103DCC0065780000742F0000687400006D6C0000B2
:103DDC000D0A00000D0A00003C680000746D000024
:103DEC006C3E00003C6200006F6400007920000013
:103DFC0073740000796C0000653D0000226D0000BA
:103E0C0061720000676900006E3A000031300000FA
:103E1C0030700000782200003E3C0000623E000042
:103E2C004D50000046530000205500007064000007
:103E3C00617400006520000053750000636300008E
:103E4C006573000073660000756C00003C2F000069
:103E5C00623E00003C7000003E3C0000612000000F
:103E6C0068720000656600003D2200002F220000F1
:103E7C003E53000069740000652000006D61000075
:103E8C00696E00002070000061670000653C000056
:103E9C002F6100003E3C00002F6200006F640000A8
:103EAC00793E00003C2F0000687400006D6C00002F
:103EBC003E00000048540000545000002F31000018
:103ECC002E31000020350000303000002049000069
:103EDC006E740000657200006E6100006C200000C2
:103EEC0053650000727600006572000020450000EA
:103EFC00727200006F7200000D0A0000436F000028
:103F0C006E6E000065630000746900006F6E000047
:103F1C003A200000636C00006F730000650D000018
:103F2C000A4300006F6E0000746500006E740000A0
:103F3C002D54000079700000653A000020740000D8
:103F4C0065780000742F0000687400006D6C000030
:103F5C000D0A00000D0A00003C680000746D0000A2
:103F6C006C3E00003C6200006F6400007920000091
:103F7C0073740000796C0000653D0000226D000038
:103F8C0061720000676900006E3A00003130000079
:103F9C0030700000782200003E3C0000623E0000C1
:103FAC004D50000046530000204900006D61000098
:103FBC0067650000204300006F72000072750000FE
:103FCC0070740000206F0000722000005772000017
:103FDC006F6E0000672000005665000072730000D1
:103FEC00696F00006E3C00002F6200003E3C000038
:103FFC00703E00003C61000020680000726500000B
:10400C00663D0000222F0000757000006C6F0000F0
:10401C0061640000223E0000547200007920000010
:10402C0061670000616900006E3F00003C2F0000DA
:10403C00613E00003C2F0000626F000064790000BC
:10404C003E3C00002F680000746D00006C3E0000C8
:10405C000048000054540000502F0000312E000086
:10406C00312000003330000032200000466F000089
:10407C00756E0000640D00000A4300006F6E0000B6
:10408C006E65000063740000696F00006E3A0000FA
:10409C00206300006C6F0000736500000D0A0000C7
:1040AC004C6F000063610000746900006F6E0000CB
:1040BC003A2000000048000054540000502F00002B
:1040CC00312E00003120000034300000332000007D
:1040DC00466F0000726200006964000064650000B5
:1040EC006E0D00000A4300006F6E00006E6500004C
:1040FC0063740000696F00006E3A000020630000DA
:10410C006C6F0000736500000D0A00000D0A0000C2
:10411C003430000033200000466F00007262000053
:10412C0069640000646500006E3A000020530000D2
:10413C00534C0000205200006571000075690000AE
:10414C0072650000642000002D20000075730000D3
:10415C00652000004854000054500000530D00002E
:10416C000A000000B69A0000B69A0000DB9A000024
:10417C00399B0000BA9B0000549C0000C19C0000BD
:10418C00319D0000979D00009D9A0000B39E000099
:10419C00609F00002FA0000061A00000436F000092
:1041AC006F6B0000696500003A000000417500006B
:1041BC00746800006F720000697A0000617400007E
:1041CC00696F00006E3A0000004300006F6E000043
:1041DC00746500006E7400002D4C0000656E0000CC
:1041EC0067740000683A000000000000D4A00000D2
:1041FC00DCA00000EBA000004745000054000000CC
:10420C00504F00005354000000750000706C00000B
:10421C006F61000064000000666F000063750000B1
:10422C0073650000722E0000687400006D000000C1
:10423C000D0A00000D0A000033300000342000008D
:10424C005265000064690000726500006374000030
:10425C003A200000004300006F6E000074650000FF
:10426C006E7400002D54000079700000653A000057
:10427C0020000000436F00006E740000656E0000AB
:10428C00742D0000456E0000636F0000646900002F
:10429C006E6700003A200000677A00006970000029
:1042AC000D0A000000430000616300006865000017
:1042BC002D4300006F6E0000747200006F6C0000E4
:1042CC003A200000006E00006F2D000063610000BA
:1042DC0063680000650000006D610000782D00002F
:1042EC0061670000653D00000036000030300000C2
:1042FC0000530000657400002D4300006F6F000038
:10430C006B690000653A0000200000000D0A0000F7
:10431C000D0A0000000D00000A0D00000A4D0000FF
:10432C00504600005302000001000000705F0000C6
:10433C0061700000705F0000636F00006E6600002B
:10434C006967000000730000726300002F480000D2
:10435C00756200002F480000756200002E6300009B
:10436C0000250000733A000025690000202500009C
:10437C00732000002D2D00002061000073730000DD
:10438C0065720000746900006F6E0000206600000A
:10439C00616900006C650000640A00000000000008
:1043AC000000000000000000000000000000000001
:1043BC0000000000000000000000000000000000F1
:1043CC0000000000000000000000000000000000E1
:1043DC0000000000000000000000000000000000D1
:1043EC0000000000000000000000000000000000C1
:1043FC0000000000000000000000000000000000B1
:10440C0000000000000000000000000000000000A0
:10441C000000000000000000000000000000000090
:10442C000000000000000000000000000000000080
:10443C000000000000000000000000000000000070
:10444C000000000000000000000000000000000060
:10445C000000000000000000000000000000000050
:10446C000000000000000000000000000000000040
:10447C000000000000000000000000000000000030
:10448C000000000000000000000000000000000020
:10449C000000000000000000000000000000000010
:1044AC000000000000000000000000000000000000
:1044BC0000000000000000000000000000000000F0
:1044CC0000000000000000000000000000000000E0
:1044DC0000000000000000000000000000000000D0
:1044EC0000000000000000000000000000000000C0
:1044FC0000000000000000000000000000000000B0
:10450C00000000000000000000000000000000009F
:10451C00000000000000000000000000000000008F
:10452C000000000000000000000000000046000039
:10453C00697200006D770000617200006520000058
:10454C003D200000257500002E250000752E000072
:10455C0025750000004C000045440000427200002C
:10456C0069740000652000003D20000025750000E6
:10457C0000480000616E000064430000747200008B
:10458C006C2000003D200000300000005769000046
:10459C00726500006420000049500000203D0000BE
:1045AC0020250000642E0000256400002E2500004C
:1045BC00642E0000256400000057000069460000CE
:1045CC00692000004D6F0000642000003D200000B9
:1045DC002564000000570000694600006943000094
:1045EC006F6E00006E2000003D200000256400006E
:1045FC00005700006946000069460000564F000055
:10460C006B2000003D2000002564000000570000D6
:10461C0069460000694600005665000072200000E3
:10462C003D200000257500002E250000752E000091
:10463C002575000000570000694600006953000012
:10464C0053490000442000003D2000002573000069
:10465C0000570000694600006941000064640000D6
:10466C00722000003D200000256400002E25000073
:10467C00642E0000256400002E250000640000005C
:10468C00576900004669000053650000634D000047
:10469C00203D000020250000630000005769000049
:1046AC004669000053650000634B0000203D00008C
:1046BC002025000073000000000000000000000036
:1046CC0000000000000000000000000000000000DE
:1046DC0000000000000000000000000000000000CE
:1046EC0000000000000000000000000000000000BE
:1046FC0000000000000000000000000000000000AE
:10470C00000000000000000000000000000000009D
:10471C00000000000000000000000000000000008D
:10472C00000000000000000000000000000000007D
:10473C00000000000000000000000000000000006D
:10474C00000000000000000000000000000000005D
:10475C00000000000000000000000000000000004D
:10476C00000000000000000000000000000000003D
:10477C00000000000000000000000000000000002D
:10478C00000000000000000000000000000000001D
:10479C00000000000000000000000000000000000D
:1047AC0000000000000000000000000000000000FD
:1047BC0000000000000000000000000000000000ED
:1047CC0000000000000000000000000000000000DD
:1047DC0000000000000000000000000000000000CD
:1047EC0000000000000000000000000000000000BD
:1047FC0000000000000000000000000000000000AD
:10480C00000000000000000000000000000000009C
:10481C00000000000000000000000000000000008C
:10482C00000000000000000000000000000000007C
:10483C00000000000000000000000000000000006C
:10484C00000000000000000053630000616E0000D7
:10485C002020000049440000203D000020250000DD
:10486C006400000053430000204900006E64000007
:10487C0065780000203D0000202500006400000049
:10488C004E650000744300006F7500006E740000EC
:10489C00203D000020250000640000005363000050
:1048AC00616E00005353000049440000203D00009D
:1048BC0020250000730000005365000063200000F9
:1048CC004D6F000064650000203D000020250000B5
:1048DC00640000004E650000742000005479000054
:1048EC0070650000203D00002025000064000000E1
:1048FC005369000067200000205300007472000010
:10490C00203D000020250000640000004C6F0000DA
:10491C0061640000446F00006E650000203D0000E3
:10492C0020250000640000000000000000000000D2
:10493C00000000000000000000000000000000006B
:10494C00000000000000000000000000000000005B
:10495C00000000000000000000000000000000004B
:10496C00000000000000000000000000000000003B
:10497C00000000000000000000000000000000002B
:10498C00000000000000000000000000000000001B
:10499C00000000000000000000000000000000000B
:1049AC0000000000000000000000000000000000FB
:1049BC0000000000000000000000000000000000EB
:1049CC0000000000000000000000000000000000DB
:1049DC0000000000000000000000000000000000CB
:1049EC0000000000000000000000000000000000BB
:1049FC0000000000000000000000000000000000AB
:104A0C00000000000000000000000000000000009A
:104A1C00000000000000000000000000000000008A
:104A2C00000000000000000000000000000000007A
:104A3C00000000000000000000000000000000006A
:104A4C00000000000000000000000000000000005A
:104A5C00000000000000000000000000000000004A
:104A6C00000000000000000000000000000000003A
:104A7C00000000000000000000000000000000002A
:104A8C00000000000000000000000000000000001A
:104A9C00000000000000000000000000000000000A
:104AAC0000000000000000000000000000000000FA
:104ABC0000000000000000000000000000000000EA
:104ACC0000000000000000000000000000000000DA
:104ADC0000000000000000000000000000000000CA
:104AEC0049500000203D000020250000642E0000ED
:104AFC00256400002E250000642E000025640000B3
:104B0C00004D0000617300006B2000003D20000090
:104B1C00256400002E250000642E00002564000092
:104B2C002E25000064000000476100007465000041
:104B3C0077610000792000003D2000002564000012
:104B4C002E250000642E0000256400002E25000098
:104B5C0064000000504E0000532000003D20000077
:104B6C00256400002E250000642E00002564000042
:104B7C002E25000064000000534E0000532000005E
:104B8C003D200000256400002E250000642E00004E
:104B9C00256400002E250000640000004465000020
:104BAC00662E000020490000502000003D2000002F
:104BBC00256400002E250000642E000025640000F2
:104BCC002E2500006400000044650000662E0000E5
:104BDC00204D0000617300006B2000003D200000A0
:104BEC00256400002E250000642E000025640000C2
:104BFC002E250000640000004448000043500000D3
:104C0C00203D000020250000640000004E650000DF
:104C1C0074420000494F0000532000003D2000006A
:104C2C0025730000004D000041430000203D0000B2
:104C3C0020250000730000000000000000000000B0
:104C4C000000000000000000000000000000000058
:104C5C000000000000000000000000000000000048
:104C6C000000000000000000000000000000000038
:104C7C000000000000000000000000000000000028
:104C8C000000000000000000000000000000000018
:104C9C000000000000000000000000000000000008
:104CAC0000000000000000000000000000000000F8
:104CBC0000000000000000000000000000000000E8
:104CCC0000000000000000000000000000000000D8
:104CDC0000000000000000000000000000000000C8
:104CEC0000000000000000000000000000000000B8
:104CFC0000000000000000000000000000000000A8
:104D0C000000000000000000000000000000000097
:104D1C000000000000000000000000000000000087
:104D2C000000000000000000000000000000000077
:104D3C000000000000000000000000000000000067
:104D4C000000000000000000000000000000000057
:104D5C000000000000000000000000000000000047
:104D6C000000000000000000000000000000000037
:104D7C000000000000000000000000000000000027
:104D8C000000000000000000000000000000000017
:104D9C000000000000000000000000000000000007
:104DAC0000000000000000000000000000000000F7
:104DBC0000000000000000000000000000000000E7
:104DCC0000000000000000000000000000000000D7
:104DDC0000000000000000000000000000000000C7
:104DEC0000000000000000000000000000000000B7
:104DFC00436F00006E66000069670000203D0000F4
:104E0C0020250000640000000000000000000000ED
:104E1C000000000000000000000000000000000086
:104E2C000000000000000000000000000000000076
:104E3C000000000000000000000000000000000066
:104E4C000000000000000000000000000000000056
:104E5C000000000000000000000000000000000046
:104E6C000000000000000000000000000000000036
:104E7C000000000000000000000000000000000026
:104E8C000000000000000000000000000000000016
:104E9C000000000000000000000000000000000006
:104EAC0000000000000000000000000000000000F6
:104EBC0000000000000000000000000000000000E6
:104ECC0000000000000000000000000000000000D6
:104EDC0000000000000000000000000000000000C6
:104EEC0000000000000000000000000000000000B6
:104EFC0000000000000000000000000000000000A6
:104F0C000000000000000000000000000000000095
:104F1C000000000000000000000000000000000085
:104F2C000000000000000000000000000000000075
:104F3C000000000000000000000000000000000065
:104F4C000000000000000000000000000000000055
:104F5C000000000000000000000000000000000045
:104F6C000000000000000000000000000000000035
:104F7C000000000000000000000000000000000025
:104F8C000000000000000000000000000000000015
:104F9C0000000000000000004E65000077200000BB
:104FAC00487500006220000049500000203D0000C0
:104FBC0020250000642E0000256400002E25000032
:104FCC00642E000025640000004E00006577000090
:104FDC002048000075620000204D00006173000045
:104FEC006B2000003D200000256400002E250000F1
:104FFC00642E0000256400002E25000064000000D3
:10500C004E6500007720000048750000622000000B
:10501C0047570000203D000020250000642E0000B2
:10502C00256400002E250000642E0000256400007D
:10503C00004E0000657700002048000075620000FB
:10504C002044000048430000502000003D20000098
:10505C0025640000004E000065770000205700001A
:10506C00694600006920000049500000203D000006
:10507C0020250000642E0000256400002E25000071
:10508C00642E000025640000004E000065770000CF
:10509C002057000069460000692000004D610000A7
:1050AC00736B0000203D000020250000642E0000E2
:1050BC00256400002E250000642E000025640000ED
:1050CC00004E000065770000205700006946000084
:1050DC006920000047570000203D000020250000FB
:1050EC00642E0000256400002E250000642E0000B4
:1050FC0025640000004E000065770000205700007A
:10510C00694600006920000044480000435000003C
:10511C00203D00002025000064000000000000007D
:10512C000000000000000000000000000000000073
:10513C000000000000000000000000000000000063
:10514C000000000000000000000000000000000053
:10515C000000000000000000000000000000000043
:10516C000000000000000000000000000000000033
:10517C000000000000000000000000000000000023
:10518C000000000000000000000000000000000013
:10519C000000000000000000000000000000000003
:1051AC0000000000000000000000000000000000F3
:1051BC0000000000000000000000000000000000E3
:1051CC0000000000000000000000000000000000D3
:1051DC0000000000000000000000000000000000C3
:1051EC0000000000000000000000000000000000B3
:1051FC0000000000000000000000000000000000A3
:10520C000000000000000000000000000000000092
:10521C000000000000000000000000000000000082
:10522C000000000000000000000000000000000072
:10523C000000000000000000000000000000000062
:10524C000000000000000000000000000000000052
:10525C000000000000000000000000000000000042
:10526C000000000000000000000000000000000032
:10527C000000000000000000000000000000000022
:10528C000000000000000000000000000000000012
:10529C000000000000000000000000000000000002
:1052AC0000000000000000000000000000000000F2
:1052BC00000000000000000000000000437500002A
:1052CC0072720000546500006D700000203D0000FB
:1052DC0020250000730000004E6F000020500000DD
:1052EC00726F0000626500000043000075720000E0
:1052FC007253000074650000702000003D20000017
:10530C00256C0000750000005461000072670000FD
:10531C005374000065700000203D00002025000043
:10532C006C75000000490000734D00006F760000A2
:10533C00696E0000672000003D200000257500000C
:10534C0000490000734800006F6D0000696E00009A
:10535C00672000003D20000025750000004900007A
:10536C0073200000486F00006D6500006420000091
:10537C003D2000002575000000540000656D000004
:10538C0070500000726F0000622000003D20000091
:10539C002575000000520000656D00006F74000060
:1053AC00654900004F2000003D20000025750000DD
:1053BC000048000043530000746100007475000045
:1053CC00732000003D200000257500000000000047
:1053DC0000000000000000000000000000000000C1
:1053EC0000000000000000000000000000000000B1
:1053FC0000000000000000000000000000000000A1
:10540C000000000000000000000000000000000090
:10541C000000000000000000000000000000000080
:10542C000000000000000000000000000000000070
:10543C000000000000000000000000000000000060
:10544C000000000000000000000000000000000050
:10545C000000000000000000000000000000000040
:10546C000000000000000000000000000000000030
:10547C000000000000000000000000000000000020
:10548C000000000000000000000000000000000010
:10549C000000000000000000000000000000000000
:1054AC0000000000000000000000000000000000F0
:1054BC0000000000000000000000000000000000E0
:1054CC0000000000000000000000000000000000D0
:1054DC0000000000000000000000000000000000C0
:1054EC0000000000000000000000000000000000B0
:1054FC0000000000000000000000000000000000A0
:10550C00000000000000000000000000000000008F
:10551C00000000000000000000000000000000007F
:10552C00000000000000000000000000000000006F
:10553C00000000000000000000000000000000005F
:10554C00000000000000000000000000000000004F
:10555C00000000000000000000000000004E0000F1
:10556C00696300006B6E0000616D00006520000037
:10557C003D20000025730000004D00006178000004
:10558C005374000065700000732000003D20000083
:10559C00256C0000750000004465000076200000BA
:1055AC005479000070650000203D000020250000AB
:1055BC0063000000544300006F6D00007020000079
:1055CC004F6E0000203D00002025000031750000CA
:1055DC0000540000434D00006F6400006520000083
:1055EC0025630000203D0000202500006400000021
:1055FC004375000072720000656E00005443000099
:10560C00203D00002025000063000000424C0000FB
:10561C00436F00006D7000004F6E0000203D0000D5
:10562C002025000075000000424C00004353000090
:10563C007465000070730000203D00002025000000
:10564C0075000000544300002053000074610000FA
:10565C0072740000203D0000202500007500000041
:10566C00484F00006E53000074610000727400001B
:10567C00203D00002025000075000000546800004B
:10568C00652000007265000063650000697600000B
:10569C0065640000206300006F6D00006D61000008
:1056AC006E6400002069000073200000666F00002B
:1056BC00726D0000617400007465000064200000CD
:1056CC00696E0000636F0000727200006563000079
:1056DC00746C000079000000546800006520000024
:1056EC007265000063650000697600006564000067
:1056FC00206300006F6D00006D6100006E6400009F
:10570C002077000061730000207400006F6F0000B0
:10571C00206C00006F6E00006700000054680000F1
:10572C00652000007265000063650000697600006A
:10573C0065640000206300006F6D00006D61000067
:10574C006E640000206300006F6E00007461000046
:10575C00696E000065640000206900006E76000030
:10576C00616C000069640000207000006172000030
:10577C00616D00006574000065720000730000002C
:10578C00546800006520000072650000636500002D
:10579C006976000065640000206900006465000003
:1057AC006E740000696600006965000072200000DC
:1057BC0077610000732000006E6F00007420000001
:1057CC0072650000636F0000676E0000697A00006C
:1057DC006564000000540000686500002063000050
:1057EC006F6D00006D6100006E640000207200009F
:1057FC0065630000656900007665000064200000A8
:10580C007761000073200000666F000072200000BA
:10581C00616E0000206900006E760000616C000073
:10582C00696400002074000061720000676500006C
:10583C007420000064650000766900006365000058
:10584C000054000068650000206300006F6D0000CC
:10585C006D6100006E640000206900007320000080
:10586C00696E0000766100006C6900006420000025
:10587C006265000063610000757300006520000024
:10588C007468000065200000646500007669000003
:10589C00636500002069000073200000686F000041
:1058AC006D6900006E670000005400006865000020
:1058BC00206300006F6D00006D6100006E640000DD
:1058CC002069000073200000696E00007661000002
:1058DC006C6900006420000077680000696C0000AF
:1058EC00652000006E6F000020740000656D0000E4
:1058FC007065000072610000747500007265000034
:10590C0020700000726F00006265000020690000CA
:10591C007320000061740000746100006368000073
:10592C00656400002E0000005468000061740000E3
:10593C0020640000657600006963000065200000AB
:10594C007479000070650000206400006F65000031
:10595C00732000006E6F000074200000657800005A
:10596C0069730000742E0000004500007272000084
:10597C006F72000020740000657800007420000035
:10598C006E6F000074200000646500006669000002
:10599C006E65000064000000556E0000616200003E
:1059AC006C650000207400006F200000636F000025
:1059BC006E6E00006563000074200000746F0000C0
:1059CC00205700006946000069200000426F00006B
:1059DC0061720000640000004E650000772000003A
:1059EC0057690000466900002073000065740000D0
:1059FC00746900006E670000732000006172000083
:105A0C0065200000696E0000636F00007272000078
:105A1C0065630000740000005468000065200000FD
:105A2C00636F00006D6D0000616E0000642000006B
:105A3C0066610000696C0000656400002062000073
:105A4C006563000061750000736500002074000040
:105A5C0068650000206600006F630000757300002D
:105A6C00657200002069000073200000646900006A
:105A7C00736300006F6E00006E65000063740000BD
:105A8C00656400000054000068650000206300009D
:105A9C006F6D00006D6100006E64000020660000F8
:105AAC00616900006C650000642000006265000004
:105ABC0063610000757300006520000074680000CD
:105ACC0065200000726F000074610000746F0000AC
:105ADC0072200000697300002064000069730000EC
:105AEC00636F00006E6E000065630000746500005B
:105AFC00640000005468000065200000636F000023
:105B0C006D6D0000616E0000642000006661000095
:105B1C00696C000065640000206200006563000091
:105B2C00617500007365000020740000686500005A
:105B3C00206600006F630000757300006572000042
:105B4C0020690000732000006E6F000074200000BC
:105B5C00686F00006D650000640000005468000070
:105B6C0065200000636F00006D6D0000616E000029
:105B7C006420000066610000696C00006564000030
:105B8C002062000065630000617500007365000011
:105B9C002074000068650000207200006F74000023
:105BAC00617400006F720000206900007320000017
:105BBC006E6F000074200000686F00006D650000BF
:105BCC006400000000000000000000000000000065
:105BDC0000000000000000000000000000000000B9
:105BEC0000000000000000000000000000000000A9
:105BFC000000000000000000000000000000000099
:105C0C000000000000000000000000000000000088
:105C1C000000000000000000000000000000000078
:105C2C000000000000000000000000000000000068
:105C3C000000000000000000000000000000000058
:105C4C000000000000000000000000000000000048
:105C5C000000000000000000000000000000000038
:105C6C000000000000000000000000000000000028
:105C7C000000000000000000000000000000000018
:105C8C000000000000000000000000000000000008
:105C9C0000000000000000000000000000000000F8
:105CAC0000000000000000000000000000000000E8
:105CBC0000000000000000000000000000000000D8
:105CCC0000000000000000000000000000000000C8
:105CDC0000000000000000000000000000000000B8
:105CEC0000000000000000000000000000000000A8
:105CFC000000000000000000000000000000000098
:105D0C000000000000000000000000000000000087
:105D1C000000000000000000000000000000000077
:105D2C000000000000000000000000000000000067
:105D3C000000000000000000000000000000000057
:105D4C000000000000000000000000000000000047
:105D5C0000000000437500007272000053740000D4
:105D6C0065700000203D0000202500006C750000CF
:105D7C00005400006172000067530000746500005D
:105D8C00702000003D200000256C00007500000014
:105D9C0043750000726500006E74000050410000F5
:105DAC00203D0000202500006C7500000054000010
:105DBC006172000067650000745000004120000013
:105DCC003D200000256C00007500000049730000A8
:105DDC004D6F0000766900006E670000203D0000EA
:105DEC00202500007500000049730000486F00007A
:105DFC006D6900006E670000203D0000202500004A
:105E0C007500000049730000204800006F6D000011
:105E1C0065640000203D0000202500007500000096
:105E2C000000000000000000000000000000000066
:105E3C000000000000000000000000000000000056
:105E4C000000000000000000000000000000000046
:105E5C000000000000000000000000000000000036
:105E6C000000000000000000000000000000000026
:105E7C000000000000000000000000000000000016
:105E8C000000000000000000000000000000000006
:105E9C0000000000000000000000000000000000F6
:105EAC0000000000000000000000000000000000E6
:105EBC0000000000000000000000000000000000D6
:105ECC0000000000000000000000000000000000C6
:105EDC0000000000000000000000000000000000B6
:105EEC0000000000000000000000000000000000A6
:105EFC000000000000000000000000000000000096
:105F0C000000000000000000000000000000000085
:105F1C000000000000000000000000000000000075
:105F2C000000000000000000000000000000000065
:105F3C000000000000000000000000000000000055
:105F4C000000000000000000000000000000000045
:105F5C000000000000000000000000000000000035
:105F6C000000000000000000000000000000000025
:105F7C000000000000000000000000000000000015
:105F8C000000000000000000000000000000000005
:105F9C0000000000000000000000000000000000F5
:105FAC0000000000000000000000000000000000E5
:105FBC004E690000636B00006E6100006D650000AF
:105FCC00203D000020250000730000004D61000002
:105FDC00785300007465000070730000203D0000D1
:105FEC00202500006C750000004400006576000060
:105FFC002054000079700000652000003D20000056
:10600C0042000000424C0000436F00006D70000025
:10601C004F6E0000203D00002025000075000000A0
:10602C00424C000043530000746500007073000084
:10603C00203D00002025000075000000484F0000A6
:10604C006E5300007461000072740000203D00006B
:10605C0020250000750000006952000065760000E4
:10606C006572000073650000203D000020250000D3
:10607C00750000004D610000785300007065000051
:10608C0065640000203D0000202500007500000024
:10609C00707200006F7400006563000074000000F3
:1060AC00736E00006D70000000610000646D0000F4
:1060BC00696E0000006D000069630000726F0000E3
:1060CC00636800006970000000730000656E0000DA
:1060DC00644300006D640000006600006F63000004
:1060EC007573000065720000312E000068740000AA
:1060FC006D000000707200006F740000656300009A
:10610C00742F0000636F00006E660000696700006A
:10611C002E680000746D0000006900007000000023
:10612C0067770000007300007562000000640000D7
:10613C006E73000031000000646E000073320000CA
:10614C00006D000061630000006800006F730000C8
:10615C00740000006468000063700000002F0000F1
:10616C00707200006F74000065630000742F0000F3
:10617C0072650000626F00006F7400002E680000F2
:10618C00746D00003F0000002F700000726F000063
:10619C0074650000637400002F6300006F6E0000D4
:1061AC0066690000672E0000687400006D00000036
:1061BC004A6100006E2000003235000020320000E1
:1061CC003031000038200000313700003A30000038
:1061DC00363A00003534000000760000352E000001
:1061EC0034320000006E0000616D0000650000009C
:1061FC006E6F0000742000007365000074000000D6
:10620C003C6200003E550000706C00006F610000A5
:10621C006420000061200000466900006C650000ED
:10622C003C2F0000623E0000006300006865000027
:10623C00636B00006564000000660000616900008B
:10624C006C000000546800006520000044790000D8
:10625C006E6100006D69000063200000444E000078
:10626C0053200000436C0000696500006E74000050
:10627C0020690000732000006E6F00007420000085
:10628C00656E0000616200006C650000642E000009
:10629C00006E00006F6E000065000000626C000074
:1062AC006F6300006B0000000000000000000000A5
:1062BC0000000000002500006C75000000000000CC
:1062CC0000000000000000000000000000000000C2
:1062DC0000000000000000000000000000000000B2
:1062EC0000000000000000000000000000000000A2
:1062FC00474500005443000046470000005300008F
:10630C00455400004C450000440000004745000087
:10631C005444000042470000005200004542000077
:10632C004F4F000054000000524500005345000040
:10633C005448000000570000465300005349000029
:10634C00440000005746000053450000434D000038
:10635C000057000046530000454300004B0000006E
:10636C005746000057450000504B000000500000FD
:10637C0055530000485700004600000057520000DB
:10638C0045530000455400000057000049460000EA
:10639C0049520000420000005746000053430000E1
:1063AC00414E000000470000455400004E450000DF
:1063BC00540000004E580000544E0000455400009C
:1063CC000047000045540000484900005000000000
:1063DC005345000054530000495000000053000086
:1063EC0045540000485300004D0000005345000088
:1063FC00544800005347000000530000455400006F
:10640C004853000044000000534100005645000072
:10641C004950000000530000495000005253000046
:10642C00540000004745000054570000495000003C
:10643C000053000045540000574900005000000074
:10644C005345000054570000534D0000005300000A
:10645C00455400005753000047000000534500000E
:10646C0054570000534400000053000041560000F4
:10647C004557000046000000257500000053000041
:10648C004554000000530000544F000052450000DA
:10649C000044000045460000415500004C540000EB
:1064AC00530000005245000053450000540000000A
:1064BC0053430000414E00000000000000000000AB
:1064CC0000000000000000000000000000000000C0
:1064DC0000000000000000000000000000000000B0
:1064EC0000000000000000000000000000000000A0
:1064FC000000000000000000000000000000000090
:10650C00000000000000000000000000000000007F
:10651C00000000000000000000000000000000006F
:10652C00000000000000000000000000000000005F
:10653C00000000000000000000000000000000004F
:10654C00000000000000000000000000000000003F
:10655C00000000000000000000000000000000002F
:10656C00000000000000000000000000000000001F
:10657C00000000000000000000000000000000000F
:10658C00000000004574000068200000536F0000FC
:10659C00636B000065740000204400006973000008
:1065AC00636F00006E6E00006563000074200000D5
:1065BC00436F0000756E0000743A0000203D00002F
:1065CC0020250000750000004574000068200000C4
:1065DC00536F0000636B00006574000020430000E3
:1065EC006F6E00006E6500006374000020430000B5
:1065FC006F7500006E7400003A2000003D20000012
:10660C002575000000450000746800002042000061
:10661C00797400006573000020520000783A000085
:10662C00203D0000202500006C75000000000000DB
:10663C0047450000544400004E4E00000047000047
:10664C004554000053540000410000004745000031
:10665C005443000046470000004400004F4800002F
:10666C00414C00005400000053450000544400000D
:10667C004E4E0000004D00004F56000041420000FD
:10668C0053000000444F0000484F00004D450000EF
:10669C0000430000454E000054450000520000002D
:1066AC0053450000544200004345000000530000D5
:1066BC0045540000424300005300000053450000C5
:1066CC00544800004F530000005300004554000094
:1066DC005443000045000000534500005454000092
:1066EC0043530000004400004F4D00004F56000083
:1066FC0045000000444F0000535400004F50000070
:10670C000053000045540000544300004D000000AD
:10671C005345000054540000434300000052000055
:10672C00455300004554000046000000534500004E
:10673C005444000045560000004D00004F56000028
:10674C0045570000460000004E690000636B0000D6
:10675C006E6100006D650000203D0000200000000F
:10676C00256C00007500000025750000000000007D
:10677C0047450000544400004E4E00000047000006
:10678C0045540000535400004100000047450000F0
:10679C005443000046470000004400004F480000EE
:1067AC00414C0000540000005345000054440000CC
:1067BC004E4E0000004D00004F56000041420000BC
:1067CC0053000000444F0000484F00004D450000AE
:1067DC000053000045540000484F000053000000D7
:1067EC00444F00004D4F000056450000004400008F
:1067FC004F530000544F0000500000005245000061
:10680C005345000054520000005300004554000052
:10681C00524500005600000053450000544400004F
:10682C004556000000530000455400004243000050
:10683C004500000053450000544200004353000043
:10684C00004D00004F560000455000004100000074
:10685C004D4F00005645000057460000004E00000A
:10686C00696300006B6E0000616D00006520000024
:10687C003D200000002500006C7500000025000084
:10688C00750000003000000073720000632F0000E0
:10689C00436C0000696500006E740000436F0000DB
:1068AC006E6E000065630000746900006F6E00007E
:1068BC00732F0000436C0000696500006E740000CB
:1068CC002E63000000250000733A000025690000CB
:1068DC0020250000732000002D2D000020610000F9
:1068EC007373000065720000746900006F6E000025
:1068FC0020660000616900006C650000640A0000FD
:10690C000021000000000000004500004E44000083
:10691C00007000005F6300006C690000656E000091
:10692C00742D00003E770000726900007465000051
:10693C0000450000525200004F5200002049000058
:10694C00442000003D2000002564000000450000AC
:10695C00525200004F5200002054000045580000D5
:10696C00542000003D200000257300000021000091
:10697C000000000008000000C80000002C0100000E
:10698C0008000000C80000002C01000008000000F6
:10699C00C80000002C0100000A000000800100006B
:1069AC00800000000A000000800100008000000050
:1069BC000A0000008001000080000000323200005C
:1069CC0030320000323000000000000000000000F7
:1069DC0000000000000000000000000000000000AB
:1069EC00000000000000000000000000000000009B
:1069FC00000000000D0A0000444800004350000055
:106A0C002F5000006F7700006572000020650000B9
:106A1C00766500006E740000206F00006363000058
:106A2C007572000072650000640000000004000034
:106A3C00A300000000000000474500004D49000085
:106A4C004E490000000000004D500000465300006D
:086A5C0002010000000000002F
:020000040000FA
:106A64000200FA00004F7800E6D6BF009E4F5000A7
:106A740014003200E6D6BF00E24F400006003200A8
:106A8400E6D6BF00D10C0700C1D420000E000900D7
:106A940031187800E001B1001E407800E6F6B70036
:106AA400E0CFB3009E4F1000060032001E80FB00B2
:106AB400C70C0700C1D420000E000900B0187800EC
:106AC400E001B1000080FA00000006000000FA00B6
:106AD400716E210091407800E6D6BF0080CF50004F
:106AE40020003200E7D6BF00E24F4000120032001F
:106AF40080CE200000017800E7D6BF000080FB00B4
:106B04007E00B900FC00400040C32000008040002B
:106B140090427800E7D6BF00AC0C070090007800E4
:106B240080FD2F00008040008402200013C0B300C9
:106B3400854078005A0C0700E6D6BF00E7F6B70098
:106B440083D6200093417800616A800080FD2F0085
:106B54000081400080CE20008402200011C0B300D8
:106B64004F0C07000080FA00000006000C00FA0039
:106B740040F92000000F780040B780000000E000DA
:106B840008003A0024B002000000000080007800F1
:106B9400F07F2000808060000040200000804000E2
:106BA40040B7880000D12000C20320008000EB0021
:106BB400640C0200000000000040EB00204F98002D
:106BC4000040EB00304F98003C0037003E489000F6
:106BD400A3FF0700910E0700904090002147980002
:106BE400C80E07008080E800004C2B0000804000A5
:106BF4009000780041079800C20E0700E4004000AE
:106C0400004C2B0000804000900078003107980071
:106C14002E4090000080FB000000E00001003200E4
:106C2400250037001E00780020079800CE00900051
:106C34003E009000008040001E004000A1022000A1
:106C4400010F400000ED21009E0F1000FDFF3E00EB
:106C54002E40900068EDB7002E0090008002B00036
:106C6400606A8800616A80004E00900000804000E5
:106C74000000E800706A8800716A80003E0090009D
:106C840000804000806A8800D0002000106B8800DB
:106C9400646DA9008DFF0700600E070010407800A6
:106CA4000FEDB700380807003E4890000040E800A8
:106CB400304F980001003700FFFF37003E48900036
:106CC400E54F5000C1FF36000080FA0000000600C6
:106CD4001200FA00100798002107980062479800F4
:106CE40043079800244F98000040EB00004F7800C1
:106CF400750037001E40780059FF0700106B8000B4
:106D0400ED0F50006F003A0070FF0700F1D0200033
:106D1400914078002E48900080CF500069003A00DE
:106D240080212000606888006E4090000004E0002C
:106D340008003A004E009000C0678800646DA80007
:106D440040002000106B8800CE009000316B88005A
:106D54005900370041B78000F03F2000808F500079
:106D64000400360041B7800080382100808F500035
:106D7400020036000040200040B7880040B7800081
:106D8400C06788000000E80040B788004E0090000B
:106D9400B0678800EE20020001000000D06A88007D
:106DA400E16A8800648DA8006E4090000080FB00BA
:106DB400000F98008E089000E38F500021003200ED
:106DC4000E089000E30F500004003C008E08900071
:106DD400E18F500038003500040037000E089000A1
:106DE400E40F500023003200330037001F0C07006B
:106DF400F0678800016888008040EB00614F9800CC
:106E04006E409000E24F500002003A0010C0B30000
:106E1400604F9800EE4890000180FB006100600024
:106E24004201DD0051688000B0FF2F000080600047
:106E340002007000506888000000EB00106B8800AE
:106E44001D0037000E80E800900090000E80E800DE
:106E54001000780080804000E20B0700F067880093
:106E640001688800E20B070020002000106B8800F6
:106E740011003700FD0B070080007800EC0D0700BF
:106E8400FA0B0700F10D0700D60B0700800078000D
:106E9400E0CF20000900090031587800A000B100BB
:106EA400A100B10050002000106B880011C0B30095
:106EB40020C0B300390507001E80FB00600798005E
:106EC400060037001E4FE80051C0B3009ECF1000EB
:106ED40088FF3600E00F2000600798006E009000E5
:106EE4000080FA00000006000400FA00DC0D070030
:106EF40002003600DE0D07000A0037001E4078004D
:106F0400D7FE0700206B800001002100410C070020
:106F140003003200658DA900D50D0700010037007C
:106F2400D60D07001E0090000080FA000000060045
:106F34000400FA00CA0D0700030036008000EB00CD
:106F440011079800080037001E407800C4FE0700AF
:106F5400106B80008000EB0011079800E70F5000D1
:106F640001003A00C20D07001E0090000080FA00E4
:106F7400000006000400FA00B90D070046003E00B8
:106F84001E407800B6FE0700B06A8000C06A880020
:106F9400106B8000DF0D0700E50F50001F0032006A
:106FA4001E009000E50F50000A003E001E009000F5
:106FB400E10F5000150032001E009000E10F500058
:106FC400160039001E009000E30F50002E003E0012
:106FD400120037001E009000EB0F50001C0032001E
:106FE4001E009000EB0F500004003E001E009000B5
:106FF400E70F500024003E000A0037001E009000F6
:10700400EE0F50001D0032001F003700E2CC0200DA
:10701400000000005C0707001F0037005A07070044
:107024001D00370011C0B30010C1B300DB0407001A
:10703400D06780000000E00002003200920D0700DB
:10704400F8FF3A0080002000106B8800120037001F
:1070540011C0B30010C1B300D0040700D067800092
:107064000000E00002003200870D0700F8FF3A003C
:10707400C0002000106B880007003700D0002000FB
:10708400106B8800040037008040EB0040C1B3005F
:10709400C20407003C0707000080FA000000060055
:1070A4000200FA006E0D070005003E001E40780045
:1070B4006BFE0700646DA9001E407800ADFF070059
:1070C4000080FA00000006000400FA00640D0700C6
:1070D400030036008000EB00110798000B00370016
:1070E4001E4078005EFE070078FE070080C2200084
:1070F400E1CF20000900090031587800B067800012
:107104009061880080C22000100798001E00900043
:107114000080FA00000006000200FA00500D07008B
:1071240007003E001E4078004DFE070067FE070082
:10713400550D070002003200570D070097040700A1
:107144000080FA00000006000600FA0020479800BC
:107154002E409000E54F500002003600510D07000C
:107164001C0037002E4090003DFE0700106B80008D
:10717400004F780070C0B3009E4F1000050032002D
:10718400B0C0B3009E4F100002003200450D07004E
:1071940010003700916A8000A06A8000808F500040
:1071A40008003900716A8000606A80000081500024
:1071B400A16A8000906A8000590D07003C0D070009
:1071C40004003700A06A8000916A8000010050002A
:1071D400370D07002E0090000080FA000000060022
:1071E4000600FA0020479800314798002E4090008E
:1071F400E54F5000020036002A0D07003200370028
:107204002E40900016FE07002E409000CEFF07008F
:10721400000F78001E00E00002003A00210D070074
:1072240029003700100020009E0F100002003A00D1
:107234002E409000B8FF07000F0B070007003A002C
:10724400BB0C07000000D1009E0F50000300390062
:107254002E409000B0FF0700650DA80063004700B2
:107264006F0B07001400200013C0B3008C0A070042
:10727400906A80000000E800906A8800916A8000AB
:10728400AF0C070001003900B00C0700100020000B
:107294009E0F100003003A002E4090009EFF07004E
:1072A40007003700AC0C070005003A0064ADA800E5
:1072B4000A2102000100000078004000F06A880002
:1072C40010002000200798002E0090000080FA0093
:1072D400000006000E00FA00A20C0700540B070081
:1072E4006E409000E54F5000030036000000EB00B4
:1072F400600798004A0037006E409000D8FD0700F0
:107304006E40900090FF0700020D07000000E000AF
:1073140005003A006E4090007FFF07000000EB007C
:10732400600798003E0037001E0090002007980078
:107334009E0090005E009000808F50000200360096
:107344005E00900020079800CB0A070007003A006F
:10735400770C07008000D100A20B0700030039005E
:107364006E4090006CFF0700650DA800916A8000D4
:107374002E00900080804000710C07000F0039003F
:10738400716A8000906A8000008F5000BD0A070077
:107394001E02780013C0B300410A07009E00780063
:1073A4004E00900001004000400798002E0090001D
:1073B4001E00500020079800640C0700B10A070063
:1073C4002E02900013C0B300350A0700916A8000B2
:1073D4002E00900000804000906A88009E0090007B
:1073E4005E009000808F500003003E006E409000CD
:1073F40049FF070007003700570C070005003A0053
:1074040064ADA8000A2102000100000078004000D9
:10741400F06A88002E0090001E004000600798006B
:107424006E0090000080FA00000006000400FA00DC
:10743400004F7800110798001E009000740D0200A0
:1074440000000000000178009E0090001E407800BB
:10745400A0FF0700800078001E009000008040001C
:107464000080FA00000006000800FA004047980077
:107474004E409000E54F5000020036005C0B0700C0
:10748400070037004E40900075FD0700280C0700E8
:10749400000FE9004E4090002BFF0700570B070038
:1074A4003E0090000080FA00000006000200FA008E
:1074B400004F78001E4078000A0007000000E0003A
:1074C400060032001E40780065FD0700B06A8000A7
:1074D400C06A8800700C0700B00307000080FA003F
:1074E400000006000400FA005D0C070002003600EC
:1074F400620C0700110037001E40780058FD070099
:10750400420B070005003900B16A8000C06A8000A0
:10751400808050001107980008003700816A8000BD
:10752400C06A800000815000B16A8000706A8000E7
:107534007B0C07000000E800100798001E00900074
:107544000080FA00000006000800FA0020479800B6
:10755400210798002E409000E2FF0700000F7800FA
:107564001E00E00002003A00210B07002100370052
:107574002E4090003AFD0700280B07000700320058
:107584004E0C0700C26A80002E00900014002000F8
:107594008141780011C0B300C1090700C06A8000AE
:1075A4000000E800C06A8800C16A8000000B070080
:1075B40002003600706A8000C06A88001000200053
:1075C4009E0F100002003A00654DA8000700370026
:1075D400E10B070005003A0064ADA8000A2102008F
:1075E40001000000A007B000F06A8800100020002D
:1075F400300798003E0090000080FA00000006006A
:107604000C00FA00404798003107980042079800A0
:10761400870A07004E409000B2FF07003D0C0700A8
:107624000000E00002003A00FF0A07003E003700B5
:107634004E4090000AFD0700CE009000E90A0700C2
:10764400020036001E00900040079800C16A8000C6
:107654004E00900080804000D50A070013003600D9
:10766400816A8000C06A800000805000000FE8003A
:10767400F00A070008003200F10A07001E02780031
:107684008141780011C0B30085090700F00A0700A2
:1076940001004000300798004E0090001E0050008A
:1076A40040079800706A8000C06A8800E10A0700F9
:1076B40005003200E20A07004E0290008141780082
:1076C40011C0B30076090700C16A80004E00900023
:1076D40000804000C06A88004E0090001E004000F8
:1076E400400798009E0090004E009000808050005B
:1076F4004E009000808F500002003E00654DA800AF
:1077040007003700940B070005003A0064ADA80099
:107714000A21020001000000A007B000F06A8800FE
:107724004E009000500798005E0090000080FA0020
:10773400000006000800FA00404798004E40900000
:10774400E54F500002003600A90A07000800370080
:107754004E409000C2FC0700816A8000706A80007D
:10776400008F50004E4090005EFF0700A30A070000
:107774003E0090000080FA00000006001000FA00AD
:10778400780B0700630798006E409000E54F5000A7
:1077940003003E005E0090000000E00002003A009A
:1077A400AE0A0700400037006E409000ACFC0700B2
:1077B4006E4090004BFF070010079800EE00900009
:1077C4005E00900080804000860A070004003600B6
:1077D4001E009000EE009000010050005007980039
:1077E400C16A80006E00900000804000200798006D
:1077F400816A80002E009000808F500004003100C8
:10780400990A07002E00900000804000A80B070092
:10781400816A80002E00900000805000000FE80074
:107824005E0090009E0F50000A003E0068CDBF002D
:10783400CE009000810278005E02900080417800C2
:107844002E01900011C0B300050078001409070050
:1078540013003700990B07004E0090001E027800B9
:10786400814178002E01900011C0B3000C0907007B
:107874005E0090009E00500082D6200012417800E5
:10788400756A80004E0090001E00400001027800DE
:10789400824178000501780011C0B3000009070097
:1078A4005E009000700798007E0090000080FA004F
:1078B400000006000600FA002047980021079800FF
:1078C400AE019000120020008E0078002E4090003F
:1078D400AAFF07001E4078000080FB000080FA0029
:1078E400000006004000FA0020779800211F98004D
:1078F400321F9800431F9800541F9800651F98007A
:107904002E709000E54F500003003E003E1890009A
:107914000000E00003003A000000EB00701F980034
:10792400BF0037002E7090004DFC07002E709000B1
:10793400ECFE0700800078004E1890000080500094
:107944004D0A0700030031008080EB00711F98008E
:10795400B30037005E1890000000E000060032001B
:10796400FE0090005E189000808F500002003600E8
:107974005E18900070079800C16A80004E1890004D
:107984000080400050079800816A80005E009000EB
:10799400808F500005003100330A07005E0090001C
:1079A400008040000000E90050079800DE009000CD
:1079B400010F9800816A80005E00900000805000F2
:1079C4000000E800600798004E18900050079800E7
:1079D400BE189000410798002E18900030079800B8
:1079E4002A0907006E1890000000E000050032002C
:1079F400260A070003003600280A070001003E009B
:107A04002A0A070000C2B300204798002C0A070086
:107A14006E009000808F5000020036006E009000CF
:107A240020479800260A07007E009000808F5000AF
:107A3400020036007E00900020479800200A0700CC
:107A440082D62000124178007200470001027800BB
:107A5400824178000E09900011C0B300900807001D
:107A6400170A07000E08900001004000000F98005C
:107A7400130A07006E009000010050006007980090
:107A84006E0090000000E00004003A00706A80007C
:107A9400000F98000080EB00600798006E189000BB
:107AA4000000E000380032000040EB00404798003E
:107AB40030003700AF0A070000C6B30080CF500083
:107AC4000F003600AB0A0700A0C7B30080CF5000F8
:107AD4000B003E004E4090000081FB00FA0A0700B4
:107AE400104078008040780000CEB30000C0400011
:107AF400804078007200470000004100014878008F
:107B0400F20907000B003A00F409070002003A00EA
:107B1400F809070042003700FF090700DB090700E6
:107B240011003600DD0907000F003E00DF090700E1
:107B34000D0037004E009000301F98001E00E0003A
:107B440009003200BE009000211F98008C0A070033
:107B5400CE09070003003600D009070001003E00EB
:107B6400D2090700320907004E4090000040E800A7
:107B740040479800CE4090002E40900080CF5000A7
:107B8400CCFF3900190037000040EB004047980053
:107B940012003700CD09070006003A00CF0907009C
:107BA40002003A00D30907001D003700DA09070074
:107BB400070037004E009000301F98001E00E000C0
:107BC40003003200BE009000211F9800AF08070098
:107BD4004E4090000040E80040479800CE4090009E
:107BE4002E40900080CF5000EAFF3900B40907000E
:107BF4007E009000010050009F090700030031003F
:107C04000080EB00701F980005003700AC090700E6
:107C14005E009000010040005007980079FF370093
:107C24007E1890000080FA00000006000800FA00A8
:107C3400004F780011479800120798002307980016
:107C4400340798008E00E800BE0290002E029000D7
:107C54009E019000120020001E40780021FF0700C2
:107C64000080FA00000006001400FA00881F780063
:107C74000040EB00004F9800580137000E48900078
:107C840077FB07000040EB002047980058090700E5
:107C9400840A0700216B800000202000008060001F
:107CA4000000E00004003A00206B80000140200046
:107CB400D80807000B00320028650200000000000D
:107CC4000000E0000700320000C1B3002047980024
:107CD400206B80004A00DE00614060000080FB00F1
:107CE400300798001C0A070008003200F86A800078
:107CF4000A21020001000000000054000000E0001E
:107D040002003C0000C1B300204798008609070028
:107D140008003200086B80000A2102000100000004
:107D2400000054000000E00002003C0000C1B30069
:107D340020479800106B8000EB0F50000A003A00B7
:107D4400086B80000A2102000100000000005400BA
:107D54000000E00004003C0010C1B300204798007C
:107D6400C0002000106B8800106B8000E40F5000EE
:107D740023003A00AE0807001E0037006D09070013
:107D84001F0032006F090700306B8000808F5000A5
:107D940017003A004DFB0700030A07006C090700AF
:107DA4003C08070010007800B06788005F0A0700ED
:107DB400EC004000390807001000BE00E908070085
:107DC4003908070020C1B300204798006000200054
:107DD400106B8800220020001E005100610907007A
:107DE400AF0707000000EB00406A8800040037007A
:107DF4001E0FE800230020009E8F1100DFFF3600D5
:107E04002E4090000004E000090032000040EB0026
:107E1400604F98000709070002003A0011C0B30040
:107E2400614F9800EE4890002E4090005B010700DF
:107E34005909070021003A00106B8000E70F500039
:107E4400E3003A00EE200200010000001B080700D6
:107E5400DF003500206B800067006000E60F5000F3
:107E64000E003A00206B80004300DE006140600099
:107E7400204798000E4890003EFC07000E489000F2
:107E84003CFC07002E4090000004E000D0003A00C3
:107E9400E0002000106B8800CD0037000BFB0700CA
:107EA40021C0B30000C1B3003C010700EE20020072
:107EB4000100000006080700C5003700EE2002009C
:107EC40001000000FD070700C1003500FFFA0700AC
:107ED400106B80006101B800020F9800130F980026
:107EE400C0002000010020000E0990009E099000AF
:107EF400A108070094003E000E0890009E08900020
:107F0400006001000C0037001F0037003500370007
:107F14003D0037008C003700570037006100370000
:107F24006D003700750037007A0037007B0037009A
:107F3400690037007F003700C6CC02000000000053
:107F44000000E0008000320010002000106B880068
:107F540050688000640060000000E000050032000A
:107F64001109070011C0B30008CD02000000000091
:107F7400750037000C09070011C0B30008CD0200DA
:107F840000000000700037006A00470038CD02008E
:107F9400000000000000E0006B003200E2CC0200B0
:107FA400000000000000E00008003200CB090700D8
:107FB400F06788000168880020002000106B8800AA
:107FC400B90707008A0707005F003700EE200200A8
:107FD40001000000C10707000000EB00106B8800DF
:107FE400590037000A21020001000000F06A8800ED
:107FF400E0CF2000A0FB02000000000030002000C1
:10800400106B88005000370021D02000E0CF200002
:10801400EEFB0200000000000000E00010003A0047
:108024000A2102000100000080007800F06A80004C
:10803400008150004067800051678000800F51002C
:10804400410036000ECDBF00E54F500001003E0058
:10805400D808070020002000106B88003A00370081
:1080640020C0B3002047980061080700500020009A
:10807400106B88003400370020C0B300F9070700F4
:108084000ECDBF00E14F50002F00360020C0B300DA
:108094000EEDB700404B2C004100200058070700AC
:1080A400290037000ECDBF00E14F500003003E0011
:1080B40020C1B300EB07070023003700C508070001
:1080C40002003200C70807001F00370020C0B300B9
:1080D400204798001C003700C708070002003E0034
:1080E400820707001800370080002000106B88000A
:1080F40010C1B3002047980013003700BE080700E2
:1081040002003E00BF0807000F003700B508070053
:108114000D003700B30807000B003700B60807004E
:1081240002003E007107070007003700AD08070092
:1081340005003700B008070002003E00B108070040
:1081440001003700A70807002E4090000004E0005B
:108154001C0032003708070017003200950807009A
:10816400A1678000A06A8000008F5000A708070064
:1081740004003100706A8000616A800001005000D0
:108184001E0F40000B0907001E00780001002000AC
:1081940058070700D06780001E004000D0678800A1
:1081A400A06A8000A06788008040EB002E40900009
:1081B4007A0007000300370011C0B3002E4090007E
:1081C400760007001508070001003200EE020700E0
:1081D4000E4890000040E800004F98000E489000C0
:1081E400E54F5000A5FE3600910707001500370043
:1081F40050080700160032000A21020001000000A6
:108204000001780049090700F20040002307070035
:10821400100078008000510070722000808F5000A0
:1082240007003600210020001E8050004D08070082
:108234009B0607000000EB00406A88001E0FE9005F
:108244001E0FE800220020009E0F1100E8FF3600F8
:108254004F0478000080FA00000006002E00FA00A7
:10826400301798004117980052179800BE109000DC
:108274009E070700760047000288BE004E1090005B
:108284001000BE007601470064080700F6004700AE
:108294000040EB0080489800F600470060C0B3003F
:1082A4009048980076004700DE1090005100980036
:1082B4007600470050009000B4B4020000000000B3
:1082C400800078007600470051009800760047004F
:1082D400C1002000F6B40200000000000080EA00A3
:1082E400101798005E109000DA6802000000000089
:1082F400201798009E1090002E109000808F500040
:10830400050032004065020000000000100020005B
:10831400601798001E0037000000EB006E1A020080
:10832400010000000E80E80041012000426B0200C1
:10833400000000000E80E800620207000E80E800E2
:108344009F0807004200DD00744F50009E80FB0030
:108354005E10900001005000740050005017980007
:108364000E80E800BE1090009C0107000000E000B1
:10837400030032000E80E800DE1090001A030700AC
:108384004065020000000000110020006117980001
:108394006E1090000080FA00000006002A00FA0027
:1083A400006F9800116F9800C8F9070031070700A3
:1083B40005003200656DA8000E689000E1CFB3009F
:1083C40001406000006F980064ADA90064CDA9006D
:1083D40064EDA900652DA900654DA900650DA900EE
:1083E40028650200000000000000E000FCFF3200ED
:1083F4000E6890000080FB00660060000000E00052
:10840400020032000A070700670037009E080700D1
:1084140002003A0006070700580037009A080700D0
:1084240019003600906A8000A1678000010F500097
:10843400D06780009E0F500002003100D06780009A
:10844400000F7800606880009E0F50000300310028
:1084540061688000010F7800654DA80068CDBF00F9
:10846400A26780001E027800804178008040EB0003
:10847400909D20000A060700A06780001E004000AF
:10848400A06788003D003700716A8000A067800003
:1084940080805000E4070700D0009000906A8000BC
:1084A40080804000606A8000008F5000D0678000A8
:1084B4009E0F500002003100D0678000000F78004A
:1084C400606880009E0F50000300310061688000E6
:1084D400010F7800654DA800D70707009E0F5000D4
:1084E400030036007C0047009E007800510098008D
:1084F400D107070071080700A26780000002780016
:10850400814178008040EB00909D2000E405070045
:10851400C90707009E001000C30707005000900021
:108524000000E0000E0032007C0047005001900083
:1085340083D6200093417800656A8000716A8000C8
:10854400A067800080805000909D20000080400043
:1085540002027800050178008040EB00D005070096
:10856400A06780001E004000A0678800A16780000B
:10857400F307070001003900B2070700B507070039
:1085840009003200D06780009E0F500006003200C0
:10859400606880009E0F5000030032000E68900057
:1085A4000004A000006F98001E00E00005003A00DF
:1085B4000E6890000080FB00630060000000E00093
:1085C40015003200D06780001E005000D06788007C
:1085D4001E00E000030032000E6890000034A0008A
:1085E400006F98001E689000A30607000500320083
:1085F4000040EB000EEDB700D01223001100200064
:10860400FF050700EE2002000100000094070700A8
:10861400648DA800290037001E68900098060700A2
:1086240012003200206B8000674060000040E800C8
:10863400674060000080FB0067016000216B8000E0
:1086440080FF2F000080600002007000206B880013
:10865400DF07070061005000E0805800260607008D
:1086640010002000000F7800140037004A070700AC
:10867400120032001E6890000080FB008306070091
:108684000B003A000ECDBF000004E00008003200E9
:108694000ECDBF000040E9000EEDB700406780003A
:1086A400516780008100D1000080D300D405070009
:1086B400EE2002000100000069070700C167800086
:1086C4006400470001087800B16780006400470037
:1086D40011009800BE070700640147004F07070018
:1086E4008067800091678000640147004001980022
:1086F4005101980064014700E2009000F0FF23005C
:10870400008060006001980064014700E20090006E
:1087140000FF2F00008060006001980064004700A3
:108724008E68900051489800E40047000000EB0078
:10873400900898009F0707001E007800A70707000D
:10874400F0050700180032000E689000EF050700DE
:1087540004003A00640147006000B800400198003A
:108764005101980050688000620060000000E00041
:108774000800320064004700B00090002000900020
:1087840061005000E080580064014700230707009F
:10879400050037008E07070061004000E0804800B4
:1087A400D50507000A2DA800320607000100320093
:1087B4000A0DA80095060700050039002B070700DD
:1087C40080005100640047007100980006003700E3
:1087D400C16A8000B06A8000008050008000E90017
:1087E40064004700710098006E65020000000000FC
:1087F400100798009E009000F0032000808F500026
:1088040002003E009D070700040037001E00900090
:1088140001FC2F000100400010079800640047008D
:10882400F00090006F060700030036009E009000E1
:1088340064004700710098006400470021010700AC
:108844001E007800740F400064014700E2009000AD
:10885400F0F02F000080600001052000010070008E
:1088640060019800A7050700150032009E007800FB
:10887400648F400020C0B300005F980040C0B30084
:10888400105F980020802100500F9800640047007A
:108894004B0707000040E8006F406000E401470018
:1088A4000080FB006F0060004401DD00E3009000E5
:1088B400F0F02F000080600002007000E0019800DA
:1088C40002C8BF008080FB0003C8BF004507070043
:1088D4000001780004C8BF008080FB0005C8BF0009
:1088E40040070700800178007C0047000288BE0032
:1088F400AD0607007C014700C8060700FC004700DE
:108904000040EB0080489800FC00470060C0B300C2
:10891400904898007C0047009E0078005100980021
:10892400C5060700B4B4020000000000800078000F
:10893400BD060700C1002000F6B4020000000000DC
:108944008080EA006400470001089800109B200022
:108954004C680200000000001E01780061C0B300F2
:10896400E0CF2000D8190200010000006400470095
:1089740041012000026C02000000000061050700B4
:10898400040032007800470041002000026C02001D
:1089940000000000509C20007068020000000000ED
:1089A4001E007800DA68020000000000100798003A
:1089B400509D20004C680200000000000E80E8007A
:1089C40021002000026C0200000000002C6702005D
:1089D400000000000080FA00000006000C00FA000D
:1089E400881F78003007980041079800A606070002
:1089F4000000E00002003A000B060700AD0037005B
:108A0400E0CFB30040479800CE009000080707006D
:108A14004E0090000D0707003E0090001000780003
:108A240080804000980607000080680010079800C6
:108A34000040EB0050479800280037005E4090004B
:108A440007F80700106B8000ED0F50002000320083
:108A5400106B8000E40F500008003A00306B800077
:108A6400BE00900091009000810F500018003A0061
:108A7400DE4090004147980015003700316B8000BC
:108A8400D805070012003A0010F807003E009000D5
:108A940090009000C0678000808F50000C003A0066
:108AA4003E00900090007800B0678000808F5000F6
:108AB40007003A00180507003B060700AE0507004B
:108AC40003003A0010002000500798007900370096
:108AD4005E4090000040E800504798005E409000DF
:108AE400E54F5000D5FF36004E409000E24F400065
:108AF400140032004E409000D9F70700F3F7070046
:108B04004E409000E24F40000E0032009E00900064
:108B1400316B88004E0090000D0607003E00900067
:108B240010007800B067880057060700C067880007
:108B3400606A8000A0678800100020005007980039
:108B44005C0037003E009000E00090000020200010
:108B5400008060000000E00003003A008000EB00A9
:108B64005107980053003700406A80000000E0007D
:108B740002003200AC0507004E0037002C05070048
:108B840018003700EB05070019003200ED05070057
:108B94003D060700808F500011003A00BD04070015
:108BA400900078003E00900010007800808F500004
:108BB4000B003A007C0607001003BE00D604070031
:108BC400820F5300838F5B0005003A001E04780077
:108BD4000A210200010000002E06070035003700BC
:108BE4001E0FE800200020009E0F1000E5FF360055
:108BF4000040EB00504798002A0037005E40900088
:108C040097F70700F305070023003200AFF70700CA
:108C1400C0678000BE00900091009000810F50005A
:108C24001D003A00B3060700808040004E0090000B
:108C340009000900B0587800A100B100A000B100FB
:108C440083050700100178007408B900EA004000A9
:108C5400670607007E05070020019000B001900020
:108C64007408B900EC0040008C0407000288BE00C0
:108C740077050700100190007408B900F000400067
:108C84005B0607001E0478000A21020001000000B0
:108C940000060700070037005E4090000040E8002F
:108CA400504798005E409000E54F5000D3FF3600D7
:108CB4005D0507005E0090004F0478000080FA0014
:108CC400000006000200FA00000F78001E00780081
:108CD40010007800B4B4020000000000F40507009E
:108CE400010878001E00780010009000B4B402005F
:108CF40000000000EE050700110098001E00780037
:108D0400B000900020009000CCB4020000000000ED
:108D14001E017800C10507001E007800D0009000F5
:108D240040009000CCB40200000000001E01780056
:108D340040019800510198001E00780070009000D6
:108D4400B4B4020000000000D905070071009800C7
:108D54001E00780000089000B4B402000000000077
:108D6400D3050700010898001E0078001008900041
:108D7400B4B4020000000000CD05070011089800FB
:108D84000080FA00000006000200FA00881F780044
:108D94004EF70700C0678000306B8800EB050700C2
:108DA400606A8000A06A8800706A8000B06A8800E7
:108DB400706A8000C06A88008605070003003200DC
:108DC40040002000000F780002003700D00020008F
:108DD400000F78001E007800106B8800640DA90055
:108DE400642DA900644DA900648DA90064ADA90097
:108DF40064CDA90064EDA900650DA900652DA90045
:108E0400654DA900656DA900658DA8000A0DA9002E
:108E14000A2DA9000A6DA9000A8DA900606A8000C4
:108E2400A0678800C8CE2000C0AF02000000000088
:108E3400000C7800C8CE2000C0AF02000000000083
:108E4400100498000080EB004068880010002000A7
:108E5400D06788004F0478000080FA000000060004
:108E64000600FA00881F7800C00020006E1A020075
:108E740001000000286B0200000000001047980069
:108E84001E4090008080FB00000F200000806000E6
:108E94004280DE0074405000104798001E4090004D
:108EA4000004E00003003A0080212000200798001D
:108EB40049003700710020000000EB00426B020003
:108EC400000000003C003700286B02000000000096
:108ED400004F78001E04E0003D00320010C0B300D3
:108EE4009E4F10003400320020C0B3009E4F10008B
:108EF40021003A001E409000E24F5000340036003A
:108F0400DE050700286B020000000000004F780017
:108F140040C0B3009E4F100009003A000E80E800E4
:108F24000004E800286B020000000000004C7800F8
:108F34000E84E800286B020000000000004C78005A
:108F44009E00900070212000808F50002000360089
:108F54009E009000405B2000808F5000030036008C
:108F6400405B2000200798001B0037001E00900083
:108F740020079800180037001E409000E14F500071
:108F840013003600286B020000000000004F780038
:108F94001E4090009E4F50000D0039009E80FB0043
:108FA4000000EB00426B0200000000001E40900035
:108FB4001E405000104798001E4090000040E900F9
:108FC400104798001E409000E14F4000BEFF3A0059
:108FD40080212000200798002E0090004F04780084
:108FE4000080FA00000006002800FA00700F9800C4
:108FF400011798007E089000D0489000614F9800B7
:109004007E08900040019000D00190005207980023
:10901400630798007E08900020019000B001900042
:109024003207980043079800640DA900642DA90035
:10903400644DA900D804070003003A00EE200200A2
:1090440001000000A2030700136B8000331798008F
:109054003E109000E40F500004003200BE10900057
:10906400E58F50001A0032003C003700130507005A
:109074000200320044FF07007E0237001205070099
:10908400060032005D0507008040EB0040C0B300DD
:10909400C2FC07003CFF0700760237000D050700FD
:1090A400090032009E0307006DFF07006068880016
:1090B40011C0B30020C1B300B8FC07006000200059
:1090C400106B88006B0237002FFF0700690237001E
:1090D400FA04070067023A00FB04070006003200A6
:1090E4009103070004003200FC040700ABFC0700F6
:1090F400010507005F023700F60407005D02320035
:10910400870307007E08900070009000D0678800F5
:1091140053FF070060688800EB0407000900320071
:109124005D0507009DFC070070002000106B88009F
:10913400EE2002000100000068030700648DA9000E
:109144004C02370011C0B30020C1B30093FC0700E8
:1091540060002000106B8800460237008E109000DB
:1091640021079800E6040700030032002E00900057
:109174000000E80020079800D6040700030032002E
:109184002E0090000000E800200798001F0407004C
:1091940004003900B504070000005100000F9800D6
:1091A40005003700C16A8000B06A8000008050006A
:1091B4000000E900000F9800826780009367800038
:1091C400130507000200500083805800200F980008
:1091D400310F98002E099000120F98002705070000
:1091E4000E040700200032000E0890000000E0008A
:1091F40026003200C404070004003500A60307005B
:10920400020036001A0507000E0037002E009000F9
:109214006101B8002E089000BE089000E703070023
:10922400FA020700070034008E0890002E00900018
:10923400008050006101B900990307000100350066
:109244000B05070094030700100034001E0890006B
:10925400AE009000010040000000E0000B0034006C
:109264000305070009003700A704070002003A00BD
:10927400FF04070005003700A304070003003500BE
:109284008503070001003600F90407001E00900062
:109294000000E00006003A009E0407000000E00021
:1092A400F4013A00FC0407003CFC0700F10137001C
:1092B4009C040700660060000000E0000200320029
:1092C400B1FE0700EB0137006E4890000F03070062
:1092D400E8013200136B8000231798002E109000D1
:1092E400EB0F500007003E00AE109000E78F5000D7
:1092F400100031002E119000E60F510005003200DD
:10930400CB003700AE119000EC8F5100C100320049
:10931400C700370004030700040032006F0407008D
:109324001EFC070074040700D201370070002000FF
:10933400106B8800916A8000A06780000080500054
:10934400A103070006003D00716A8000606A800086
:10935400808050004E08900001004000400F9800AB
:10936400940407004E089000860307009A03070040
:1093740086030700110034006B0307000600320067
:109384005E099000EE09900010002000010020000A
:1093940079030700040032008040EB0000C1B300F1
:1093A400FEFB0700B3013700CC0407006100500046
:1093B400E080580050079800610798003B030700BD
:1093C4008503070011040700040031005803070057
:1093D40002005000838058007F0307006B030700DE
:1093E4002E00340052030700630307002B003900EA
:1093F4000A6DA9000A8DA900650DA900A16A800063
:10940400410F9800A16A80005E089000008040002F
:10941400A06A8800A16780004E089000808F5000E9
:1094240007003900F9030700100031006104070048
:10943400A16A8000A0678000420307000B00370088
:109444002003070000004100400F9800A16A80003B
:109454004E089000808F5000040036005504070029
:10946400A16A80004E08900036030700A16A8000BC
:109474003304070004003900A26A80002C040700AA
:1094840000005100A06A8800A16780002C04070036
:109494001B003900EB03070019003700A16A8000A4
:1094A400A0678000808F5000150032005068800053
:1094B400680060000000E000100032005068800086
:1094C400700060000000E0000B003200F7020700AB
:1094D40089020700CD0307000400310035040700AA
:1094E40013040700CF80DE0082020700A06A800018
:1094F400A0678800654DA8000A8DA8000A6DA80021
:10950400A16A8000906A8000808F50000D003A00AC
:10951400D003070005003A00EE200200010000001D
:109524006B020700648DA900060037007E02070065
:1095340004003A00FC02070002003200648DA90016
:10954400656DA9007E08900070019000200407005A
:10955400800078005E00900000805000000F5100F1
:10956400D06780000000E00003003A001E00E00025
:1095740001003200652DA8001E017800D267880022
:10958400106B8000E80F50000E003A0066020700DE
:1095940027003A00E402070025003200EE20020012
:1095A400010000000001BE0020BC2E00B10020001C
:1095B40019020700648DA80090002000106B880039
:1095C4001B003700106B8000E90F50000A003A00BE
:1095D400D4030700AD02070015003A003F0407005A
:1095E400450207008040EB0040C1B3006BFB07005D
:1095F400E5FD07001F013700106B8000EA0F5000E3
:109604000B003A00480207001A013A00DEFD070089
:1096140018013700EE03070061014000E0814800B3
:109624004202070013013A00D7FD07001101370079
:10963400BC0307004500DE00FB0107000D013A00F2
:10964400106B8000EB0F50000A013200106B800099
:10965400EA0F500007013200106B8000EC0F50003D
:10966400040132000E1090000000E000A900320056
:109674001E0890000000E00053003C002D0207008B
:10968400800078001E089000008050006E1A0200CE
:10969400010000008E1090001E0890000080400021
:1096A400001798008E1090000E089000808F5000D4
:1096B400020036008E08900001179800826780002F
:1096C400936780000E1090001F020700D901070065
:1096D40012003600816A8000B06A80000080500069
:1096E4000000E800400F9800F4030700B06A80000F
:1096F4004E0A90007502070069010700170207006F
:1097040067010700726A80008E1090004E08900076
:1097140003040700B06A880009003700E703070064
:10972400B06A80000E129000680207005C01070016
:10973400B16A80000E10900000804000B06A88007A
:1097440040688000E10F400072003200820207008E
:109754000E1090000080500040688800E16780008F
:1097640040688000008040009702070003003D002D
:109774000080EB0040688800660037004068800085
:109784000000E00063003C00826780009367800073
:109794004E089000EC0107004E0890000080400045
:1097A400B06A8800B16A80008102070003003600B5
:1097B400B26A8000F2010700B06A88000080EB0002
:1097C40040688800530037001E0890000000E00045
:1097D400500034008E1090001E08900080804000DD
:1097E4000E089000808F5000040036000E08900090
:1097F4009E0890000100500000179800CD0107005A
:109804006E1A020001000000B16A80001E08900078
:10981400808040008701070016003600816A8000BE
:10982400B06A8000808050001E08900000805000C4
:109834000000E8006402070008003500D5010700B5
:109844004E0A9000210207008540780014010700A9
:10985400C201070012010700090037001E020700B9
:1098640000814000C6010700CD0107000C0107007C
:1098740003003700C7010700C901070008010700FA
:1098840040688000E10F400005003A001E08900087
:10989400406888000E119000E26788001D003700C0
:1098A4002D0207001E089000808F50000E00360025
:1098B400BF01070003003E00C5010700808F500070
:1098C400030031008E119000E36788000300370025
:1098D400C401070000805000E06788001E08900063
:1098E400406888000B003700B1010700090036000A
:1098F400BC010700808F500006003900E267800039
:10990400B301070080805000E067800084030700F3
:10991400E06788004102070015003200106B8000E8
:10992400E70F500002003200B06A8000C06A88006D
:10993400206B800001082000B601070004003200FB
:109944005503070095FA070060F407000800370084
:1099540064EDA8007402070005003A0064CDA80075
:109964000A21020001000000D003B000006B88004F
:10997400E30207003F0032008067800091678000A7
:1099840061024000E08248002E0090006101B800AE
:109994001F03070009020700800F5200818F5A003D
:1099A40034003A008067800091678000ED01070071
:1099B400106B8000101798009E109000E78F5000E5
:1099C400140032001E119000E70F510004003E0005
:1099D4009E119000E68F51000800320023003700EA
:1099E4001E109000E80F5000110032009E109000ED
:1099F400E98F5000180032001C003700C00020001E
:109A0400106B880011C0B30010C1B30063FA0700E3
:109A140018003700B0002000106B88000A210200F3
:109A240001000000A007B000006B88000F003700A1
:109A34003D01070005003A008040EB0000C1B3007F
:109A440056FA0700D0FC07000A003700A0002000E7
:109A5400106B8800050037008040EB0000C1B300A4
:109A64004EFA0700C8FC0700020037000A0307008B
:109A74004AFA07000080FA00000006001000FA000D
:109A8400B8020700434F98006E409000E54F500025
:109A940002003600F10107007E0037006E4090009E
:109AA400EFF307004E0090000000E00002003A00CF
:109AB4001000200040079800816A8000606A8000DE
:109AC40000805000FA02070049010700808F50000F
:109AD40002003600E10107006E003700FBF30700C7
:109AE4004E4890000080FB00630060000000E0002E
:109AF40003003A004E4890003040B300404F9800B5
:109B04005E009000000F780039010700010050004A
:109B1400200798004E4890005901070009003200C0
:109B24004E48900054010700040032002E009000BB
:109B34000000D1001E0F4000020037002E009000EC
:109B44001E0F4000606A80001E0040000000E80014
:109B540020079800B06A80001007980040688000D1
:109B6400E10F40000C003200260107001E009000A7
:109B74000100400010079800816A800099010700E5
:109B840005003100B80107001E009000008040006D
:109B94000000E90010079800A90007000A0031003E
:109BA400C16A80002E009000808F500013003100A5
:109BB400A500070002003200A801070035003700A5
:109BC400A50007000D0037009D0007000A003600BD
:109BD400716A80002E009000808F500007003100D1
:109BE40099000700020032009C0107002900370099
:109BF4009900070001003700970007009000070054
:109C0400160036009000070014003200716A8000CC
:109C14001E00900001005000A8020700726A800034
:109C240085D62000954278000002780081417800B2
:109C3400854078002E00900019000700730107008A
:109C440006003100B26A8000716A80002E00900024
:109C54000080500000005100B06A88002E0090007F
:109C6400706A8800606A8000A0678800606A80006B
:109C7400A06A880035020700106B8000E70F5000CF
:109C840002003A0084020700C4F907001000200013
:109C9400700798007E0090000080FA000000060023
:109CA4001000FA00000F780021479800220798005E
:109CB40063479800440798006E4090000080FB00C2
:109CC400700798007E0090000000E0001F00320042
:109CD4007E009000E10F500001003200390037008F
:109CE4002E4090000080FB00600798006E009000FA
:109CF4000000E0000A0032006E009000E10F500006
:109D0400010032002F003700AE0090001E007800E2
:109D14004E019000280D02000000000029003700C9
:109D24000080EB009E0F1000030032001E0078003C
:109D34004C680200000000002E009000CE0090004D
:109D4400026C0200000000001E0037002E4090004C
:109D54000080FB00500798005E0090000000E000C7
:109D64000F0032005E009000E10F5000010032004D
:109D7400140037002E009000E10F40000300320071
:109D84002E00900070680200000000001E007800A1
:109D9400CE009000426B0200000000000900370072
:109DA4004E019000AE0090001E0078007C69020015
:109DB40000000000106B0200000000000000E00042
:109DC400FCFF32000080FA00000006000080FB0067
:109DD4007E00B9008000780040C32000008040006D
:109DE400000006004E009000940007001F0037009A
:109DF4000040EB000EEDB7008009200001002000B8
:109E0400406788005167880000000600E00F50009A
:109E1400E08F580000000600E8000700D06A8800C0
:109E2400E16A880000000600610060000004E000B0
:109E3400000006000E10900080804000DC00370017
:109E4400C16A8000E70037004E4890000080FB00A4
:109E54004200DE00F4FF37002E009000C06A880044
:109E64002E009000B06A8800000006001E009000DA
:109E7400AE00900000000600206B8000011020005E
:109E8400640037004E00900065003700BC010700F5
:109E94006700370025020700EA00400000D12000D7
:109EA400008040000000060001688000F067800028
:109EB40080804000B0678000600037000001BE0071
:109EC400D06A8000E16A800094000700CFFF370069
:109ED40042782D00730120005D0037000001BE00B0
:109EE40040782D0071012000CBFF370000C1B30082
:109EF4005C0037008900070060678800716788008C
:109F0400000006000E6890005D0037000080FB0032
:109F14004400DE005D003700CE009000730037007F
:109F2400BB0107008F003700A2010700EB01070007
:109F3400910037007E089000A10107000080FB001B
:109F44004200DD00000006008E00070080678800E4
:109F540091678800B16A8000000006008E109000AE
:109F64004E08900000805000D4010700756A8000FC
:109F74000002780055000700050078000000060084
:109F8400716A8000806A8000E50107000000E90032
:109F9400000006005000070000804000000006009A
:109FA4000E1290004900070085407800000006006A
:109FB4009E0890000E10900000814000660007008B
:109FC400E067800000804000800F51000000060020
:109FD4009E0890000E109000808040004068800031
:109FE40000000600070007001E089000000006009D
:109FF400CE0090005E009000808040002E00900013
:10A004000000060054000700E067800080804000E4
:10A0140000000600010060000000E00000000600EF
:10A0240000017800A5010700906A80000000060086
:10A034000000EB00000F7800000006008080400064
:10A04400C067800000806800306B88000000060054
:10A054000000410081804900D06A8800E16A8800DC
:10A0640000000600204798001000200030079800E8
:10A07400000006000E6890000080FB006AFF3700B5
:10A084000080FB000000D10067FF37006100600022
:10A094000000E000000006000E0890006101B80016
:10A0A4002E089000BE0890003300370041010700DD
:10A0B400A1678000A06A800000805000CF80DE008D
:10A0C40016003700A2678000190137008041EB00B9
:10A0D4000081EB000000060085D620009542780040
:10A0E400B16A80001E089000000006001182FB0087
:10A0F400114090007C01070004007000000178000A
:10A10400214090000082FB0031409000760107005E
:10A114000400700080017800000006000000510077
:10A12400818059000000060050688000D7FF370086
:10A13400FF0007006101B8005E089000EE0890007F
:10A14400000006000080500024010700A06A80007F
:10A15400A067880000000600406880008000780046
:10A164000000060061004000E0804800806788002D
:10A174009167880000000600800F5100818F59000C
:10A1840000000600010020000C0037005E01900072
:10A19400EE0190005E089000EE089000DFFF0700DB
:10A1A4000D0007005E089000EE08900017FF3700CE
:10A1B400806A8000808F500000000600020040008A
:10A1C4008380480000000600400F98004E0890006D
:10A1D4000000E00000000600500F9800610F980096
:10A1E400000006001E009000808F50000000060052
:10A1F4000000EB003007980000000600450107004E
:10A204001E0010003007980000000600B16A8000AC
:10A21400C06A8000808F5000000006002E0090006D
:10A224000000E000000006000000EB00500798006A
:10A23400000006003E0090000000E0000000060060
:10A244001E010700C26A80003E0090000000060064
:10A254009E0078003E009000000006000000EB0025
:10A264007007980000000600716A8000806A800010
:10A27400808050000000060070079800FE009000E7
:10A284003E189000808F500000000600BE409000F1
:10A2940000C6B30080CF500000000600BE4090000E
:10A2A400A0C7B30080CF5000000006003E409000DD
:10A2B40001CEB30001404000304798000000060082
:10A2C4002E4090008080FB0000000600A9000700DB
:10A2D4003E40900080CF5000000006003E189000E1
:10A2E4000000E900301F98003E1890000000E000D4
:10A2F40000000600DE0090004E00900080805000B8
:10A304004E4090000080FB00008040000000E80008
:10A31400701F98000000060099000700100020003C
:10A32400000F780000000600206B8000010420006C
:10A3340038FF370099000700100078000000E000A3
:10A344000000060095000700900078000000060059
:10A35400E1CF200009000900B0587800A000B10046
:10A36400000006007400B90000017800EF00070047
:10A374008000780040D220000080400080027800F5
:10A38400890007000202780013C0B30005017800B9
:10A3940011C0B30000000600206B80007000600054
:10A3A4000000E00000000600F06780000168800003
:10A3B400000006000ECDBF000040E8000EEDB7001F
:10A3C40040678000516780000000400081804800A1
:10A3D4008BFE3700206B8000680060000000E00006
:10A3E4000000060040C1B300204798001000200080
:10A3F40020079800000006000ECDBF00E24F500079
:10A404000000060010C1B30016FF3700A1678000EA
:10A41400A06A8000808F5000000006002001980090
:10A4240031019800000006007C00470051009800AC
:10A434007C004700000006007C00470050009000AC
:10A44400000006001FFF070000005100A0678800FD
:10A4540000000600206B800001802000EDFE370024
:10A464004267800053678000F9FE3700816A8000EC
:10A47400706A800000815000B16A8000C06A800068
:10A4840000805000000006003E0090001000900084
:10A4940000000600000178007440B900F20040009A
:10A4A400530007008000EB005107980000000600ED
:10A4B400800078001E0078000000060015000700E8
:10A4C4000004E00000000600160007004400DE005F
:10A4D40055FE37006E489000E9FE37003C00070047
:10A4E40030079800410798004400070011C0B300EA
:10A4F40040C0B30000000600450007007EFE3700A0
:10A504006E489000DCFE37002E089000BE089000D4
:10A514003EFE3700030007004200DE0061006000D9
:10A52400000006006E4890000080FB00000006005A
:10A53400716A8000606A800000805000000006009C
:10A54400706A8000808F500000000600606A8000FE
:10A55400906A880000000600206B80000102200041
:10A56400ACFE3700604798004107980052079800F6
:10A574000000060054000700904078000000060028
:10A584002E18900090407800314798002E189000C3
:10A594000000E800201F9800000006006300070088
:10A5A400F00040003DFE37005200070000804000EC
:10A5B40000000600626780007367800000000600E8
:10A5C400600090004400DE006F4060000000060060
:10A5D400606780007167800000000600E9FE0700E4
:10A5E40045FE37004000070001007000000006002F
:10A5F4002AFE070002087800000006005E019000B1
:10A60400EE0190006267880073678800000006000E
:10A614003E009000CE0090000000060039000700C4
:10A6240080007800004C2B000080400000000600F1
:10A63400214090000081FB00314090002A00070077
:10A644000200700000017800000006009080FB000A
:10A6540010409000E3FF0700800041000000060066
:10A66400004F780050C0B3009E4F10000000060059
:10A674001000200010079800000006000000EB0006
:10A684001007980000000600916A8000A06780000F
:10A69400808F50000000060011C0B30000C1B30059
:10A6A400000006000000EB002007980000000600F0
:10A6B4000000E900200798000000060081D6200071
:10A6C40091407800000006004E4090008080FB001E
:10A6D4007200470000804000000006005E00900009
:10A6E400EE009000000006000080FB004800DD0042
:10A6F400000006000D0007008000780000D1200053
:10A70400000006003E4890000080FB006600B9008F
:10A7140000000600100798001E00900000000600CC
:10A724000080500000004100000006001E00780078
:10A734007400B900000006000800FA00008FBE0093
:10A744001E00BE00200798003107980090002000EA
:10A75400010020002E019000BE0190008007070038
:10A764002B003E002E009000BE009000006001000F
:10A77400090037000B0037000D0037000F003700C9
:10A784001100370013003700150037001700370099
:10A79400190037001B003700E09C2900A5060700BC
:10A7A40020003700C2AD0200000000001D00370089
:10A7B400909D29009F0607001A003700D2AD0200C1
:10A7C400000000001700370030AE02000000000057
:10A7D40014003700FCAD0200000000001100370037
:10A7E4001AAE0200000000000E00370044AE020062
:10A7F400000000000B0037007EAE020000000000E5
:10A804000800370092AE0200000000000500370087
:10A81400439E2900E1070700830078006C39020099
:10A82400000000000080FA00000006000000FA00AA
:10A834009C070700E1C7B300F238020000000000E3
:10A844000080FA00000006000200FA00881F780069
:10A854000040EB0098F0B7001D0037009407070094
:10A8640098D0BF000084FB0084C0B300030520001F
:10A874000041EB006000B8006A36020000000000EE
:10A8840000417800010921004240DD000080E80019
:10A894000100400002487800890707008B07070081
:10A8A400B40607004C680200000000008A07070095
:10A8B400026C0200000000001E0078004C680200D8
:10A8C4000000000098D0BF000040E80098F0B700F6
:10A8D40098D0BF00E14F5000E0FF36000040EB008D
:10A8E40098F0B7004F0478000080FA0000000600DA
:10A8F4000200FA000040EB00004F78002B00370004
:10A90400B6060700E24F400027003200B3060700F6
:10A9140076370200000000000000E000160032005C
:10A924001E40780026000700610707006D07070036
:10A93400040032000ED0BF00A0B8020000000000E6
:10A944005F0707000FD0BF00E14F40000400320052
:10A954000FD0BF00A0B80200000000005B07070092
:10A964005007070043C0B3000001EB0011002000B2
:10A97400404D0200000000001E80FB005C07070041
:10A984000000E00005003A0094060700743A020053
:10A99400000000000000E000030032001E407800C8
:10A9A40007000700240007001E4FE80010C0B30092
:10A9B4009E4F1000D2FF36000080FA00000006000F
:10A9C4000400FA0020479800810921009140780092
:10A9D4002E409000814F500015003200650607009C
:10A9E4004C680200000000003B070700026C0200F4
:10A9F400000000001E0078004C6802000000000007
:10AA04002E4090005C060700706802000000000001
:10AA140031070700426B0200000000001E007800AE
:10AA240070680200000000002E40900098F0B7000B
:10AA34000080FA00000006002A00FA00881F78004F
:10AA44003007070098D0BF000080FB0028070700EC
:10AA54006101B8000217980013179800B000200095
:10AA6400010020000E1190009E119000BC0607000A
:10AA740034033E000E1090009E1090000060010010
:10AA84000B00370028003700140137007601370027
:10AA94009001370094013700DE013700ED013700E3
:10AAA40054023700F7023700070337001403370056
:10AAB400FC060700743A02000000000014070700B7
:10AAC4000000E0001F033200600121005080880074
:10AAD4003E070700100020008008780000C0EB004B
:10AAE40011F0B7000040EB0010F0B700EE200200B8
:10AAF40001000000090707000080EB008080EB00E4
:10AB04000E070700230607000040EB008EF0B70095
:10AB1400E406070053C0B3000001EB00110020005D
:10AB2400404D02000000000007070700183E020025
:10AB340000000000E10F40000F003A00D9060700B2
:10AB44009C3B0200000000000000E00001003A000D
:10AB540024060700EE20020001000000FD060700A5
:10AB6400F8023400CF060700BC37020000000000E2
:10AB740065060700F3023700EE2002000100000022
:10AB8400E6060700FB060700183E0200000000006E
:10AB9400DF060700E50F50000200360050002000D9
:10ABA400400798007106070061012100023B020082
:10ABB400000000003200200021102A006001210062
:10ABC400200C0200000000000000E00003003A0036
:10ABD4000000EB00908088000D0037004200200048
:10ABE40061102A0060012100200C02000000000016
:10ABF4000000E00003003A0010002000908088006C
:10AC04000300370070002000F7050700CD0237006D
:10AC1400D8060700183E0200000000004007980014
:10AC240055060700F1C3B300183E020000000000FF
:10AC340030079800CE009000311798003E01900034
:10AC440022179800AE1190003E109000808F5100A2
:10AC540002003600BE109000211798002E119000BB
:10AC640042079800CE009000B0062000808F50006C
:10AC740002003600DB050700B20237004206070077
:10AC8400023B020000000000300798004206070063
:10AC94004606070060012100D5030700600121007A
:10ACA400740D0200000000003007980070012100BC
:10ACB40072002000B1102A00200C020000000000E5
:10ACC4000000E0000F003A0070012100DAA7020042
:10ACD4000000000011F0B700908080000000E00048
:10ACE40003003A00800020009080880002003700B2
:10ACF40090002000908088002F06070003060700BC
:10AD04009002370030060700040032007001210071
:10AD140062B70200000000000EF0B70071060700E1
:10AD240013003A0028060700030032001A06070041
:10AD3400F0C2B3002D060700BE00900060012100A0
:10AD44000080400023112A000B00090033587800CA
:10AD5400C000B1003E0090006B0040003007980036
:10AD64007001210062B70200000000000EF0B7007D
:10AD74003E009000610121008100E900010F4000C4
:10AD8400060037001E00780090407800E0C2B3004F
:10AD940080CF5000040032001E0FE9006001210042
:10ADA4009E0F1000F7FF3A001E0FE8000000EB00B2
:10ADB400A08088000E003700A08080008000400042
:10ADC400E0A1290000804000100078008000780095
:10ADD4001E00780036B40200000000000004E00009
:10ADE40006003200A08080000000E800A0808800F7
:10ADF400A0808000EA0F5000EFFF360070012100B0
:10AE0400DAA702000000000011F0B70035060700C1
:10AE14000E0032000ED0BF00E6BB020000000000AE
:10AE24000000D100610060000004E000070032006F
:10AE34000ED0BF00F4BC0200000000000000E800D7
:10AE440052B80200000000000FF0B70049060700E6
:10AE5400183E0200000000002D0607000000E0007C
:10AE64001500320010C0B30010F0B7000D06070043
:10AE7400EA004700A63A0200000000004E009000DD
:10AE84000000E90040079800CE0090005007200021
:10AE9400808F500002003600520507002902370057
:10AEA40058808000B8050700023B02000000000043
:10AEB40000004400D205070023060700183E0200E4
:10AEC4000000000040079800D4050700023B020080
:10AED40000000000B8050700000037001A0607004C
:10AEE400183E02000000000009060700E10F4000C0
:10AEF4000F003A00EB0507009C3B02000000000035
:10AF04000000E00001003A0036050700EE200200D0
:10AF1400010000000F0607000A023400E1050700E3
:10AF2400BC37020000000000770507000502370067
:10AF3400EE20020001000000F80507004E0090001A
:10AF4400E10F50000A003A00D60507002200200055
:10AF54008000EB00023B0200000000001B0607001B
:10AF6400300020008008780068050700F5013700EC
:10AF740081050700A1C3B300183E020000000000D1
:10AF84000080E80030079800600507003E0090004C
:10AF9400F00F500004003600A0050700023B020039
:10AFA40000000000CDFF3700BE050700EB0047009E
:10AFB4003E019000023B0200000000003E009000B1
:10AFC4000001E900EB0047000040EB0000F17800CD
:10AFD400CE0090003E009000008050004007980092
:10AFE4000040EB0040479800120037004E409000AC
:10AFF4000080FB0080004000C00F2A000080400059
:10B00400900078006B004700540C02000000000020
:10B014000000E00004003A004E4090003A020700AD
:10B02400B8050700060037004E4090000040E800D5
:10B03400404798004E409000E24F5000EBFF36002E
:10B044007905070004003200BF050700183E02001E
:10B05400000000004007980070050700023B020052
:10B06400000000009DFF370011D0BF000004E00085
:10B074000300350030002000DB040700B101370075
:10B08400518080004905070060012100D8020700B3
:10B094005080880090808000E80F500002003A0041
:10B0A400D2040700A7013700C805070040002000AC
:10B0B4008008780010D0BF000004E00001003A00CE
:10B0C4005C050700110507000040EB0010F0B70015
:10B0D4009C0137003EA8020000000000E20F50006F
:10B0E40098013200530507006E050700743A020008
:10B0F400000000006101B800BF04070009003A0025
:10B10400EE20020001000000920507000500340053
:10B1140064050700BC37020000000000FA040700C1
:10B124008801370090808000E10F50000600320053
:10B1340090808000E80F500033003600908080003B
:10B14400EB0F500030003E0090808000E80F50006C
:10B154000A00360090808000EB0F500007003E008C
:10B16400A0030700204F98002E4890000004E00040
:10B1740005003A009D04070072013700A6A80200EA
:10B1840000000000204F98002E489000E24F50002D
:10B1940007003A0043050700743A0200000000006B
:10B1A4000000E90001002000640507006501370084
:10B1B4002E489000E14F500013003A003905070073
:10B1C400743A020000000000010020005B05070043
:10B1D400EE2002000100000050050700680507008A
:10B1E40085040700050036002E0507009C3B02007D
:10B1F400000000000000E00052013A00600020005E
:10B20400790407004F013700700507006000200033
:10B21400800878003305070003003A00400020004E
:10B2240071040700470137005A0407000FD0BF001C
:10B23400E14F400002003A00020507000400370015
:10B244000FD0BF00E1FF200060B902000000000041
:10B254005A0507001305070023C0B3000001EB00E3
:10B2640011002000404D020000000000908080008A
:10B2740080004000800B2A0062040700183A020094
:10B284000000000090808000EC0F50000D003A0098
:10B29400F1040700183A020000000000E2112A003D
:10B2A4005B040700183A020000000000EA040700EB
:10B2B400183A020000000000EA040700183A0200ED
:10B2C40000000000908080000000E00005003200D3
:10B2D40090808000E10F5000020032002B0507002F
:10B2E40018013700A0808000EB0F50000D003200E1
:10B2F40012132A0046040700183A02000000000056
:10B30400A080800080004000E0A929003D040700DF
:10B31400183A020000000000D2040700183A0200A4
:10B32400000000000ED0BF00E6BB020000000000D9
:10B33400610060000004E0000400320002142A00EE
:10B3440033040700183A02000000000092152A0096
:10B354002F040700183A02000000000090808000CB
:10B36400E10F500006003200F27F8000038080006D
:10B374000080EB008080EB007904070005003200B8
:10B3840092162A0022040700183A02000000000066
:10B394000800370022172A001D040700183A02008B
:10B3A40000000000B2172A0019040700183A02002E
:10B3B40000000000AB040700183A0200000000007F
:10B3C40010D0BF000004E00004003200FF040700B6
:10B3D400800020008008780004003700A1040700E2
:10B3E400183A020000000000A10407004704070007
:10B3F400D400370060012100608088009A00370083
:10B40400F2172A0002040700183A020000000000A4
:10B4140033003700AE48900000C2B30080CF500024
:10B4240004003A0096040700F2380200000000000D
:10B434002B003700AE489000F0C2B30080CF50001C
:10B4440014003600AE48900090C3B30080CF500083
:10B4540004003600AE48900000C4B30080CF500012
:10B464000C003600AE489000A0C5B30080CF500059
:10B4740004003600AE48900000C6B30080CF5000F0
:10B4840004003600AE489000A0C7B30080CF50003F
:10B49400100036007D040700F238020000000000AE
:10B4A4002E48900000B4020000000000DB030700F7
:10B4B400F2380200000000002E4890001CB4020084
:10B4C40000000000D5030700F2380200000000006D
:10B4D40003003700D3030700F23802000000000025
:10B4E40060808000700F9800FE0890001140780082
:10B4F400204F98002E489000006F98000E6990002D
:10B504000204E0000200320013C0B300036F98008D
:10B514008E6890007E0990000200E8006080880038
:10B524000104E000BBFF3A005E040700D1C3B3008E
:10B53400F23802000000000033003700AE489000EB
:10B5440000C2B30080CF500004003A004C0407004E
:10B55400F2380200000000002B003700AE489000D3
:10B56400F0C2B30080CF500014003600AE48900003
:10B5740090C3B30080CF500004003600AE48900062
:10B5840000C4B30080CF50000C003600AE489000D9
:10B59400A0C5B30080CF500004003600AE48900030
:10B5A40000C6B30080CF500004003600AE489000BF
:10B5B400A0C7B30080CF500010003600330407004A
:10B5C400F2380200000000002E48900000B402008F
:10B5D4000000000091030700F238020000000000A0
:10B5E4002E4890001CB40200000000008B030700EA
:10B5F400F23802000000000003003700890307004E
:10B60400F23802000000000063808000630F98009D
:10B61400EE08900011407800204F98002E489000CA
:10B62400106F98001E6990000204E00002003200CE
:10B6340013C0B300136F98009E6890006E099000C9
:10B644000200E800608088000104E000BBFF3A00CB
:10B6540004040700183A02000000000010D0BF00E4
:10B664000040E90010F0B70010D0BF000004E00073
:10B6740063FF3A00FB030700183A020000000000D1
:10B68400FB030700A1030700330007000000E000EC
:10B69400060032000ED0BF00A0B802000000000077
:10B6A400070407003904070016040700FD03070018
:10B6B400A6380200000000000000E00021003A006B
:10B6C400100407001F0037000E040700F5030700ED
:10B6D400A638020000000000EF0F500019003600E9
:10B6E400108080002180800013FC07004F030700B6
:10B6F40014003A0085030700DD030700110037003A
:10B70400F8030700040032000ED0BF00A0B8020006
:10B7140000000000EA0307000FD0BF00E14F400023
:10B72400040032000FD0BF00A0B8020000000000E7
:10B73400E6030700DB030700BC370200000000003B
:10B74400DB030700B8030700BDFC32004F04780098
:10B754000080FA00000006005200FA00D10307003E
:10B76400A638020000000000000F7800F27F80007D
:10B77400038080006B0307000001510081815900A0
:10B784001E0078006102B80074279800052F980005
:10B7940052279800632798005E209000EE209000C6
:10B7A4007E2190008E299000820F5000838F5800D4
:10B7B400040036007E2290008E2A900054279800C0
:10B7C40065279800DE22900015079800EC03070017
:10B7D4001E00900001002000020040008380480009
:10B7E400ED020700180037001E0090001403070044
:10B7F4000200360002042000422798000ED0BF0049
:10B80400E50047004E2190000AB902000000000044
:10B81400000F78001E00E00003003A00130020002F
:10B8240033279800350037009E030700E5004700E2
:10B834001E0178006C390200000000001E00900018
:10B844001E0050001007980077030700E6FF3A0037
:10B85400CB030700F07F80000180800040030700D5
:10B8640024003A00D9030700A000200080087800D3
:10B874006000B800B10307000ED0BF008000EB00E9
:10B88400B2B80200000000000ED0BF00E400470080
:10B89400B2B80200000000000000E0000500320021
:10B8A400EC020700CE409000E0C7B30080CF500008
:10B8B400F5FF3A00E70207000FD0BF002100210086
:10B8C40060B90200000000000FD0BF00E1FF2000BB
:10B8D40060B90200000000000000E00005003A002A
:10B8E400580307000FD0BF00A0B8020000000000FA
:10B8F400760307000002EB00342798003E209000F6
:10B904000080FA00000006000200FA00004F7800F0
:10B914001E04E00002003A00580007000900370046
:10B9240010C0B3009E4F100002003A000700070049
:10B934000400370020C0B3009E4F100001003A00FD
:10B944008F0007000080FA00000006002E00FA00B5
:10B9540011D0BF000004E000460035005103070089
:10B96400620020008000EB00023B020000000000A7
:10B97400BC020700743C020000000000BD02070086
:10B9840063004000100798009E009000C00F200044
:10B9940000806000B7020700601798004002200092
:10B9A400EE109000808F500002003600400220000C
:10B9B40060179800EE10900011079800640F47007C
:10B9C4000F003700750307009E007800023B020059
:10B9D40000000000330020001E0178004100200018
:10B9E4001E00780006B20200000000001E00900055
:10B9F40064005000100798001E007800630F400098
:10BA040009030700EFFF3A001E0078008040EB00B6
:10BA140001487800BD020700640F470009003700A1
:10BA24001E00780090407800A0C3B30080CF50007F
:10BA3400080032001E0090000000E8001007980083
:10BA44001E0FE8009E00900070022000808F5000BE
:10BA5400F3FF36009E007800D40207001E0FE800B2
:10BA6400640047009E00780010A802000000000057
:10BA740011F0B7000080FA00000006000A00FA0086
:10BA840078020700743C020000000000000F7800F8
:10BA94006001210061072000808040005080800008
:10BAA400008050009E0F500031003E0050002000E6
:10BAB40090808800410307002F0037009C02070094
:10BAC400B1C3B300183E0200000000001007980044
:10BAD40050808000300798009E0090004107980035
:10BAE4001E00780020079800AE0090004E009000E1
:10BAF400808F500002003600CE009000210798008D
:10BB040053808000E70207002E0190008300780034
:10BB1400023B020000000000BE00900000804000D4
:10BB2400B70207001E0090009E0F50000C00310069
:10BB340053020700A63A0200000000000300370089
:10BB44004F020700A63A02000000000009030700A4
:10BB5400183E0200000000000000E000F8FF320080
:10BB640040020700743C020000000000000F78004F
:10BB74001E00E000D1FF3A000080FA000000060039
:10BB84000C00FA0037020700743C020000000000B9
:10BB9400000F7800900020009E0F10000400360073
:10BBA4002000200090808800FA0107000E00370072
:10BBB400BC0207008E80E8001E017800023B0200F0
:10BBC40000000000000F78009E0078000E80E8005E
:10BBD40080804000750207000E80E800900D02008E
:10BBE40000000000EC0107000080FA0000000600DD
:10BBF4000C00FA00500798005E009000740D0200DB
:10BC040000000000100798005E00900020079800D4
:10BC14002E00900030079800330037003E0090005B
:10BC2400104F780019020700D0C3B3009E4F1000D4
:10BC34000300320060C2B3009E4F100002003A00BD
:10BC4400D801070028003700B0C2B3009E4F10008F
:10BC540004003A00AE00900000C2B300D301070014
:10BC64002100370050C2B3009E4F10001B003A0061
:10BC74001E009000E10F500002003E002302070066
:10BC840019003700680047008000E8003E0090007B
:10BC94001040780055020700E80047003E0090007D
:10BCA4001040780080487800F80107001E009000DA
:10BCB4000000E900100798006800470010007800B1
:10BCC4008AB3020000000000804078002E0090003B
:10BCD40001487800B6010700030037002E009000E9
:10BCE4001E487800B20107004F020700CBFF3A005C
:10BCF400AC010700AE0090002C0207002E0090005B
:10BD04000080FA00000006000600FA00000F780028
:10BD140011079800170037009E0078001E0090005D
:10BD2400540C0200000000000000E00007003A008C
:10BD34001E009000740D0200000000001E00400070
:10BD44000000E80020079800100037001E0078006B
:10BD5400740D0200000000001E004000000FE80007
:10BD64001E007800740D0200000000001E00400058
:10BD7400000FE8001E007800104078000004E00086
:10BD8400E5FF3A000000EB00200798002E00900029
:10BD94000080FA00000006000600FA00C201070055
:10BDA400D0C3B3002D000700000F78001E02070067
:10BDB400060032001E009000104078000004E000ED
:10BDC400020032001E00900089FF07001E00780068
:10BDD4000080FA00000006000600FA00889FBE00FA
:10BDE400B101070060C2B3001C000700000F780017
:10BDF400200020009E0F10000C003A0026020700CD
:10BE0400743A02000000000001002000800F54007A
:10BE1400818F5C0005003A002E0190009E00900086
:10BE24000040EB000D000700000F7800FE01070042
:10BE3400060032001E009000104078000004E0006C
:10BE4400020032001E00900069FF07001E00780007
:10BE54004F04BE000080FA00000006000C00FA0047
:10BE6400889FBE0040479800310798004207980019
:10BE74004E4090000004E00006003200AC010700D0
:10BE8400CE409000183E020000000000000F780031
:10BE94000400370003020700743A020000000000A7
:10BEA400000F78000080EB009E0F100003003A00A2
:10BEB4002000200050079800460037004E009000F4
:10BEC400E10F500009003E003E0090000000E00039
:10BED4000600320079010700023B02000000000066
:10BEE4007901070007020700300037003E00900088
:10BEF4000000E00006003A0070010700023B020067
:10BF040000000000700107008001070027003700CF
:10BF14004E0090000080E9009E0F5000190031008F
:10BF2400D87F8000E97F80004E0090000081E90006
:10BF3400DC010700BE009000023B0200000000008C
:10BF440061010700D87F8000E97F80004E009000E7
:10BF54001E0010000081E80049010700023B0200B6
:10BF64000000000058010700CE0090003E00900041
:10BF7400008040008080E9008C010700E101070097
:10BF84000A0037006E010700BE009000023B020069
:10BF9400000000004C0107009E0078003E00900065
:10BFA4008080400081010700580107004E40900046
:10BFB4000004E00005003200B70107008000EB0038
:10BFC400A63A0200000000003F0107001E00900096
:10BFD400500798005E0090004F04BE000080FA00F5
:10BFE400000006001A00FA00889FBE0090808000BE
:10BFF400400F98004E089000EA0F50005A0032009B
:10C004004E089000EB0F5000440032004E089000A0
:10C01400E90F50000100320080003700C6182A00E2
:10C024004A0107004200200086007800743C0200A8
:10C03400000000000F010700E10F40002E00320055
:10C04400980107001E0190008000EB00023B0200F3
:10C0540000000000DA00070092010700743A0200B1
:10C0640000000000E90F500006003E001E00900092
:10C074000000E8001007980010002000300F98001E
:10C084006800370014010700A2002000023B0200F0
:10C0940000000000CA00070064004700A20020005E
:10C0A40011192A00200C0200000000000000E0002A
:10C0B4000C003A00A00020009080880070BA0200B2
:10C0C400000000000EF0B70064004700E4004000E8
:10C0D4000ED0BF0062002000F8BA02000000000089
:10C0E40002003700B000200090808800200020006B
:10C0F400300F98004B0037006A010700743A0200C1
:10C104000000000064015000DD000700023B020053
:10C1140000000000AA000700400037005E0107008D
:10C12400743A020000000000E70007005D01070008
:10C13400583A020000000000910107003006200078
:10C144000100200006010700050036008C010700ED
:10C154000000200001002800010107002F00360024
:10C16400E00007002F0037004E010700743A020078
:10C1740000000000BF0007006101B800E9000700EB
:10C18400F70007001A003600E600070010079800C1
:10C19400170037001E009000200F98002E08900012
:10C1A400F00F50000200360000012000200F98001C
:10C1B400C90007002E099000023B020000000000A5
:10C1C400000F78006E0107001E0078007F00070052
:10C1D4001E0090001E005000100798000ED0BF00F3
:10C1E400E40047001E017800F8BA020000000000D5
:10C1F4000D010700E7FF3A00CA000700E00F5000F6
:10C20400E08F580005003A001000200052BB0200E5
:10C2140000000000B30007000200370010002000F7
:10C22400300F98003E0890004F04BE000080FA00D2
:10C23400000006004A00FA00881F780030279800A2
:10C244007A0007000D003A003E20900062B7020019
:10C2540000000000004F780000C0EB009E4F10006B
:10C2640041003200680021001E407800F4BC020046
:10C2740000000000000C78000F003700600021006F
:10C284001000780052B8020000000000004F78004F
:10C2940080C0EB009ECF100033003200600021000C
:10C2A400100090006101B800210020001E407800B9
:10C2B40080B9020000000000FA000700A63802005E
:10C2C40000000000200798001C0037002E0090009A
:10C2D4005B0007000200360000042000402798009D
:10C2E400E60047004E2190001E4078000AB9020083
:10C2F4000000000010079800CB00070006003A0079
:10C304001E407800A0B80200000000006000B800E1
:10C314000A01070014003700E2000700E6004700A6
:10C324001E0190006C39020000000000AE00900075
:10C334001E00900000805000200798002E009000FE
:10C344000000E000E1FF3A00680021001E40780090
:10C35400DCBC020000000000100498001E407800BD
:10C36400A0B80200000000004F0478000080FA002A
:10C374000000060098D0BF008080FB006009200008
:10C384000088B9008000780000ED210000804000A2
:10C39400000006006000B800D07F8800E17F8800BC
:10C3A40000000600AE0090000040EB0080487800DA
:10C3B4002E0090000000E80020079800000006000E
:10C3C40010079800EE0007001E00900001002000F6
:10C3D4000000510081805900EFFF37001E80FB00F0
:10C3E400430037005000200090808800F0000700D0
:10C3F4001007980000000600308080004180800013
:10C4040057003700008040001000780000017800D9
:10C41400A4000700820078000000060000417800B4
:10C424003D0037002E4990003B00370030808000EB
:10C4340041808000E00F5000E08F580000000600AB
:10C444004027980000042000CE209000808F5000E8
:10C45400000006003300070061004000E08048004F
:10C46400CDFF37003900070022002000919E2900EB
:10C4740000000600100798001E009000000006004F
:10C48400880007008000EB00000006003E009000DA
:10C494000000E800300798001E0090000000E9004A
:10C4A4001007980000000600100798002107980064
:10C4B4002E0190009E00900000000600200007005E
:10C4C4008000EB0000000600010020000000540082
:10C4D40081805C00B0FF370072000700E400470071
:10C4E40000000600B2000700300F980000000600AC
:10C4F400010921004200DD000080E8000100400045
:10C504001040780000000600A00007000000EB00C7
:10C5140010079800000006006200070082407800BF
:10C5240000000600D07F8000E17F8000000006004C
:10C534009C0007008001EB000001EB0000000600F6
:10C54400550007001E017800000006005500070092
:10C554008002EB000002EB008001EB00000006000B
:10C56400800F5100818F5900000006004E0090009A
:10C574000001E8004B0037008A000700CE0190005C
:10C584000001EB0000000600460007004E01900089
:10C5940061012100000006003E009000FC00400004
:10C5A400A0FF200080804000000006000040EB0057
:10C5B4008048780000000600840007002000200066
:10C5C40080087800000006003E0090000000E900AA
:10C5D400FC004000A0FF2000008040009040780054
:10C5E400F0C2B30080CF50000000060080487800FD
:10C5F4003E0090000000E8003007980000000600AC
:10C60400508088005180800060C2B3008048780068
:10C614000100E8005080880000000600D3FF0700F6
:10C624008000EB00000006001E0090000000E00007
:10C634000000060065000700500020008008780014
:10C64400000006000080EB008080EB00F07F880093
:10C65400018088000000060012000700610121002B
:10C66400000006000F000700919E2900000006004C
:10C6740056000700900020008008780000000600A3
:10C6840008000700B1C2B30000000600050007005F
:10C6940051C2B30000000600D87F8000E97F80000B
:10C6A4000000370098D0BF000080FB0090FF3700E7
:10C6B400460007000000EB00800878000000060038
:10C6C40000C0EB000EF0B7000000060000C0EB0055
:10C6D4000FF0B70000000600000F7800A0FF200054
:10C6E400610905000ED0BF00E14F400000000600C4
:10C6F400010921004200DD00010040001000780023
:10C70400000006001000200010079800000006003A
:10C71400400798004E009000000006000001BE0093
:10C72400209D2400B10620000200400083804800C0
:10C734001080880021808800000006003080880076
:10C74400418088000000060079FF0700A1C0B30003
:10C75400000006000001BE001080800021808000DF
:10C764000000510081805900E00F5000E08F580014
:10C77400000006006EFF070001C2B30000000600BF
:10C78400D27F8000E37F8000000006000F000700D6
:10C79400B00020008008780000000600C1FF0700F8
:10C7A40042000500BFFF07000002EB000000060086
:10C7B400020007000000EB00000006000300070071
:10C7C40070002000800878000000060098D0BF00A8
:10C7D4000080FB00010921004200DD0081004000CF
:10C7E400000006000400FA00CD22A800C922A90016
:10C7F4000000EB0000128800F000200010128800F6
:10C804000000EB00201288004302A80042A2A80006
:10C8140041E2A80000003700320407000E80E8005F
:10C82400D1C1B300440407002E409000004F7800AB
:10C834001E80FB004300DE00610060000004E00095
:10C84400F5FF3A001E80FB000080EA0061006000F2
:10C854000004E000F0FF3A001000200020B588003A
:10C864000000EB0000B588008040EB0080C0B300FE
:10C874007E0407008040EB0090C0B3007B040700F7
:10C8840011CAB300C0C0B3007804070091C0B3005C
:10C89400D0C0B3007504070011CAB300A0C0B30030
:10C8A4007204070091C0B300B0C0B3006F04070066
:10C8B40021CAB30040C0B3006C04070091C0B300A8
:10C8C40050C0B3006904070021CAB30020C0B300FC
:10C8D4006604070091C0B30030C0B30063040700CE
:10C8E4000040EB00B603070000202000B40407005A
:10C8F400D1C0B3000040EB005C04070021C3B300C7
:10C9040020C0B3005904070021C1B30040C0B300E4
:10C914005604070001C4B30030C0B3005304070039
:10C92400F1C3B30090C0B3005004070021C1B300A9
:10C9340060C0B3004D040700C1C0B30070C0B300B1
:10C944004A040700E1CEB300A0C0B30047040700C7
:10C9540051C0B300B0C0B30044040700403020000D
:10C9640097040700F18220009140780040C0B30092
:10C974003E040700018320009140780050C0B300BA
:10C984003A040700118320009140780020C0B300CE
:10C9940036040700218320009140780030C0B300A2
:10C9A4003204070031832000914078000040EB00FE
:10C9B4002E040700418320009140780010C0B3008A
:10C9C4002A0407008040EB0050C1B300270407008D
:10C9D4006300470021C1B300D70307003E40900025
:10C9E400A6F6B7000110200000C1B30058040700E8
:10C9F4002147230040C1B300550407008000EB0029
:10CA04000040EB00520407000000EB006C04070038
:10CA140041C0B300F0C1B3003B0407000080FA003A
:10CA2400000006000200FA0011C0B3000E007800F6
:10CA3400E70307001E0078004200DE00614060004A
:10CA44000080FB000080FA00000006000200FA00EB
:10CA5400F1C1B3000E007800B70307001E40780050
:10CA64000080FB004300DE000004A2000080FB0005
:10CA7400610060000080FA00000006000200FA0075
:10CA840020B580000000E00011003A0010002000F2
:10CA940020B5880000B580000000E900A904070063
:10CAA40002003600109A2000000F780001C4B30081
:10CAB400E0C1B300140407009E407800C0C0B30076
:10CAC400EA0307009E409000D0C0B300E7030700CC
:10CAD4000080FA00000006000C00FA00901120000B
:10CAE400370407006400470091C1B30092030700B4
:10CAF4004E409000004F7800E00020003004070012
:10CB040065004700E1C0B3008B0307005E4090005E
:10CB14002047980066004700F1C0B3008603070071
:10CB24006E409000304798009011200024040700C4
:10CB34006700470091C1B3007F0307007E40900067
:10CB4400804078001E40780080CF5000E5FF3A0016
:10CB5400C00020001A04070068004700C1C0B300E9
:10CB6400750307000E489000004F780069004700E5
:10CB7400D1C0B300700307001E489000104798000E
:10CB84009E0090001E007800808F50000700360041
:10CB94009E0090001E00780080805000109A2000B3
:10CBA40001005000500798000C0037009E009000D0
:10CBB4001E007800808F500003003A00109A200075
:10CBC40050079800050037001E0078009E00900072
:10CBD400010050000000E900500798005E0090003A
:10CBE4000080FA00000006001E00FA00300F9800D2
:10CBF400410F980090112000F10307007A004700CC
:10CC040091C1B3004C0307002E589000004F7800E8
:10CC14000000EB00EA0307001E04E00003003A00F2
:10CC24000000EB00600F98005D00370020B5800025
:10CC34000000E00004003A0090FF07000000EB0051
:10CC4400600F98005600370000B5800010B58800CA
:10CC5400216A2100914078000040EB008303070023
:10CC6400316A21009140780010C0B3007F030700AF
:10CC74000E80E80041012000810207000E80E800D8
:10CC840010089000B4B40200000000008000780096
:10CC94000E80E800110898000E80E80090007800EB
:10CCA400109A2000808F50001B003E000E80E80088
:10CCB40010407800614060000004E00016003A0073
:10CCC4000E80E800A00090000000280000806000B2
:10CCD4000000E00010003A000E80E8002000900000
:10CCE400700060000000E0000B003A000E80E800D5
:10CCF40090009000E05E2000808F500006003E000F
:10CD04000E80E800A0009000000820000080600071
:10CD14000000E00001003A000000FE000E80E80080
:10CD24001000780000B58800BE0890000E80E8006E
:10CD34006C00400005000900B05878006100B100A3
:10CD44006000B100CE08900000C0EB00804878007D
:10CD54000E80E80030509000E84F50000C003A007C
:10CD64000E80E800205090000004E000040032002F
:10CD74000E80E80020509000E64F500004003A0076
:10CD84000E80E800A05090004E0890000148780002
:10CD94000000EB0020B5880010002000600F980010
:10CDA4006E0890000080FA00000006000800FA00F7
:10CDB400000F7800214798002207980031CAB30079
:10CDC40020C0B3002903070091C0B30030C0B300F2
:10CDD40026030700AE009000009B20000080400066
:10CDE40020079800640047009040780060C0B300BA
:10CDF4001E030700640047009040900070C0B30019
:10CE04001A0307001E007800610020007C0207005E
:10CE1400F0822000610020007902070080C0B30086
:10CE2400670207002E4090000004E00003003A006F
:10CE34000040EB00604798000200370060C0B30078
:10CE4400604798006E4090005D0207000080FA0081
:10CE5400000006001800FA00E60307002A03070092
:10CE6400E403070016030700A1C0B300C0C1B30068
:10CE740013030700E203070023030700A6D6BF003D
:10CE8400E54F500003003200A6D6BF00E64F500025
:10CE94006F003A000000EB00100798007000470094
:10CEA400C1C1B300A40207000E5090000080FB0033
:10CEB4006A0060000000E00007003A001E009000D5
:10CEC4000000E800100798009E009000703E2000CB
:10CED400808F5000F1FF360071004700C1C1B300DC
:10CEE400950207001E509000624060000004E000BC
:10CEF40004003A009E009000703E2000808F500095
:10CF040053003600BE030700ED020700720047001D
:10CF14008040EB0088020700BC030700860207007C
:10CF24003E509000504798007400470061C0B30021
:10CF3400810207004E50900060479800750047003A
:10CF440071C0B3007C0207005E50900070479800E7
:10CF5400B3030700EE4090000040EB00C30207005B
:10CF6400FE40900010C0B300C002070068004700F4
:10CF740081002000C20107000040EB00004F780050
:10CF84002A00370076004700C1C1B3006A020700D7
:10CF94006E509000624060000004E0002600320001
:10CFA40068004700900090000000220000806000AC
:10CFB4000000E000200032008E030700D2020700C8
:10CFC4008C030700BE020700A1C0B300C0C1B300B8
:10CFD400BB0207008A030700CB0207007700470063
:10CFE400C1C1B300540207007E5090000080FB00D2
:10CFF4006A0060000000E000F8FF320080030700D0
:10D00400AF020700EE4090000040EB0097020700DB
:10D01400FE40900010C0B30094020700680047006F
:10D0240081002000960107001E4FE800F0C0B30005
:10D034009E4F1000D3FF3600CE4090000040EB001E
:10D044008A020700DE40900010C0B3008702070088
:10D054000080FA00000006000400FA00100798009F
:10D0640011B580001E0090001E0307000100360069
:10D074006F0307009E4078000040EB007B0207002E
:10D084009E40900010C0B300780207000080FA00B0
:10D09400000006000600FA0010079800640047002C
:10D0A40021C0B300240207006603070031C0B300A7
:10D0B400210207006703070020C0B3006B020700CA
:10D0C4000E80E8009040900030C0B3006702070073
:10D0D4001E0078000080FA00000006000600FA0036
:10D0E40010079800640047008040EB00120207001C
:10D0F4005403070011C0B3000F02070055030700D3
:10D104000040EB00590207000E80E80090409000B8
:10D1140010C0B300550207001E0078000080FA001A
:10D12400000006000A00FA002103070011B5800080
:10D134002E009000EB020700010036003C030700BC
:10D14400680047008040EB00FB0107000E48900098
:10D15400204798006900470011C0B300F60107009A
:10D164001E489000304798009E4078000040EB0035
:10D174003E0207009E40900010C0B3003B0207002F
:10D184003E0090000A000700000F7800AE409000B7
:10D194000040EB0035020700BE40900010C0B30011
:10D1A400320207001E0078000080FA00000006002A
:10D1B4002400FA00700F98006000B800FC02070019
:10D1C400000220000E0040008040EB00DA0107005E
:10D1D4000E60900020479800100220000E004000CE
:10D1E40011C0B300D40107001E60900030479800BE
:10D1F4002B0037007E089000101798001E10900036
:10D20400F40F50000200360040012000101798006F
:10D214001E10900040079800CE0090006A0047005E
:10D2240017010700CE0090007E0890000100500016
:10D23400700F9800680047001000780061006000DB
:10D244000000E00008003200EA0047004E009000B1
:10D25400808040000040EB00804878004E00900041
:10D264000000E800400798006A0F470009003700F3
:10D274002E019000BE0190001E007800100078007E
:10D28400B30207001E8FE8004E0090000080E90002
:10D29400400798004E0090000000E000F4FF3A00C0
:10D2A4007E0890000000E000D2FF3A00AE409000FB
:10D2B4000040EB00ED010700BE40900010C0B30039
:10D2C400EA0107002E0090006101B8003E009000C2
:10D2D4009F020700AE0090003E00900000804000D6
:10D2E400200798002E0090000080EA000080FA00D9
:10D2F400000006001800FA00881F78004007980014
:10D3040051079800620798000000EB00200798007E
:10D314000000EB00300798000000EB0010079800B5
:10D324000000EB00000F78004E009000E10F400079
:10D334000F003A0010002000100798006E0047000C
:10D3440021C0B3007C0107006E4890000080FB0000
:10D3540040079800680047000004E8006F00470099
:10D3640031C0B300740107007E489000004C78007F
:10D374005E009000E10F40000F003A001000200012
:10D38400000F7800700047008040EB006A0107003E
:10D394000E5090000080FB00500798006A00470080
:10D3A4000004E8007100470011C0B30062010700E7
:10D3B4001E509000004C78006E009000E10F500069
:10D3C40041003E001E00E00007003A0072004700E2
:10D3D4008040EB00580107008C020700560107004B
:10D3E4003E509000504798001E0090000000E0005E
:10D3F4000A003A007400470021C0B3004E01070040
:10D404004E509000604798007500470031C0B3004B
:10D41400490107005E509000704798006A00470079
:10D42400904078000040EB00900107006A0047003C
:10D434008D02070010C0B3008C010700680047008C
:10D444009040780020C0B3008801070068004700BE
:10D454008502070030C0B3008401070002003700D2
:10D464007A000700D60007006E0090000000E90073
:10D47400600798006E009000E10F4000F8FF3A004A
:10D484001E00E00006003A00CE4090000040EB0091
:10D4940076010700DE40900010C0B300730107005E
:10D4A4001E0090000000E00059003A00EE40900099
:10D4B40020C0B3006D010700FE40900030C0B300EF
:10D4C4006A010700520037001E0090000000E000CF
:10D4D4000A003200CE0090006E00900000804000F0
:10D4E40030079800EE40900020C0B3005F010700B1
:10D4F400FE40900030C0B3005C010700DE009000E5
:10D504006E009000008040000000E9006007980071
:10D5140076004700F1C1B300070107006E50900088
:10D524000042B2000004E000F9FF3A006A0047003C
:10D534009040780000C1B3004C0107006A00470026
:10D544004902070010C1B300480107006800470002
:10D554009040780040C1B3004401070068004700D0
:10D564004102070050C1B30040010700DE009000F3
:10D57400DF01070004003E00EE009000DC0107001C
:10D58400010036003B0207006C0047009040780021
:10D5940020C1B300350107006C00470032020700C8
:10D5A40030C1B3003101070001C1B300F0C1B300C1
:10D5B4004301070001C2B300F0C1B30052010700E8
:10D5C4001E00E000120032006E0090000000E8002F
:10D5D40060079800DE009000C501070004003E00CB
:10D5E400EE009000C201070001003600210207008E
:10D5F4006C004700904078000040EB001B010700DE
:10D604006C0047001802070010C0B30017010700A0
:10D614004F0478000080FA00000006000200FA00BF
:10D62400F1C1B3000E007800C30007001E4078006B
:10D634000080FB004500DE000004A2000080FB0027
:10D64400610060000080FA00000006000200FA0099
:10D65400AA01070000A02300401288000000370040
:10D6640009020700FEFF3A00BD010700FCFF32007B
:10D67400BD0107001E80FB000080FA0000000600C8
:10D684000A00FA003007980041079800CD22A9004B
:10D69400A0032000401288000000EB00000F780077
:10D6A400FD010700040032003E0090000000E90084
:10D6B4003007980000003700F3010700FEFF3A002E
:10D6C400A7010700FCFF32004012800020479800A9
:10D6D4004E009000E10F5000320036008801070030
:10D6E4000000EB00401288001E8FE80000003700A5
:10D6F400E5010700FEFF3A0099010700FCFF320034
:10D704004012800020079800E3010700080032005F
:10D71400C3010700DE4090003E00900001487800FD
:10D72400BF010700CE4090003E0090000148780001
:10D734004E0090001E005000E10F50000100360022
:10D74400E7FF3700D7010700160037000000EB00A1
:10D75400401288001E0FE800CF0107000B003200C2
:10D76400AF01070000003700C7010700FEFF3A00C1
:10D774007B010700FCFF32004012800080407800EB
:10D784003E0090000148780006003700BE01070003
:10D79400FEFF3A0072010700FCFF320040128000D5
:10D7A400204798004E0090009E0F1000E7FF3900BC
:10D7B400CD22A8001E0078000080FA0000000600B8
:10D7C4000400FA00204798004C0107002E40900006
:10D7D4008080FB0000A027000080700040128800B9
:10D7E40000003700A8010700FEFF3A005C010700B3
:10D7F400FCFF32005C0107000080FA000000060014
:10D804000800FA006A010700CD22A900A007200041
:10D8140040128800000037009B010700FEFF3A0019
:10D824004F010700FCFF3200A20107003E009000F8
:10D83400E10F5000260036006001070030010700A8
:10D844001E009000401288003E0090000080E90015
:10D85400300798003E009000E10F500008003600A9
:10D86400560107000000370087010700FEFF3A0059
:10D874003B010700FCFF32008E010700F0FF370078
:10D8840081010700FEFF3A0035010700FCFF32006A
:10D8940088010700830107000D0037002E00900067
:10D8A40010407800500107004B0107003E00900033
:10D8B4000000E900300798000000370072010700FB
:10D8C400FEFF3A0026010700FCFF32007901070041
:10D8D40071010700F1FF3A00CD22A8000080FA0090
:10D8E400000006000200FA0001C2B300E0C1B30068
:10D8F40073000700100020009824020001000000BB
:10D90400CD22A900F00F200040128800000037004B
:10D914005D010700FEFF3A0011010700FCFF320021
:10D9240012010700100020009824020001000000EA
:10D934000080FA00000006000600FA000E0107004D
:10D944000000370050010700FEFF3A000401070001
:10D95400FCFF32000D010700000037004A010700F8
:10D96400FEFF3A00FE000700FCFF32000B01070037
:10D974000080FA00000006000600FA00FE0007001E
:10D984000000370040010700FEFF3A00F4000700E2
:10D99400FCFF3200FD000700000037003A010700D9
:10D9A400FEFF3A00EE000700FCFF3200F70007001C
:10D9B4000000370034010700FEFF3A00E8000700CA
:10D9C400FCFF3200F50007000080FA0000000600AA
:10D9D4000800FA00300798002147980040212000F1
:10D9E40077000700AE40900040C1B3001F0007005D
:10D9F40011C0B30020C1B3001C000700A0302000F8
:10DA04006F00070063004700A1C0B300DAFF0700FE
:10DA14003E409000BE000700FAFF3A00402120007B
:10DA2400670007008040EB0020C1B3000F0007002F
:10DA34006400470081C1B300CFFF07000101070064
:10DA440091C1B300CCFF07005E40900010479800DE
:10DA54000000EB005A0007003E0090001E0878000A
:10DA64003E0090000080FA00000006000400FA0066
:10DA7400AA00070000C4B300AD000700000037008F
:10DA840001010700FEFF3A00B5000700FCFF320069
:10DA9400A900070000003700FB000700FEFF3A0062
:10DAA400AF000700FCFF3200020107000000000085
:10DAB40000000000CD22A8000080FA00000006004B
:10DAC4000400FA009500070000CAB300980007009C
:10DAD40000003700EC000700FEFF3A00A00007003A
:10DAE400FCFF32009400070000003700E600070046
:10DAF400FEFF3A009A000700FCFF32009B0007007B
:10DB04000080FA00000006000400FA008300070009
:10DB140000C8B3008600070000003700DA000700E1
:10DB2400FEFF3A008E000700FCFF3200820007006F
:10DB340000003700D4000700FEFF3A008800070009
:10DB4400FCFF3200890007000080FA000000060094
:10DB54000600FA00004F78001107980040212000C9
:10DB6400170007009E40780040C1B300BFFF0700C4
:10DB74000E80E8009040780060C1B300BBFF07004E
:10DB84000E80E8009040900070C1B300B7FF07001A
:10DB9400A03020000A00070064004700A1C0B300C1
:10DBA40075FF07004E40900059000700FAFF3A0045
:10DBB4000000EB00020007000080FA0000000600ED
:10DBC4000200FA00000F780031C0B300F0C1B300C6
:10DBD400BBFF07000E00780090409000F0C1B30036
:10DBE400C9FF07000080FA00000006000200FA00E6
:10DBF40041C0B300F0C1B300B1FF0700D1C1B3000D
:10DC04000E0078004CFF07001E407800644060005E
:10DC14000004E000F9FF3A000E00E800F1C1B3008F
:10DC240045FF07001E409000684060000004E000CB
:10DC3400F9FF3A0001C2B300E0C1B300B2FF07002C
:10DC44000080FA00000006000200FA0001C2B300DE
:10DC5400E0C1B3009AFF0700D1C1B3000E00780001
:10DC640035FF07001E40780029000700FAFF320044
:10DC740041C0B300F0C1B300A3FF07000080FA0065
:10DC8400000006000200FA00004F78005031200026
:10DC9400CBFF07009E40780050C1B30073FF07001C
:10DCA4000000EB00C6FF07000080FA000000060039
:10DCB4000400FA0050312000C1FF07000E80E80084
:10DCC40051C1B3001CFF07002E409000004F7800A4
:10DCD4000000EB00BAFF07001E80FB000080FA0082
:10DCE400000006000080400074004000150037006A
:10DCF400109A2000808F500000000600CD22A90059
:10DD040041E2A9004342A80041E2A8000000060045
:10DD1400614060000004E000000006002047980015
:10DD240031479800CD22A900AE40900000000600C3
:10DD340000C070002C0037005E0007003E409000D9
:10DD440029003700000F78009E007800E8FF3700B4
:10DD540001002000020040008380480014003700C6
:10DD640040C2BF00EAFF37004E0007005100070021
:10DD7400CD22A80000000600200798002147980043
:10DD8400CD22A9002E40900017003700490007005B
:10DD94000000EB004012880000000600F3FF0700BB
:10DDA4002E0090001E4878002E009000000006000F
:10DDB4002007980031079800000006002E0090000C
:10DDC4001040780030479800030007002E009000B0
:10DDD40010407800204798002E0090000000E800D2
:10DDE40020079800000006000080FB004012880015
:10DDF4000000060001C8B300F0C1B3000000060033
:10DE040081C0B300F0C1B300000006002E509000A2
:10DE1400404798007300470011C0B300000006009B
:10DE24003E0090000000E800300798000000060063
:10DE34001E007800E1652F0001004000000F78000B
:10DE4400000006004E409000004F78006500470037
:10DE5400000006005E409000104798000E80E80025
:10DE640090407800000006000000E8009040780030
:10DE7400000006006E009000E1652F0001004000E4
:10DE8400600798000000060040C2BF0062406000C6
:10DE94000004E000000006003E0090000000E000E6
:10DEA4000000060041E2A9004342A90041E2A800A3
:10DEB4000000060040128000004F780000000600B9
:10DEC4000400FA0070040700090037007104070019
:10DED400008F40009E0078000000EB009000980046
:10DEE4009E00780000C0EB00805098006E0407008C
:10DEF4001E009000E20F5000F4FF36000080FA008C
:10DF0400000006000E00FA00200798003107980070
:10DF140042079800C0562100100798002E00900078
:10DF2400E20F500003003200E00F20005007980079
:10DF3400430037004E0090000000E00010003A005B
:10DF4400BE0090006107980040062000EE0090009B
:10DF5400808F500008003200E0062000EE009000A0
:10DF6400808F5000010032000500370010012000AE
:10DF74004007980002003700600020004007980026
:10DF84000040EB00004F7800280037001E0090008E
:10DF9400100090000000E00020003A001E009000F5
:10DFA400BE00900001087800BE009000E00620004A
:10DFB400808F500009003A004E009000F10F50008D
:10DFC40006003A009E009000100020009000980087
:10DFD4001E80FB005007980019003700BE00900017
:10DFE40040062000808F500009003A004E00900047
:10DFF400E60F500006003A009E009000100020003A
:10E00400900098009E80FB00510798000C00370098
:10E01400E00F200050079800090037001E4FE80069
:10E024001E009000720040001007980021C0B30049
:10E034009ECF1000D5FF3600E00F20005007980057
:10E044005E0090000080FA00000006000E00FA0056
:10E054006047980041079800520798006E4090006E
:10E06400E24F500002003600130407002C00370072
:10E07400A6030700E10F5000030032008080EB008C
:10E0840061079800260037005E009000EF0F5000F3
:10E0940002003E000804070021003700CE00900073
:10E0A400110798009E009000060407001E00E0007F
:10E0B40004003A0006040700020036000040200075
:10E0C40000B788000A0407000E003A000002EB00C3
:10E0D4009E0178000041EB006000B80048C60200D1
:10E0E40000000000804078002E009000015098004D
:10E0F4005E040700E14F400002003A00EE0307000F
:10E10400070037002E0090009E0078002100980040
:10E11400AE00900020002000FA030700600798007A
:10E124006E0090000080FA00000006000E00FA0065
:10E13400004F9800510798000E489000E24F50009D
:10E1440002003600DC030700610037000E4890002F
:10E1540049040700300798003E009000EC030700D4
:10E16400030032008080EB006107980058003700FC
:10E174003E009000EA03070003003A003E009000CE
:10E18400E0009000510798003E009000E70307006C
:10E19400470032003E009000E103070044003200D3
:10E1A400C50307004A0037000040EB00004F780029
:10E1B400B503070037003700DF0307000000E00065
:10E1C40033003A003E00900020009000A4C0B30049
:10E1D400800178000041EB006000B8006A3602005C
:10E1E40000000000404798004E409000E24F40007D
:10E1F40003003A008080EB00610798003400370088
:10E204004E409000763702000000000010C0B300BA
:10E21400004F7800BE00900030002000900098006D
:10E224003E009000DE009000610098004203070069
:10E23400CE40900001487800C3030700400020004E
:10E24400800878001E0090007200B900EE004000C3
:10E25400C056210080804000100020008008780013
:10E264009E0090003E009000200190007208B900CA
:10E27400E400400032030700020878008503070029
:10E2840080804000400620008008780004003700A9
:10E29400850307001E009000E20F5000C6FF360001
:10E2A4001E04E00002003A00830307000800370060
:10E2B4005E0090000000E900500798005E009000A6
:10E2C400E10F4000B8FF3A008000EB0061079800BE
:10E2D4006E0090000080FA00000006001200FA00B0
:10E2E400204F980061079800720798002E4890000C
:10E2F400E24F500002003600960307005A00370030
:10E304002E489000DC030700400798004E00900060
:10E3140083030700020032008E0307005200370017
:10E324004E0090007A0307000200320089030700C0
:10E334004D00370054030700470037007E030700F1
:10E34400E40F500043003A001E009000FF02070053
:10E354004E00900020009000808F50003D003A0055
:10E36400F5020700104F78001E407800763702004F
:10E37400000000001E4078009A37020000000000F0
:10E384000000E000330032001E40780066380200CE
:10E3940000000000300798006E0090000000E000CC
:10E3A400170032007E0090000000E00014003200EC
:10E3B4007E00900010007800EF0F500002003E0035
:10E3C40064030700280037006E00900020079800BF
:10E3D4003E0090001001BE00AE00900060030700F4
:10E3E400F04098003E009000D0019000AE009000F4
:10E3F40071030700FE0090000001200080087800EF
:10E404009E0090003E009000500190007208B900F8
:10E41400E6004000CA020700020878009E0090004F
:10E424003E0090001001BE007208B900E8004000F0
:10E43400C30207000288BE004303070060002000F7
:10E44400800878001E0090000080FB00000F9800F8
:10E4540005003700140307001E009000E20F50006F
:10E46400B6FF36003B0307000E0890000080FA0058
:10E47400000006001600FA00404F9800710798004B
:10E48400020F98004E489000E24F500003003600FF
:10E494000080EB00200F9800950037004E48900054
:10E4A40075030700500798005E009000100090006C
:10E4B4000000E00003003A008080EB00210F980088
:10E4C4008B0037000E089000EF0F500003003E0051
:10E4D4000081EB00220F980085003700FE019000B8
:10E4E40043079800CE0090003F03070010079800F0
:10E4F400CE0090009A020700220798003307980084
:10E504002E009000BE009000E00F5000E08F5800F5
:10E51400030032001E0090000000E00003003A00F7
:10E524000080EB00200F9800710037005E0090001F
:10E53400F702070047003A005E00900010009000C8
:10E54400100F98009E089000E58F50000F003200D5
:10E554001E099000E50F510005003E009E09900041
:10E564000300E900E10F500037003E001C003700B3
:10E574001E089000E60F5000010032003200370000
:10E584008000EB00210F9800590037004E4890009E
:10E59400260207000000E000030032000081EB00C7
:10E5A400220F9800520037005E0090000050900047
:10E5B4009A370200000000000000E00003003A0067
:10E5C400E3FF2F00230F980049003700DE0090007E
:10E5D40060002000CB020700200F980044003700A1
:10E5E400B4C0B3009E01900032C0B3002E0090006E
:10E5F400BE0090006A3602000000000067020700B7
:10E60400E24F400003003A008080EB00210F9800A5
:10E61400370037005E00900000509000763702000B
:10E6240000000000DE0090000000EB00F000980005
:10E63400DE0090005000200090009800E2FF2F00C0
:10E64400220F98002A0037008081EB00230F9800E6
:10E65400270037005E00900010009000E10F50008A
:10E6640013003A009A02070002003600004020001E
:10E6740000B788001E0290009E0178000041EB0064
:10E684006000B80048C60200000000004302070012
:10E69400E14F400003003A000080EB00200F980097
:10E6A40013003700DE009000200020009000980046
:10E6B4005E0090009D020700030032008080EB00A2
:10E6C400210F98000A0037005E0090001E019000A0
:10E6D400320098005E0090002E019000BE01900070
:10E6E40042009800530098008001EB00230F98002B
:10E6F4002E0890000080FA00000006000800FA00CE
:10E70400004F7800110798002207980033079800FB
:10E714008002EB000002EB00BE0190002E0190008D
:10E724009E0090001E407800020007000080FA005E
:10E73400000006002E00FA000067980011179800E8
:10E74400221798003317980044179800551798001B
:10E754000080EB00100798000E609000E24F50001C
:10E7640002003600130207009B0037000E60900081
:10E77400E70107000000E00003003A008080EB009E
:10E784006117980094003700590207006F003A009F
:10E794002E009000D00090004000900066014700D9
:10E7A4000089BE002E009000B0009000010F780098
:10E7B4004E1090000000E0001D0032005E1090003A
:10E7C400F00F500002003200FA0107008200370007
:10E7D400CE1090003B020700CE109000E00107002D
:10E7E400660047000288BE002E00900010009000D2
:10E7F400E10F50000E003A0070004700000178005D
:10E80400EF01070064014100ED010700F00047003B
:10E81400020120000E6090000CFE0700E10F400092
:10E8240003003A008080EB00611798006A0037000B
:10E83400660147001200780092009000E00F50003B
:10E84400E08F580004003A00660147000080EB00A6
:10E854008080EB000089BE00DF0107001002BE00CB
:10E86400660147001200780092009000800F520069
:10E87400818F5A002400320066004700E400400003
:10E8840066004700EEFB0200000000000000E0000C
:10E89400080032005B0207008080400066004700E9
:10E8A40009000900B0587800A100B100A000B1002F
:10E8B40015003700EE200200010000000001BE0038
:10E8C40040AB800051AB80000001510081815900B0
:10E8D400A025260021002000800F5100818F5900BF
:10E8E4000700360066004700A0FB0200000000009D
:10E8F400EE2002000100000040AB880051AB88000C
:10E90400AC0107003400370058020700DEC80200DB
:10E91400000000000000E0002E003200B1010700FA
:10E924001E087800AE1090001E1090003EC9020030
:10E93400000000001007980086C9020000000000D3
:10E944009E00900061179800230037002E0090006D
:10E95400EF0107001F003A002E0090001000900005
:10E96400E60F500002003200920107001A0037003F
:10E974000E6090002D0107000000E000030032004B
:10E984008080EB0061179800130037002E10900070
:10E994000000E00003003A000000EB00601798005C
:10E9A4000D0037002E1190009E1090002F020700DA
:10E9B4006C39020000000000100798001E0090004F
:10E9C4000000E000030032009E00900061179800F0
:10E9D40001003700770107006E1090000080FA00F4
:10E9E400000006000C00FA00204798002107980058
:10E9F40032079800430798007F01070002003600A1
:10EA0400800107002E0037002E409000800107008F
:10EA1400BF01070013003A001E00780010009000A8
:10EA2400E60F500002003200760107002400370090
:10EA34002E409000FD0007000000E00002003200BC
:10EA4400700107001E0037003E019000AE009000E8
:10EA540073010700023B0200000000005007980009
:10EA6400170037001E00780090007800E0062000B0
:10EA7400808F500010003A001E007800AB010700A0
:10EA8400020032005F0107000D0037006401070037
:10EA9400DCC90200000000000000E00006003200B3
:10EAA400BE0090002E00900038CA02000000000052
:10EAB40050079800020037000000EB005007980050
:10EAC4005E0090000080FA00000006001400FA00C6
:10EAD4006047980041079800520798006307980020
:10EAE40074079800050F98006E409000DC01070041
:10EAF4007E009000100798007D01070023003A0073
:10EB04002E00900089010700030032000000EB0092
:10EB1400100F980036003700D4010700DCC902004A
:10EB2400000000000000E000150032007E009000AC
:10EB34000000E0000C0032000E0890000000E0002D
:10EB4400090032000E08900010007800EF0F50000A
:10EB540005003600200107003401070021010700E9
:10EB64009001780036010700DE0090004E0090000E
:10EB740038CA020000000000100F98001C00370083
:10EB84000000EB00100F9800190037007E00900081
:10EB94000000E000100032000E0890000000E000C9
:10EBA4000D0032000E08900010007800EF0F5000A6
:10EBB40009003600AD0107006638020000000000BD
:10EBC400000F78001E007800180107001E0078006E
:10EBD400D00190001A0107008001EB005E01900053
:10EBE400CE0090006E4090007EFF0700100F98004A
:10EBF4001E0890000080FA00000006000C00FA00D5
:10EC04003007980041079800000120002007980071
:10EC14001D0107000B0037001E009000FC0040009F
:10EC24002080200000804000104F780000C2B30014
:10EC34009E4F1000070032001E04E0000500320061
:10EC4400190107009E0090002E009000808F500054
:10EC5400F1FF39001E009000200798002E0090005C
:10EC64008000E8004E009000808F500002003400C5
:10EC7400E40007000C0037003E009000E181200012
:10EC84002E019000280D020000000000AE0090004C
:10EC94003E009000808040000040EB0080487800F7
:10ECA4000000EB00500798005E0090000080FA001E
:10ECB400000006000800FA00404798004E4090000B
:10ECC400E24F5000030036000080EB00300798004C
:10ECD400530037004E409000CD0007001000900014
:10ECE4000000E00003003A000000EB003007980049
:10ECF4004B0037001E007800050107003E003A0073
:10ED04001E0078000601070016003A000040EB00E0
:10ED140020479800100037003E010700E40F500020
:10ED24000C003A00CC0007000A003A002E40900084
:10ED34000080FB007A00070010407800523802007F
:10ED44000000000037010700808040000000EB0055
:10ED540080087800C5000700A7000700EEFF360012
:10ED64002B0037001E007800ED0007002800360055
:10ED74001E007800700090000000E00016003200D1
:10ED84000040EB00204798000D003700BB0007004F
:10ED94000A003A00B000070008003A00A00007008B
:10EDA400BC370200000000009E00780040002000F4
:10EDB400D40007003007980019003700AB000700A3
:10EDC4008D000700F1FF360095000700523802005D
:10EDD400000000000E0037001E00780010009000B4
:10EDE400E70F50000A0032008D000700523802007D
:10EDF40000000000060037001E007800CB0007006A
:10EE040003003A008600070092C8020000000000D8
:10EE14009E0078000000EB00BA000700300798005D
:10EE24003E0090000080FA00000006000A00FA008C
:10EE34006047980035000700E70F500003003A00D0
:10EE440010002000400798002D003700070107003C
:10EE54007637020000000000000F78002E009000BA
:10EE6400700090000000E000180032000040EB0049
:10EE740020479800130037008000070010003A0074
:10EE84002A0007002E00900020009000808F500080
:10EE94000B003A001E00E00003003A000000EB0003
:10EEA4004007980016003700AE0090004000200094
:10EEB40090009800100020004007980010003700D0
:10EEC4006A0007004C000700EBFF36001E00E0005C
:10EED40009003200E500070052380200000000007B
:10EEE400AE009000700020009000980010002000F8
:10EEF40040079800020037000000EB00400798002C
:10EF04004E0090000080FA00000006006E40900061
:10EF1400D30007002E0090001000900000000600AF
:10EF24007200B900F0004000050037002E40900048
:10EF34000080FB00050037001E009000F8FF37003A
:10EF4400C056210000804000000006007200B90095
:10EF5400E4004000FAFF070090007800000006007B
:10EF6400414090000082FB00514090000080FB0073
:10EF74004800DD000400700000017800614090004A
:10EF84000082FB00714090000080FB004800DD001F
:10EF940004007000800178000000060080407800C2
:10EFA4005E009000015098005E00900000509000B8
:10EFB400000006000080EB006017980000000600C7
:10EFC4006000B8000089BE00640141006000B80020
:10EFD4000089BE00000006008A000700008040008F
:10EFE400000006009A000700EA00400020502100BB
:10EFF40000804000000006002E409000E24F5000C8
:10F00400000006000080EB00500798000000060096
:10F014009C000700008F40001E00780000000600DE
:10F024001E00780000509000000006001001BE0091
:10F034009E0090004A000700F0409800000006007F
:10F044009E0090005C0007008E08900000012000E4
:10F054008008780000000600B4FF07001E00780056
:10F0640020009000808F5000000006002E40900089
:10F074000040E800204798000000060065000700F3
:10F08400E30F5000000006000000EB00100798009A
:10F09400000006001E0090007200B9008000780095
:10F0A400C0562100000006001E0090000000E80089
:10F0B40010079800000006000080EB00600798002D
:10F0C4000000060048000700000F7800000006005A
:10F0D40000B78000000F78000000E80000B7880047
:10F0E40001B7800080382100808F500000000600A6
:10F0F4002E00900090007800E0062000808F5000E1
:10F1040000000600900098000000EB0000000600DC
:10F114009000780040062000808F50000000060018
:10F1240010009000E30F5000000006001000900053
:10F13400E20F50000000060040000700008040007D
:10F1440010007800000006003C00070080804000AA
:10F1540000000600E00F2000000F980000000600E9
:10F16400F00F200000026100414090006040600008
:10F1740004407000C04098004812DE0051409000E6
:10F184006040600004407000D0409800F00F200000
:10F1940000826100614090006040600004407000A3
:10F1A400E04098004819DE00714090006040600023
:10F1B4000240700000000600F00F20000081610092
:10F1C400214090006040600002407000A040980020
:10F1D4004819DE0031409000604060000240700039
:10F1E400B040980000000600214090000081FB0020
:10F1F400314090000080FB004800DD0002007000F8
:10F204000000060012000700800078002050210052
:10F214000000060003000700008040001000780092
:10F22400000006002E4090000080FB007200B90030
:10F234008080E800C0562100000006001E009000F7
:10F244007200B9008080E800C0562100000006006A
:10F25400060007000080FB007800B90000000600EB
:10F264000500070020079800000006002E0090000B
:10F2740000509000000006000200070000804000DB
:10F28400000006000080FB007200B90080007800D6
:10F29400C0562100000006000600FA00505021006C
:10F2A4000100200010079800210798000000EB00DF
:10F2B400000F7800150037001E009000AE0090008B
:10F2C4004509DD00CB01DE00830171004501DD004D
:10F2D4001E009000AE0090000201400083814800AF
:10F2E4009E00780000382100008040001040780023
:10F2F4000080FB00010020000200400083804800E1
:10F3040010079800210798001E0FE8009E0078005F
:10F3140060032000808F5000E7FF36001E0090003D
:10F32400AE0090000080FA00000006000800FA0019
:10F33400889FBE00000F78001107980022079800EC
:10F344000D03070010C0B300E0000700BBD3BF00EB
:10F354008080FB00BCD3BF00B80307000004780022
:10F36400BDD3BF008080FB00BED3BF00B303070042
:10F3740080047800C8FF0700800F5400818F5C0070
:10F38400030032001000200030079800CB00370043
:10F39400A1030700EB0F500003003200110020000E
:10F3A40031079800C50037001E0178007100410044
:10F3B4006338210010000900335878001001B100AF
:10F3C400A10220001E804000A1392100160407007C
:10F3D40091392100180407004170980009D4BF0036
:10F3E40061406000804078001E00780021C89800C9
:10F3F4009E00780010C0B300E0C09800513821008E
:10F404000D040700015098000AD4BF006140600059
:10F414001E01780061406000C201DD00F2489000E6
:10F42400B0CFB30000C06000034070007049980082
:10F4340097D3BF008080FB0098D3BF007F030700F1
:10F44400804078001E00780021609800FD030700CA
:10F454004200DE007403070000014000C310900066
:10F46400D0FF2F00FA030700C0119800F13D2100DE
:10F47400F1030700614898001E007800720307003A
:10F484001E00780052009800630098001E00780067
:10F49400E0009000500090001E01780010019800D8
:10F4A400210198001E007800A00090001000900038
:10F4B4001E0178003001980041019800413D21006F
:10F4C400DD030700617898001E007800E30307005D
:10F4D400800078001E00780061189800F13B21003C
:10F4E400D5030700217898001E007800E503070083
:10F4F4001E0078003218980043189800D1030700C2
:10F504000000D100614060001E0178000080FB0013
:10F51400E1016000C2109000E0FF2F000080600055
:10F524000300700040119800C60307004600DE0087
:10F534003D0307004201DD00C3109000B0FF2F001F
:10F54400C3030700C01198001E0090006E00400025
:10F55400A33A210010000900335878001001B100CB
:10F56400413A2100914078001E00900071589800A3
:10F57400B40307004700DE001E01900061406000F4
:10F58400C201DD00D2489000B0CFB30000C06000DB
:10F594000340700050499800A5D3BF008080FB0051
:10F5A4001E00900001109800A60307004300DE002F
:10F5B400B803070000014000B3109000D0FF2F00F3
:10F5C400A3030700B0119800413F21009140780047
:10F5D4001E009000414898001E009000B0030700F0
:10F5E4001E00900042009800530098001E009000F6
:10F5F400D0009000400090001E0190000089BE00E1
:10F604001E0090001000BE001E0190002001980012
:10F61400310198008B0307004400DE009D030700BE
:10F624004201DD00B3109000B0FF2F0088030700F3
:10F63400B0119800830307004500DE0061406000BC
:10F644001E0190000080FB00E1016000B2109000F8
:10F65400E0FF2F000080600003007000301198006C
:10F66400A6D3BF008080FB00A7D3BF00F30207002E
:10F6740000017800A8D3BF008080FB00A9D3BF009D
:10F68400EE020700800178000200BE001E01900017
:10F694001011980021119800213821009140780020
:10F6A4001E0090002178980084D3BF008040780029
:10F6B4002E00900001487800440307003E009000AB
:10F6C4004F04BE000080FA00000006000200FA00A9
:10F6D400004F7800B2C8B300013821001E40780002
:10F6E400460207000080FA00000006000000FA004D
:10F6F400513F210075030700F5F3B700613F210076
:10F7040072030700F6F3B700713F21006F0307008F
:10F71400F7F3B700813F21006C030700F8F3B7004B
:10F72400913F210069030700F9F3B700A13F2100CD
:10F7340066030700FAF3B700B13F21006303070033
:10F74400FBF3B700C13F210060030700FCF3B700DF
:10F75400D13F21005D030700FDF3B700E13F210025
:10F764005A030700FEF3B700F13F210057030700D7
:10F77400FFF3B700014021005403070000F4B70071
:10F78400114021005103070001F4B700214021007A
:10F794004E03070002F4B700314021004B03070079
:10F7A40003F4B700414021004803070004F4B70004
:10F7B400514021004503070005F4B70061402100D2
:10F7C4004203070006F4B700714021003F0307001D
:10F7D40007F4B700814021003C03070008F4B70098
:10F7E4003E0307000082FB00D80207001001BE00A0
:10F7F4004220DD003C03070038030700F4F3B700A0
:10F80400D20207006E004000A13A21001000090056
:10F81400B05878001001B100CC0207007058900075
:10F82400A4F3B700C902070000109000A5F3B700C5
:10F834003E0307000000D1003F0307004301DD0041
:10F844004003070070CFB300870207003010900018
:10F854004200DE00380307004401DD0039030700DD
:10F86400F0CEB30080020700A010900010109000AA
:10F874000001BE0036030700A6D3BF00370307000C
:10F88400A6F3B700C810DE00A7D3BF0033030700F8
:10F89400A7F3B700F00F200080806100A8D3BF0059
:10F8A4002E030700A8F3B700C818DE00A9D3BF00D1
:10F8B4002A030700A9F3B7001C0307001E0307006F
:10F8C4004501DD001F030700F0CDB3006602070009
:10F8D400504890000080FB004200DE006140600060
:10F8E400C700DD0009D4BF000074A100014070000E
:10F8F40009F4B7000080FA00000006000000FA00D6
:10F90400013E2100F1020700E0F3B700113E21009F
:10F91400EE020700E1F3B700213E2100EB020700ED
:10F92400E2F3B700313E2100E8020700E3F3B70039
:10F93400413E2100E5020700E4F3B700513E2100F7
:10F94400E2020700E5F3B700613E2100DF02070091
:10F95400E6F3B700713E2100DC020700E7F3B700CD
:10F96400813E2100D9020700E8F3B700913E21004F
:10F97400D6020700E9F3B700A13E2100D302070035
:10F98400EAF3B700B13E2100D0020700EBF3B70061
:10F99400C13E2100CD020700ECF3B700D13E2100A7
:10F9A400CA020700EDF3B700E13E2100C7020700D9
:10F9B400EEF3B700F13E2100C4020700EFF3B700F5
:10F9C400013F2100C1020700F0F3B700113F2100FD
:10F9D400BE020700F1F3B700213F2100BB0207007C
:10F9E400F2F3B700313F2100B8020700F3F3B70088
:10F9F400DD0207000082FB0077020700100190007F
:10FA0400A00190004220DD000106200076020700DC
:10FA1400D5020700DFF3B7006F02070020789000DB
:10FA2400BFF3B7006C02070060789000D4F3B7000E
:10FA34006902070020C890006140600061416000D5
:10FA4400C0020700E0CFB300490207007100400084
:10FA54006138210010000900B05878001001B1008D
:10FA64005D020700A002B00080007800A0392100E8
:10FA74006D020700580207004070900099F3B70028
:10FA8400550207000050900085F3B70052020700AA
:10FA9400206090000081FB00AD02070097D3BF00F7
:10FAA400AE02070097F3B700C810DE0098D3BF007A
:10FAB400AA02070098F3B70047020700401090001D
:10FAC4000000D1009C0207004201DD009D020700F6
:10FAD400B0CFB3002A02070097020700004140009C
:10FAE40098020700D0CFB300250207004200DE00D1
:10FAF400910207004601DD0092020700F0CBB3003B
:10FB04001B020700704890000080FB004200DE00EA
:10FB14006140600061416000A14021009140780093
:10FB2400E0CFB30000C06000024070000AF4B700E8
:10FB34000080FA00000006000000FA0021E82F000F
:10FB440066005700010040001040780084F3B700BD
:10FB54000080FA00000006000000FA0080D3BF0015
:10FB640060406000B040B30080F3B70081D3BF00B1
:10FB74006040600081F3B700C7FD07000001BE00CC
:10FB840073020700BBD3BF0074020700BBF3B700C6
:10FB9400C810DE00BCD3BF0070020700BCF3B7007E
:10FBA400F00F200080806100BDD3BF006B0207000E
:10FBB400BDF3B700C818DE00BED3BF00670207005C
:10FBC400BEF3B700020007000080FA000000060040
:10FBD4000000FA00B2C8B3000138210010C0B3001D
:10FBE400480107000080FA00000006001000FA0037
:10FBF400700798007E00900020789000E3010700D1
:10FC0400003C2100E40107007E0090002078900071
:10FC14008080FB007E00900030199000C019900095
:10FC24004208DD00010420009301070003003700AF
:10FC340093010700220107009D0107003E00900088
:10FC4400E30F5000FAFF34009D0107000A0107008A
:10FC54009E01070008010700A00107000601070034
:10FC6400A201070004010700304F98004E039000E2
:10FC7400DE0390007E00900002020700820F530012
:10FC8400838F5B00060032007E0090002078900095
:10FC94008040E8007E00900021789800D5FF37006E
:10FCA4007E009000607890000080FB00000040001F
:10FCB40080007800503D210000804000200798001B
:10FCC400AE0090001E009000008F50007E00900057
:10FCD400607890008080FB007E009000E019900026
:10FCE40001804000B4010700F00F20000081610092
:10FCF40011409000B2010700904098004819DE00BE
:10FD040021409000AE010700A0409800AF01070019
:10FD1400030037005A010700E900070064010700E7
:10FD24003E009000E10F5000FAFF34006401070028
:10FD3400D1000700404F98001E00780000C0E80082
:10FD4400CD000700504F9800EE0190007E00900017
:10FD5400C2010700808F5100060032007E0090002F
:10FD6400607890008040E8007E0090006178980000
:10FD7400CBFF37000080FA00000006000E00FA00F6
:10FD8400600798006E009000604890007F010700B3
:10FD9400003E210059010700604890008080FB006C
:10FDA4006E00900010019000A00190004208DD0058
:10FDB400010620003001070003003700300107006E
:10FDC400BF0007003A0107003E009000E30F500017
:10FDD400FAFF34006E009000A00090001000900024
:10FDE4006E019000500198006101980034010700F1
:10FDF400A1000700350107009F0007003701070035
:10FE04009D000700390107009B0007003E01070021
:10FE14000D010700820F5300838F5B00070032003F
:10FE24006E009000604890008040E8006E009000F2
:10FE3400614898006E009000D0FF07000080FA002F
:10FE4400000006000E00FA00600798006E009000A3
:10FE5400404890004D010700503F21002701070052
:10FE6400404890008080FB006E0090001001BE00AE
:10FE74004208DD009C01070054010700030037001D
:10FE8400FF0007008E000700090107003E009000F4
:10FE9400E30F5000FAFF34006E0090001000BE0023
:10FEA4006E01900040019800510198000401070080
:10FEB40071000700050107006F0007000701070034
:10FEC4006D000700090107006B0007000E01070021
:10FED40073010700820F5300838F5B000700320019
:10FEE4006E009000404890008040E8006E00900052
:10FEF400414898006E009000D2FF07000080FA008D
:10FF0400000006000400FA002047980020002000AA
:10FF1400000F78002E40900082F3B7009E00780016
:10FF2400003821000080400090407800E400070081
:10FF34006300070008FF07000080FA0000000600C5
:10FF44000000FA00B40007000001E8008001070087
:10FF540080D3BF008101070080F3B700C810DE0022
:10FF640081D3BF007D01070081F3B70018FF0700AC
:10FF74000080FA00000006000000FA00C482A80015
:10FF840020122000101388000000280000138800AD
:10FF94000080FA00000006000200FA00004F78001A
:10FFA4001E80FB004013880060C2BF0061406000F7
:10FFB4000004E000FCFF3200401380000080FB00DE
:10FFC4000080FA00000006000200FA00C482A900C2
:10FFD40050C0B300F0FF07000040EB00EEFF070045
:10FFE4000080FB00000F7800C482A8001E00780087
:10FFF4000080FB000080FA00000006000800FA0000
:020000040001F9
:10000400881F7800204798002107980062479800CD
:10001400EDFF0700C1000700FDFF3A00C482A900FC
:1000240030C0B300DCFF07002E409000DAFF070069
:100034000040EB00004F7800080037001E80FB00F2
:10004400800078002E009000008440000040EB0007
:10005400D1FF0700004C78001E4FE8006E4090006E
:100064009E4F1000F5FF3900C482A8004F047800A9
:100074000080FA00000006000400FA0020479800FF
:10008400D1FF0700A5000700FDFF3A00C482A900C4
:1000940030C0B300C0FF07002E409000BEFF070031
:1000A4000040EB00BCFF0700004F7800C482A800AA
:1000B4001E4078000080FB000080FA00000006006B
:1000C4000200FA00004F780011479800BEFF0700B5
:1000D40092000700FDFF3A003F000700C482A90018
:1000E40020C0B300ACFF07001E407800AAFF070041
:1000F4001E409000A8FF0700C482A8000080FA00F8
:10010400000006000800FA00204798002107980024
:1001140062479800ACFF070080000700FDFF3A002B
:100124002D000700C482A90020C0B3009AFF070075
:100134002E40900098FF07000040EB00004F78002D
:100144001B0037002E009000904078002E00900095
:100154000000E80020079800014078008EFF0700A7
:100164002E4090000040E800204798002E40900068
:100174000080FB006F0060000000E0000B003A000C
:10018400C482A80090FF0700290007000004E000D3
:10019400FCFF3A0010000700C482A90020C0B3008D
:1001A4007DFF07002E4090007BFF07001E4FE800F4
:1001B4006E4090009E4F1000E2FF3900C482A800F8
:1001C40081FF07001A0007000004E000FCFF3A006A
:1001D4000080FA00000006000000FA00C482A900B2
:1001E40060C0B3006CFF0700C482A8000080FA005E
:1001F400000006000200FA00000F7800D002200080
:100204009E00400062C0B300A0CFB3007BFF070094
:100214000080FA000000060080D3BF008080FB004D
:1002240081D3BF0005003700614060009E01780063
:100234000080FB006100600000000600E30007008E
:10024400010070000000060060489000CE00070026
:100254000106200035003700DC00070004007000B0
:10026400800178000000060000C0600002407000B9
:1002740009F4B700350037005B000700530037006E
:100284003E0090009E0040000038210000804000A5
:10029400104178001E007800804078003E009000F5
:1002A40000C040000040E8008240780000000600E2
:1002B4003E0090000000E8003007980000000600AF
:1002C4001E0078000040E80000000600004F98007F
:1002D4001E00780000C0E80000000600104F9800DF
:1002E4001E0078006340400000000600204F980084
:1002F4001E0078006440400000000600260007004D
:100304006E00900000000600304F98004E039000ED
:10031400DE0390006E009000000006000080FB00E9
:10032400630060000000E000000006000C0007000D
:100334001182FB00114090009600070021409000BC
:100344000082FB0031409000C3FF3700A1FB2F0067
:10035400660057000100400000000600410720002D
:1003640080804000003821008080400000000600AA
:1003740000C060000240700009F4B70016003700A6
:10038400FBFF070040109000000006007E000700FD
:1003940080007800000006000080400020079800DC
:1003A4000038210010079800AE0090001E00900055
:1003B400008F50000000060041052000E8FF3700D0
:1003C4006040600002407000000006000000EB0086
:1003D400300798000000060001F52F006600570062
:1003E4000100400000000600DDFF0700F00F2000C0
:1003F4000000610011427800E048620091487000FA
:100404004812DE0067000700F00F20000082610040
:10041400690007004819DE0031409000E8FF07003A
:10042400B040980000000600520007005100070089
:100434001108780000000600914078001E00780042
:100444000000060009D4BF000080FB000000060085
:1004540000806000020070000000060060789000D8
:100464000080FB0000004000D3FF07001140900013
:100474000081FB002140900054000700020070003E
:1004840000000600207890003F00070001042000CF
:10049400A6FF3700614060009E01900064FF3700B2
:1004A4004048900038000700ACFF0700114090005E
:1004B4000082FB002140900036000700314090008C
:1004C4000082FB004140900063FF370091407800B8
:1004D40000C0EB0000C07000000006009BFF070096
:1004E40040489000000006009CFF0700F00F200029
:1004F400000261002B0007004812DE002E000700F6
:10050400F00F2000008261003140900060406000E4
:1005140004407000B04098004819DE00414090004B
:10052400A7FF0700C04098000000060087FF0700EF
:1005340030109000000006006140600061406000DF
:100544000000060091402100914078000000060060
:10055400F00F200080006100000006006040600091
:1005640001407000000006009BFF070060489000F7
:10057400000006001101BE000288BE0064004000B5
:10058400E4804000000006000080FB004200DD0023
:10059400000006000D000700040070000001780050
:1005A40000000600114090006040600004407000AC
:1005B40090409800000006002140900060406000D8
:1005C40004407000A0409800000006000080FB007A
:1005D4004800DD00000006000200FA00000F780069
:1005E400A2040700C0D098001E017800C2E0900069
:1005F400E0CFB30000C0600040E198009E007800A6
:100604000000EB00903098001E0178006000B800F4
:1006140010019800210198001E0178006000B800C4
:1006240030019800410198001E017800F2489000C2
:10063400E0CFB30090040700D0CFB3008E040700CE
:10064400B0CFB3008C040700F0CDB30000C060004D
:10065400704998009E00780010C0B300E0C0980074
:10066400610620001E804000BC0002000100000062
:100674000080FA00000006000200FA00000F780073
:100684009E00780060C4B300905098009E007800EB
:10069400F0C6B300A05098009E00780030C6B300A6
:1006A400B05098009E00780050C7B300C050980026
:1006B4009E00780030C7B300D05098009E007800A8
:1006C40050C6B300E05098009E00780020C7B300E5
:1006D400F0509800650407008058980063040700F0
:1006E4009058980061040700A05898005F04070020
:1006F400B05898005D040700C05898005B040700D8
:10070400D058980059040700E05898001E0178005A
:10071400C2109000E0FF2F0000806000401198009C
:100724005A0407005001980061019800570407001B
:10073400100198002101980054040700300198002A
:10074400410198009E00780010C4B30080509800C6
:1007540046040700A078980044040700E078980055
:1007640042040700A0C898004B040700D01098006A
:1007740049040700E010980047040700F0109800AF
:100784004504070080189800430407009018980057
:100794009E00780010C4B300C07098009E007800DA
:1007A40080C2B300A06098001E017800C2109000BF
:1007B400D0FF2F0000806000401198009E00780058
:1007C400411090000020A000C01098000080FA00A2
:1007D400000006000400FA00000F78006106200003
:1007E4001E8040005A01020001000000E0B68000B3
:1007F40080007800110798000000E800E0B6880047
:100804001E009000E10F50000B0032009E0090008B
:10081400E18F5000050039001E009000E20F5000E7
:10082400080032000000EB00E0B688001E007800EB
:100834000C000700060037001E0078009300070034
:10084400030037001E007800601102000100000060
:100854001E0078007ED30200000000000080FA0031
:10086400000006000E00FA00881F78004007980078
:100874004E00900030309000E20F5000060032002D
:1008840007040700A4030700CE0090000000EB005B
:10089400B08898007A0037004E00900040309000F5
:1008A400E10F500074003A004E0090003088900030
:1008B400EE0F500026003C004E0090004092900045
:1008C400D09290004E00900020919000B091900042
:1008D4000400BE0016070200000000000000E00053
:1008E40001003A00660037004E009000D09090005E
:1008F400409090004E019000209198003191980012
:100904004E009000308C90004E009000D0909000EB
:100914004090900002002400C36124001A070200E2
:1009240000000000820702000000000000017800BF
:10093400CE009000080044008007B00002B07800A8
:100944008800E8004E009000318898004C00370081
:100954006000B80020079800310798000000EB0001
:10096400100798001E0037001E009000CE00900073
:10097400000040008007B000608478006140B90046
:10098400C0060200000000005007980061079800AC
:100994000800E00008003D00020020000378240065
:1009A4005E009000EE00900082050200000000004E
:1009B40050079800610798005E019000EE019000D6
:1009C400BC03070082050200000000002007980015
:1009D400310798001E0090000000E80010079800FE
:1009E4001E009000EE0F5000DFFF340002002000D4
:1009F40003172400AF0307003C06020000000000B8
:100A04002007980031079800CE0090000000EB000A
:100A1400B0889800A7030700B80702000000000090
:100A24004200DD00000F78001E007800A2002000C4
:100A3400110009000280D800000F7800E092200025
:100A44009E0050004E009000518898004E00900087
:100A540050889000800078004E00900001087800D3
:100A64004E019000F248900000C2B30000C0700034
:100A74002903070002003700890307007049980022
:100A84004F0478000080FA00000006000400FA0019
:100A9400000F78001E00780040309000E20F5000F4
:100AA400040032001E0178001D03070084030700C0
:100AB400360037009E007800714890000034A00092
:100AC400F04898002F03070030003A001E00780019
:100AD40060889000100798001E009000E10F5000FD
:100AE4001D0032001E009000E20F50002100320071
:100AF400290307000A003E002203070023003A00EE
:100B04009E00780010002000E08898006011B80072
:100B14001E007800DED60200000000001B00370033
:100B240022030700190036001603070017003A00D5
:100B34009E00780020002000E08898001E007800C5
:100B440050299000E02990001E007800DED60200B3
:100B5400000000000D0037000F0307000B003600F3
:100B64001E007800D2D602000000000054030700E3
:100B7400060037000D03070004003E001E00780045
:100B8400D2D60200000000004D0307000080FA00E6
:100B9400000006000400FA004D0307001E00E000F8
:100BA40008003D009E009000D0C2B3008048780049
:100BB4009E0078000080EB000088B900000F7800E8
:100BC400030037009E009000B0C2B3008048780054
:100BD4001E0090008000E8001E00780042062000FD
:100BE400811F7800F602070001017800CF00780029
:100BF4000043B000804878001E00780042062000C0
:100C0400EF02070080007800400620000088B90049
:100C14001E0F10001E0090008080E8001E00780067
:100C2400A2002000811F7800E5020700010178007E
:100C3400CF0078000043B000804878001E00900088
:100C4400E3004000E0C2B300804878001E00780052
:100C5400A2002000DA0207006A00B9001E0F10008B
:100C64001E009000E40040001E0078000043B00025
:100C7400804878001E009000E50040000040EB0032
:100C8400804878000080FA0000000600D200FA00D4
:100C940000AF9800C0892A00C7000900305F7800BF
:100CA4008E0CB1000D0307000042B2000004E00006
:100CB40015003200800C20000E00400041892A00FB
:100CC40007000900315878008000B10009030700CB
:100CD40010007800810C20008E804000ADFF0700DA
:100CE400800C20000E004000801F780040962A00EF
:100CF400801F78000E007800EA0C0200000000005B
:100D0400E48757000800370020972A00801F7800E6
:100D140040962A00801F78000E007800EA0C02003A
:100D240000000000E4875700A80207000200010049
:100D3400EA020700624060000004E000090032009B
:100D44006000B800809FBE00B0972A00801F780022
:100D54000E007800EA0C020000000000E68757004D
:100D64000A003700E3020700A00090001000900082
:100D7400809FBE00B0972A00801F78000E00780084
:100D8400EA0C020000000000E68757008F0207000B
:100D940002000100D7020700C0009000300090005C
:100DA400809FBE00A0982A00801F78000E00780063
:100DB400EA0C020000000000E687570083020700E7
:100DC40002000100C5020700C7020700801F780067
:100DD40090992A00801F78000E007800EA0C020027
:100DE40000000000E48757007802070002000100B9
:100DF4007B0207000000D100BB020700801F7800BF
:100E0400709A2A00801F78000E007800EA0C020015
:100E140000000000E48757006C0207000200010094
:100E24006F0207004200DE00AF020700801F780057
:100E3400509B2A00801F78000E007800EA0C020004
:100E440000000000E4875700600207000200010070
:100E5400630207004500DE00A3020700801F78003C
:100E6400309C2A00801F78000E007800EA0C0200F3
:100E740000000000E487570054020700020001004C
:100E8400570207004300DE0097020700801F780026
:100E9400109D2A00801F78000E007800EA0C0200E2
:100EA40000000000E4875700480207000200010028
:100EB4004B0207004400DE008B020700801F78000D
:100EC400F09D2A00801F78000E007800EA0C0200D2
:100ED40000000000E48757003C0207000200010004
:100EE4000080FA0000000600CC00FA0050A7980029
:100EF4000E80E800D19E2A00C7000900315878000E
:100F0400800CB1000E81E8007A02070071004000F5
:100F1400801F780050AB2A00801F78000200780000
:100F2400EA0C020000000000E48757002F020700CB
:100F3400020001006F020700E02890005028900092
:100F44000E81E800809FBE0030AC2A00801F78002C
:100F540002007800EA0C020000000000E687570057
:100F64002202070002000100620207000050900004
:100F74000000FB008E80E800801F780020AD2A006E
:100F8400801F780001007800EA0C020000000000D5
:100F9400E48757001502070002000100550207000C
:100FA40020C890000000FB008E80E800801F7800BD
:100FB40000AE2A00801F780001007800EA0C0200CD
:100FC40000000000E4875700080207000200010047
:100FD40010C4B3001047980010C4B3001047980021
:100FE4001B0037009E409000F0CBB30000C04000CF
:100FF400004F78001E81FB0001F52F0066005700AA
:101004008100400002004100A002B000E0807800AE
:101014001E4090000000FB000E81E800811F780054
:10102400801F7800F0AE2A00801F7800020078004C
:10103400EA0C020000000000E6875700EB010700FD
:10104400020001001E4090000040E8001047980094
:101054009E40900050C4B30080CF5000E1FF3400A4
:1010640024020700407090000000FB008E80E8001E
:10107400801F7800E0AF2A00801F7800010078000C
:10108400EA0C020000000000E4875700D7010700C3
:1010940002000100DA0107000000D100DB010700B3
:1010A400801F7800C0B02A00801F780001007800FB
:1010B400EA0C020000000000E4875700CB0107009F
:1010C400020001000B020700206090000080FB007A
:1010D4008E80E800801F7800A0B12A00801F78006D
:1010E40001007800EA0C020000000000E4875700C9
:1010F400BE01070002000100C1010700C30107008F
:10110400801F780080B22A00801F780001007800D8
:10111400EA0C020000000000E4875700B301070056
:1011240002000100B60107004200DE00B70107001B
:10113400801F780060B32A00801F780001007800C7
:10114400EA0C020000000000E4875700A701070032
:10115400020001000080FA00000006000800FA0006
:101164001007980021079800320798000101200019
:101174003E009000FA24020001000000004F7800B5
:101184001E80FB000000E00005003A002100200062
:101194002E0090003A090200010000001000370000
:1011A4001E00900071004000BE009000180D020067
:1011B400000000009E0090000F0BB00000F52F000F
:1011C4000080470094010700807C020000000000BA
:1011D40000F52F0080874700AE7D0200000000006C
:1011E4000080FA00000006000A00FA0010079800C8
:1011F40021079800320798008C01070010C4B3003F
:1012040080CF5000100032008801070020C4B300D2
:1012140080CF50000C0032008401070030C4B300BA
:1012240080CF5000080032008001070040C4B300A2
:1012340080CF5000040032007C01070050C4B3008A
:1012440080CF500003003A001000200040079800AF
:10125400020037000000EB00400798000E489000A1
:10126400004F78001E80FB000000E00005003A00FB
:10127400210020002E0090003A0902000100000025
:101284000E003700690107001E00900041709800AD
:101294009E0090000F0BB00000F52F000080470067
:1012A4005D010700807C02000000000000F52F00B3
:1012B40080874700AE7D0200000000000080FA0035
:1012C400000006000C00FA0030079800410798005F
:1012D40052079800580107001000200010079800DA
:1012E40058010700E40F500003003C0055010700BB
:1012F4000000E00005003D00210020004E009000A9
:101304003A09020001000000490037004D010700BE
:10131400200798005E0090000000E80090407800EC
:10132400B0C2B30080CF500003003A001000200088
:10133400100798000E0037005E0090000000E800DF
:1013440090407800D0C2B30080CF500003003A0030
:101354000080EB00100798000500370021002000F2
:101364004E0090003A0902000100000030003700EE
:101374005E00900063004000104078008000FB0095
:10138400400620000088B900000178005E0090004B
:101394000080E800104078008000FB0000FD2F0072
:1013A40080804000803E20000088B9000001410098
:1013B4005E00900064004000104078000000FB00D4
:1013C4006A00B900800041005E00900065004000A2
:1013D400104078000000FB008080400000B32E0025
:1013E400008F40009E0078001E0090000088B90025
:1013F400000F78002F01070000004000A002B00099
:101404001EB07800BE0090000F0BB00000F52F0056
:101414000080470000010700807C020000000000FB
:1014240000F52F0080874700AE7D02000000000019
:101434000080FA00000006000600FA000701070019
:101444009040780010C4B30080CF500005003200F3
:10145400110020001E0090003A0902000100000063
:101464000F0037002E009000904078001E00780096
:10147400015098009E0078000F0BB00000F52F007B
:1014840000804700E4000700807C020000000000A8
:1014940000F52F0080874700AE7D020000000000A9
:1014A4000080FA00000006000600FA00A100070010
:1014B40006003200510020001E0090003A0902008C
:1014C40001000000DC0007000200370010002000CB
:1014D400200798002E0090000080FA00000006000B
:1014E4000600FA00930007000600320051002000B5
:1014F4001E0090003A09020001000000CE0007001F
:101504000D0037001E0078007048900064406000B1
:101514000004E00006003A00C10020001E00900014
:101524003A09020001000000C3000700020037006E
:1015340010002000200798002E0090000080FA0080
:10154400000006000400FA007C00070002003200DC
:1015540010C0B3003047980080000700000140002D
:10156400C3109000D0FF2F00810007000F0BB000C4
:1015740000F52F0000804700A7000700807C0200D0
:101584000000000000F52F0080874700AE7D0200B8
:10159400000000000080FA00000006000600FA00C7
:1015A400AE000700804078001E007800216098009B
:1015B4009E0078000F0BB00000F52F00008047005C
:1015C40095000700807C02000000000000F52F0059
:1015D40080874700AE7D0200000000000080FA0012
:1015E400000006000400FA00540007000200320064
:1015F40010C0B30030479800580007004201DD00D6
:10160400C3109000B0FF2F00590007000F0BB0006B
:1016140000F52F00008047007F000700807C020057
:101624000000000000F52F0080874700AE7D020017
:10163400000000000080FA00000006000600FA0026
:10164400A3000700424798001E00780070489000ED
:101654000042B2000004E00005003A0071002000DE
:101664001E0090003A090200010000000E0037003D
:10167400CE4090001E00780021C898009E0078009B
:101684000F0BB00000F52F00008047006200070038
:10169400807C02000000000000F52F0080874700D6
:1016A400AE7D0200000000000080FA000000060089
:1016B4000400FA00000F7800214798002E409000A3
:1016C400614060001E0178000080FB00E1016000C1
:1016D400C2109000E0FF2F00008060000300700043
:1016E400401198009E0078000F0BB00000F52F0009
:1016F4000080470048000700807C020000000000D2
:1017040000F52F0080874700AE7D02000000000036
:101714000080FA0000000600704998004E01900015
:10172400F248900070CFB30000C060007049980088
:10173400000006006600070012003700000F780062
:10174400214798002E4090000080FB008040EB0071
:10175400314798000000E000000006009E01780078
:10176400BE4090000180FB006100600000000600A4
:101774000080600002007000C01198009E00780094
:10178400000006001E00780070489000624060006F
:101794000004E000000006001E007800E0909000C5
:1017A400E0232000808F5000000006001E00780017
:1017B400E0909000502D2000808F50000000060023
:1017C400110009000200D800000006000EA89000D5
:1017D4001001900011C0B3000E0078000000060054
:1017E4003E0007000080FB00000006005EA09000A1
:1017F400100190000E80E80011C0B3000000060044
:101804003C0007004010900000000600360007006E
:101814008E80E800000006005700090031187800A7
:10182400000BB100010BB100000006003E00900067
:1018340090407800000006000000EB0020079800AC
:10184400000006005E009000104078008000FB005D
:10185400F0FB2F0000804000000006001C00070081
:10186400220798002E009000000006009E007800D9
:101874000040EB000000060000C0600070499800C2
:101884001E017800F2489000000006001E01780056
:1018940000102E00010005009E0078006005050080
:1018A4004E019000F2489000F0CDB30000C06000FB
:1018B400000006002E009000BE009000000006000C
:1018C4009E0078000000EB00E0889800000006000D
:1018D400000F7800110798000000060005000700BB
:1018E4007048900000000600614060000080FB002A
:1018F4000000060001F52F006600570001004000BB
:10190400000006000400FA00000F78001107980098
:101914001E0090000000E0000F003A00217D21002D
:10192400C0192A00801F780030012000801F780031
:10193400901A2A00801F7800701B2A00801F7800EC
:1019440001007800720C020000000000E8875700D4
:10195400BE0C0200000000001E0078009E009000F3
:10196400110098009E00780000C3B300C0409800A6
:101974009E00780000C3B300D04098009E00780019
:1019840000C3B300E04098001E00900082150200DE
:10199400010000000080FA00000006000200FA00C6
:1019A400000F78009E007800B0C4B300804878002F
:1019B4000080FA00000006000200FA00000F780020
:1019C400E103070070B4800081B48000800F5100EF
:1019D400818F590007003200DB03070072B48800CE
:1019E40083B48800D80307000200BE003C1602003E
:1019F4000100000090B48000A1B48000E00F50000A
:101A0400E08F5800070032003904070092B48800C0
:101A1400A3B48800360407000200BE000A160200C0
:101A240001000000D20307008080FB00B0B48000F6
:101A3400808F50000D003200CD0307000080FB00B2
:101A4400B0B48800B0B480000000E00004003200AC
:101A54000040EB00ACE2020000000000030037008D
:101A64000040EB0092E20200000000000080FA0057
:101A740000000600CC00FA0050A798000E00E80011
:101A8400511D2A00C700090031587800800CB100AC
:101A94008E00E8000000EB00801F7800200020008A
:101AA400801F780010002000801F7800D0292A00B1
:101AB400801F780001007800EA0C0200000000009A
:101AC400E88757001404070002000100EE03070032
:101AD4001040780015040700801F7800102B2A009E
:101AE400801F780001007800EA0C0200000000006A
:101AF400E487570008040700020001000E00E80014
:101B0400F12B2A000C00090031587800D000B100F4
:101B14000104070002000100070407008E00E8002A
:101B2400831F7800841F7800821F7800801F78004C
:101B3400C02C2A00801F780001007800EA0C020003
:101B440000000000EA875700F303070002000100C9
:101B5400CD03070040D89200F4030700801F7800EB
:101B6400302E2A00801F780001007800EA0C020061
:101B740000000000E4875700E703070002000100AB
:101B8400C103070070E89000E8030700801F780095
:101B9400102F2A00801F780001007800EA0C020050
:101BA40000000000E4875700DB0307000200010087
